:100000000C9443240C9470240C9470240C9470244D
:100010000C9470240C9470240C9470240C94702410
:100020000C9470240C9470240C9470240C94702400
:100030000C9470240D9406270C9470240C94702456
:100040000C9470240C944DBE0C9470240C94702469
:100050000C9470240C9470240C9498740D949F2527
:100060000C9470240C9402950C9470240C947024BD
:100070000C9470240C9470240C9470240C947024B0
:100080000C9470240C9470240C9470240C947024A0
:100090000C9470240C9470240C9470240D94031C04
:1000A0000C9470240C9470240C9470240C94702480
:1000B0000C9470240C9470240C9470240C94702470
:1000C0000C9470240C9470240C9470240C94702460
:1000D0000C9470240C9470240C9470240C94702450
:1000E0000C947024084AD73B3BCE016E84BCBFFD04
:1000F000C12F3D6C74319ABD56833DDA3D00C77FF8
:1001000011BED9E4BB4C3E916BAAAABE0000008090
:100110003F05A84CCDB2D44EB93836A9020C50B91F
:10012000918688083CA6AAAA2ABE000000803F004B
:10013000060900FE06018902FE20FFFE07FE06FEFC
:10014000000000060007010606060200808080808D
:100150000080030303060103A0A0A0050707060013
:10016000FF5050F850F850500509090600FE207065
:10017000A8A07028A870200608080600FF40A8481C
:1001800010204854080507070600FF60909060980B
:1001900090680103030602038080800207070602BD
:1001A000FF408080808080400207070602FF804079
:1001B00040404040800505050600008850F8508802
:1001C0000505050600002020F82020020404060290
:1001D000FEC0404080050101060002F8020202064E
:1001E0000200C0C0040606060100101020408080F6
:1001F00004060606010060909090906003060606D3
:10020000010040C0404040E0040606060100609046
:10021000102040F0040606060100F020601010E0F7
:1002200005060606000010305090F8100406060679
:100230000100F080E01010E0040606060100608076
:10024000E0909060040606060100F0101020404087
:1002500004060606010060906090906004060606A1
:100260000100609090701060020505060200C0C099
:1002700000C0C00207070602FEC0C000C0404080A8
:1002800005050506000018608060180503030600D8
:1002900001F800F8050505060000C0300830C0046C
:1002A0000707060100609010604000400506060642
:1002B00000007090A8B0807005060606000020506F
:1002C00088F88888050606060000F088F08888F01F
:1002D0000406060601006090808090600406060611
:1002E0000100E090909090E0040606060100F08086
:1002F000E08080F0040606060100F080E080808047
:10030000040606060100609080B0906004060606B0
:1003100001009090F0909090030606060100E040E6
:10032000404040E0050606060000381010109060BE
:1003300004060606010090A0C0A0909004060606E0
:1003400001008080808080F005060606000088D8C5
:10035000A8A8888804060606010090D0B090909066
:100360000506060600007088888888700406060660
:100370000100E09090E080800407070601FF609094
:1003800090D0B06010040606060100E09090E09066
:100390009004060606010060904020906005060665
:1003A000060000F820202020200406060601009008
:1003B0009090909060040606060100909090F06086
:1003C000600506060600008888A8A8D888050606E5
:1003D0000600008850202050880506060600008888
:1003E0008850202020040606060100F010204080DE
:1003F000F0030606060100E080808080E004060627
:10040000060100808040201010030606060100E06F
:1004100020202020E005030306000320508805016A
:10042000010600FEF80202020602048040040404F1
:10043000060100709090700406060601008080E0BE
:100440009090E004040406010070808070040606A9
:100450000601001010709090700404040601006002
:10046000B0C070040606060100205040E040400481
:1004700006060601FE6090907010600406060601F4
:10048000008080E09090900306060601004000C0C6
:100490004040E00308080601FE200060202020A064
:1004A000400406060601008080A0C0A09003060656
:1004B000060100C040404040E0050404060000D0B2
:1004C000A8A888040404060100E0909090040404A5
:1004D000060100609090600406060601FEE0909020
:1004E000E080800406060601FE70909070101004F3
:1004F0000404060100A0D0808004040406010070FA
:10050000C030E00406060601004040E040502004F0
:100510000404060100909090700404040601009009
:1005200090606005040406000088A8A85004040434
:10053000060100906060900406060601FE9090900F
:10054000709060040404060100F02040F0030707E7
:10055000060100204040804040200107070602FFBE
:1005600080808080808080030707060100804040F3
:100570002040408004020206010350A0FFFFFFFF5D
:10058000FFFFFFFFFFFFFFFFFFFFFFFFFFFFFFFF7B
:10059000FFFFFFFFFFFFFFFFFFFFFFFFFF00000068
:1005A00006000701060606020080008080808004A5
:1005B00006060601FF2070A0A070200507070600B0
:1005C000FF304840F04040F8050505060000A850FF
:1005D0008850A80506060600008850F820F820017B
:1005E00007070602FF8080800080808004070706DE
:1005F00001FF708060906010E0030101060105A01A
:10060000060707060000788494A4948478030505FF
:1006100006010160A06000E0050505060000285005
:10062000A05028040303060100F010100401010685
:100630000102F00607070600007884B4A4A48478B9
:10064000040101060105F004030306010260906045
:100650000507070600FF2020F8202000F803050505
:1006600006010140A02040E0030505060101C0206D
:100670004020C00202020602044080040505060173
:10068000FF9090B0D08005060606000078E8E86884
:100690002828010101060202800202020602FE4031
:1006A0008003050506010140C04040E00305050642
:1006B000010140A04000E0050505060000A050280B
:1006C00050A00508080600FF40C040507030781068
:1006D0000508080600FF40C04050680810380508AB
:1006E000080600FFC0204030F030781004070706ED
:1006F0000100200020608090600507070600004090
:100700002020507088880507070600001020205020
:1007100070888805070706000020502050708888E0
:100720000507070600002850205070888805070735
:10073000060000500020507088880507070600005A
:100740002050205070888805060606000078A0F02A
:10075000A0A0B80408080601FE6090808090602088
:10076000400407070601004020F080E080F0040705
:10077000070601002040F080E080F0040707060132
:10078000002050F080E080F00407070601005000D0
:10079000F080E080F00307070601008040E0404061
:1007A00040E00307070601002040E0404040E0032E
:1007B000070706010040A0E0404040E003070706AD
:1007C0000100A000E0404040E00506060600007081
:1007D00048E848487004070706010050A090D0B0D0
:1007E00090900407070601004020609090906004FC
:1007F00007070601002040609090906004070706FC
:10080000010020506090909060040707060100509E
:10081000A06090909060040707060100500060906F
:100820009090600505050600008850205088040857
:10083000080601FF1070B0B0D0D0E08004070706B2
:10084000010040209090909060040707060100206E
:10085000409090909060040707060100205090900F
:1008600090906004070706010050009090909060FF
:1008700005070706000010208850202020040606E7
:1008800006010080E09090E080040606060100600A
:1008900090A0A090A00407070601004020007090DF
:1008A00090700407070601002040007090907004CB
:1008B000070706010020500070909070040707069B
:1008C000010050A0007090907004060606010050D0
:1008D000007090907004070706010020502070906F
:1008E000907005040406000070A8B078040606069F
:1008F00001FE708080702040040707060100402040
:100900000060B0C07004070706010020400060B01E
:10091000C07004070706010020500060B0C07004DA
:100920000606060100500060B0C07003070706010C
:1009300000804000C04040E003070706010020405F
:1009400000C04040E003070706010040A000C0408F
:1009500040E0030606060100A000C04040E0040796
:1009600007060100306010709090600407070601D0
:100970000050A000E090909004070706010040207E
:10098000006090906004070706010020400060901E
:1009900090600407070601002050006090906004FA
:1009A000070706010050A00060909060040606064C
:1009B00001005000609090600505050600002000D1
:1009C000F8002004040406010070B0D0E00407071A
:1009D0000601004020009090907004070706010077
:1009E00020400090909070040707060100205000FE
:1009F0009090907004060606010050009090907050
:100A00000409090601FE2040009090907090600457
:100A100008080601FE8080E09090E08080040808CD
:100A20000601FE500090909070906000060900FE54
:100A3000070199032B20FFFE08FE07FE00000006B9
:100A4000000001070706020080808080800080038C
:100A50000303060104A0A0A00507070600005050EC
:100A6000F850F850500507070600002070A07028C5
:100A7000702005070706000048A8502050A89005E0
:100A8000070706000040A0A040A8906801030306E5
:100A900002048080800307070601002040808080D8
:100AA00040200307070601008040202020408005E9
:100AB00005050600018850F8508805050506000167
:100AC0002020F820200303030601FF604080050179
:100AD00001060003F80303030601FF40E040050799
:100AE0000706000008081020408080050707060060
:100AF00000205088888850200507070600002060E5
:100B0000A0202020F8050707060000708808304064
:100B100080F8050707060000F808103008887005FF
:100B2000070706000010305090F810100507070660
:100B30000000F880B0C8088870050707060000307C
:100B40004080B0C88870050707060000F80810103C
:100B5000204040050707060000708888708888706C
:100B600005070706000070889868081060030707EB
:100B70000601FF40E0400040E0400307070601FF98
:100B800040E040006040800407070601001020405C
:100B900080402010050303060002F800F804070750
:100BA0000601008040201020408005070706000055
:100BB0007088102020002005070706000070889824
:100BC000A8B0807005070706000020508888F888C4
:100BD00088050707060000F04848704848F00507F8
:100BE000070600007088808080887005070706006F
:100BF00000F04848484848F0050707060000F8801C
:100C000080F08080F8050707060000F88080F080FB
:100C1000808005070706000070888080988870052E
:100C20000707060000888888F88888880307070671
:100C30000100E04040404040E00507070600003862
:100C40001010101090600507070600008890A0C0E3
:100C5000A09088050707060000808080808080F8CB
:100C60000507070600008888D8A888888805070730
:100C70000600008888C8A89888880507070600002D
:100C800070888888888870050707060000F08888C3
:100C9000F08080800508080600FF7088888888A892
:100CA0007008050707060000F08888F0A090880506
:100CB000070706000070888070088870050707061F
:100CC0000000F820202020202005070706000088CB
:100CD00088888888887005070706000088888850FB
:100CE000505020050707060000888888A8A8D888E3
:100CF00005070706000088885020508888050707E8
:100D000006000088885020202020050707060000E4
:100D1000F80810204080F8030707060100E08080F3
:100D2000808080E0050707060000808040201008D2
:100D300008030707060100E02020202020E005032B
:100D4000030600042050880501010600FFF8020296
:100D50000206020680400505050600007008788836
:100D6000780507070600008080B0C888C8B0050570
:100D700005060000708880887005070706000008D7
:100D80000868988898680505050600007088F8804E
:100D900070050707060000304840F0404040050756
:100DA000070600FE7888887808887005070706001F
:100DB000008080B0C88888880307070601004000CB
:100DC000C0404040E00409090601FE100030101048
:100DD0001090906005070706000080808890E090E2
:100DE00088030707060100C04040404040E0050579
:100DF00005060000D0A8A8A888050505060000B0D3
:100E0000C8888888050505060000708888887005F0
:100E100007070600FEB0C888C8B08080050707062F
:100E200000FE68988898680808050505060000B067
:100E3000C880808005050506000070807008F005F8
:100E400007070600004040F0404048300505050611
:100E50000000888888986805050506000088885085
:100E600050200505050600008888A8A8500505053E
:100E700006000088502050880507070600FE888875
:100E80009868088870050505060000F8102040F8ED
:100E9000040707060100304020C02040300107074A
:100EA00006020080808080808080040707060100A1
:100EB000C02040304020C005030306000448A8902D
:100EC000000000010000000000010000000000011F
:100ED0000000000000010000000000010000000010
:100EE00000010000000000010000000000010000FF
:100EF00000000001000000000001000000000001EF
:100F000000000000000100000000000100000000DF
:100F100000010000000000010000000000010000CE
:100F200000000001000000000001000000000001BE
:100F300000000000000100000000000100000000AF
:100F4000000100000000000100000000000100009E
:100F5000000000010000000000010000000000018E
:100F6000000000000001000000000001000000007F
:100F7000000100000000000100000000000100006E
:100F80000000000100000000000600000107070645
:100F90000200800080808080800507070600FF2017
:100FA00078A0A0A07820050707060000304840E0A0
:100FB0004048B00505050600008870507088050897
:100FC000080600FF88885020F82020200107070627
:100FD0000200808080008080800508080600FF7085
:100FE00080E09048380870030101060107A005075A
:100FF000070600007088A8C8A888700406060601C5
:10100000017090B05000F0060505060000244890DD
:101010004824040202060102F01004010106010343
:10102000F00507070600007088E8C8C88870050149
:1010300001060007F803030306010440A04005066B
:10104000060600002020F82020F80405050601030C
:1010500060902040F0040505060103E0106010E0F8
:1010600002020206020640800506060600FF888886
:1010700088C8B08005070706000078E8E8682828D7
:1010800028010101060203800202020602FE4080DE
:1010900003050506010340C04040E00406060601C2
:1010A000016090906000F00605050600009048245D
:1010B00048900609090600FF40C04040E40C143C7B
:1010C000040609090600FF40C04040E81404081C5B
:1010D0000509090600FFC0204020C8182878080527
:1010E0000707060000200020204088700508080639
:1010F00000004020708888F88888050808060000ED
:101100001020708888F8888805080806000020509C
:10111000708888F8888805080806000048B070883C
:1011200088F888880508080600005000708888F84C
:1011300088880508080600002050708888F888888C
:101140000607070600003C50909CF0909C0509099A
:101150000600FE70888080808870204005080806A0
:10116000000040F88080F08080F805080806000044
:1011700010F88080F08080F805080806000020F84C
:101180008080F08080F805080806000050F8808014
:10119000F08080F80308080601008040E0404040ED
:1011A00040E00308080601002040E040404040E0E5
:1011B00003080806010040A0E040404040E003086A
:1011C00008060100A000E040404040E00507070697
:1011D0000000F04848E84848F005080806000028E4
:1011E0005088C8A898888805080806000040207024
:1011F0008888888870050808060000102070888894
:101200008888700508080600002050708888888843
:1012100070050808060000285070888888887005C6
:101220000808060000500070888888887005050549
:1012300006000088502050880507070600007098B7
:1012400098A8C8C87005080806000040208888884B
:10125000888870050808060000102088888888881B
:1012600070050808060000205000888888887005EE
:1012700008080600005000888888888870050808DB
:10128000060000102088885020202005070706004F
:101290000080F088F08080800507070600007088D5
:1012A00090A09088B0050808060000402000700853
:1012B00078887805080806000010200070087888F3
:1012C0007805080806000020500070087888780526
:1012D000080806000028500070087888780507077D
:1012E000060000500070087888780508080600009D
:1012F00020502070087888780605050600007814CC
:101300007C907C0507070600FE708880887020406E
:101310000508080600004020007088F88070050865
:10132000080600001020007088F880700508080684
:1013300000002050007088F8807005070706000044
:1013400050007088F8807003080806010080400093
:10135000C0404040E0030808060100408000C04053
:101360004040E003080806010040A000C0404040A3
:10137000E0060A0A0600FEA4A800FC84808080849F
:10138000FC060A0A0600FE549400FC84040404844B
:10139000FC050808060000285000B0C888888805A9
:1013A00008080600004020007088888870040A0A37
:1013B0000602FE30408090909090909090040A0A2F
:1013C0000600FEC020109090909090909006070725
:1013D000060001448C8C8480403C0607070600010F
:1013E00088C4C4840408F00505050600012000F83F
:1013F000002005080806000040F0C888889878108A
:10140000050808060000E0F88888888888F805053F
:10141000050600012030F8302005080806000020ED
:1014200070F820202020E00509090600FF2070A8A0
:10143000A8B8888850200509090600FFE080C0B0E0
:10144000A8A83028280509090600FFF8A888888878
:101450008888A8F8050A0A0600FE205050505088D7
:10146000A8A8887000000000000000000000000034
:101470007FFFE0000000000000000000000000709E
:1014800000E0000000000000000000000000630C0D
:1014900060000000000000000000000000470E2077
:1014A0000000000000000000000000004F0F2000BE
:1014B00000000000000000000000005F0FA000001E
:1014C000000000000000000000005E07A07F800018
:1014D000000000000000410400406020FFC0000048
:1014E000000000000020820040F020FFC00000004B
:1014F0000000000020820040F020FFC0000000003B
:101500000000004104004060207F800000000000D7
:1015100000008208005E07A07F800000000000003D
:10152000010410005F0FA0FFC000000000000001D8
:101530000410004F0F20FFC00000000000000082D8
:101540000800470E20FFC00000000000000041041A
:1015500000630C603F00000000000000000000007D
:101560007000E01E0000000000000001FFFF807F0F
:10157000FFE00C0000000000000001FFFF80000001
:10158000000000000000000000000000007FFFE0FD
:101590000000000000000000000000007000E000FB
:1015A000000000000000000000000061F860000082
:1015B0000000000000000000000041F820000000D2
:1015C00000000000000000000040F02000000000CB
:1015D000000000000000000040602000000000004B
:1015E000000000000000005801A07F800000000003
:1015F0000000004104005C63A0FFC0000000000088
:1016000000002082005EF7A0FFC000000000000084
:10161000002082005EF7A0FFC00000000000000074
:101620004104005C63A07F80000000000000008295
:1016300008005801A07F8000000000000001041095
:1016400000406020FFC00000000000000104100006
:1016500040F020FFC00000000000000082080041B0
:10166000F820FFC00000000000000041040061F805
:10167000603F00000000000000000000007000E07B
:101680001E0000000000000001FFFF807FFFE00C53
:101690000000000000000001FFFF80000000590072
:1016A0002D2D3A2D2D20202D2D2E2D2500202020D2
:1016B0003130302500202000B02000B02000000094
:1016C000000000000000000000000000000000001A
:1016D000000000000000000000000000000000000A
:1016E000000C000000000000000C000000000000E2
:1016F00000120000000000000023000000000000B5
:101700000021000000000000004C800000000000EC
:10171000005E800000000000009240000000000019
:1017200000A1400000000000012120000000000096
:10173000027F900000000000020010000000000086
:1017400007FFF8000000000004000800000000008F
:10175000080004000000000008000600000000006F
:101760001000020000000000301E01000000000018
:10177000207F81000000000041FFE08000000000A9
:1017800043FCF08000000000873B7840000000012F
:101790008EDBFC60000000010FEBCC20000000029B
:1017A0001FEDB610000000021FDEB610000000049E
:1017B00039CD7F080000000436E0FF080000000873
:1017C0007EC0BB84000000187F005D860000001012
:1017D0007FC0ED82000000203CC0730100000020AB
:1017E0003B337F01000000701BE77E03800000C8D0
:1017F0001DEEDE04C00000880FDEDC044000012482
:101800000FDF3C092000012607DBF81920000272D7
:1018100003E7F0139000025101FFE02290000489D9
:10182000007F802448000904801E004824000BFE2D
:10183000400000DFF40010004000008002001FFFA5
:10184000FFFFFFFFFE00000000000000000000009E
:101850000000000000000000000000000000102256
:10186000103C3C0E1F001022100422110400102214
:10187000100822110400102210083C11040010224C
:1018800010102211040010221020221104001E1C2E
:101890001E3C3C0E040000000000000000000000A0
:1018A0000000000000000000000000000000000038
:1018B0000000000000000000000000000000000028
:1018C0000000000000000000000000000000000018
:1018D0000000000000000000000000000000000008
:1018E00000000000000000000000000000000000F8
:1018F0000000000000000000000000004E6F2053B8
:10190000442063617264005072696E742066726F65
:101910006D2053440053746F70207072696E7400B0
:10192000526573756D65207072696E7400506175D3
:101930007365207072696E7400436F6E66696775B7
:10194000726174696F6E0054656D70657261747553
:101950007265004D6F76656D656E740054756E65C9
:1019600000496E666F2073637265656E0050726920
:101970006E742066726F6D205344005072696E74ED
:101980002066726F6D20534400F92E2E004D616960
:101990006E004D3234004D32332025730050726991
:1019A0006E742061626F7274656400526573746F47
:1019B000726520746F20466163746F7279004C6F9A
:1019C00061642073657474696E6773005361766532
:1019D0002073657474696E677300416476616E6329
:1019E00065642073657474696E6773004D61696E18
:1019F000004573746570732F6D6D00457374657069
:101A0000732F6D6D005A73746570732F6D6D005A6E
:101A100073746570732F6D6D005973746570732FD7
:101A20006D6D005973746570732F6D6D005873740C
:101A30006570732F6D6D005873746570732F6D6DC5
:101A400000412D7265747261637400412D7265747A
:101A50007261637400416D6178206500416D617849
:101A6000206500416D6178207A00416D6178207AAF
:101A700000416D6178207900416D617820790041E5
:101A80006D6178207800416D61782078005654723D
:101A90006176206D696E005654726176206D696EB4
:101AA00000566D696E00566D696E00566D61782046
:101AB0006500566D6178206500566D6178207A006A
:101AC000566D6178207A00566D6178207900566DE8
:101AD0006178207900566D6178207800566D6178C4
:101AE00020780056652D6A65726B0056652D6A6513
:101AF000726B00567A2D6A65726B00567A2D6A6594
:101B0000726B005678792D6A65726B005678792D64
:101B10006A65726B00416363656C00416363656C69
:101B2000005A204F666673657400436F6E6669677E
:101B300075726174696F6E005A204F6666736574C2
:101B4000007F80FFC0FFC0FFC07F807F80FFC0FF9D
:101B5000C0FFC03F001E000C00FFFFFF001FE000A1
:101B6000303000400800800401800601000207C0F8
:101B700002038002010002000002000002000006D1
:101B8000000004000008003030001FE006000600DE
:101B900006000600060006003FC01F800F0006007A
:101BA00007F8000C0C0010020020010060018040CA
:101BB00000804003E04001C0400080400000400041
:101BC000006000002000001000000C0C0007F8006E
:101BD00006000F001F803FC006000600060006003A
:101BE0000600060006000F001F803FC0060006002A
:101BF00006000600060006000600060006000600B5
:101C000006000600060006000600060006000600A4
:101C10003FC01F800F000600436F6F6C646F776ECC
:101C20000046616E2073706565640046616E2073C6
:101C3000706565640042656400426564004E6F7AB9
:101C40007A6C65004E6F7A7A6C65004D61696E0042
:101C50004D6F76652061786973004D3834004469B2
:101C60007361626C65207374657070657273004790
:101C70003238004175746F20686F6D65004D616981
:101C80006E004D6F766520302E316D6D004D6F7694
:101C90006520316D6D004D6F76652031306D6D00C2
:101CA0004D6F76656D656E74004578747275646508
:101CB00072004D6F7665205A004D6F766520590091
:101CC0004D6F76652058004D6F7665206178697399
:101CD000004578747275646572005A0059005800A6
:101CE0004D363030004368616E67652066696C610F
:101CF0006D656E74004C61796572004C6179657236
:101D00000046616E2073706565640046616E2073E5
:101D10007065656400466C6F7700466C6F770042B3
:101D2000656400426564004E6F7A7A6C65004E6FA0
:101D30007A7A6C65005370656564005370656564FC
:101D4000004D61696E004C756C7A426F742054418D
:101D50005A20362072656164792E004361726420D6
:101D6000696E736572746564004D3330302053368C
:101D700039382050323030004D3330302053363532
:101D80003920503230300043616E6E6F7420656EC2
:101D9000746572207375626469723A20004D323442
:101DA000004D3233202573006175746F25692E67ED
:101DB000006572726F722077726974696E67207441
:101DC0006F2066696C65004E6F74205344207072FA
:101DD000696E74696E67002F005344207072696EDB
:101DE00074696E67206279746520002E0044656C0A
:101DF0006574696F6E206661696C65642C20466944
:101E00006C653A200046696C652064656C65746594
:101E1000643A002E006F70656E206661696C6564BF
:101E20002C2046696C653A200057726974696E67A8
:101E300020746F2066696C653A20002E006F706513
:101E40006E206661696C65642C2046696C653A2079
:101E5000002E006F70656E206661696C65642C20D1
:101E600046696C653A200046696C652073656C654F
:101E700063746564002053697A653A200046696C92
:101E800065206F70656E65643A20002E006F706586
:101E90006E206661696C65642C2046696C653A2029
:101EA000004E6F772066726573682066696C653ACC
:101EB00020004E6F7720646F696E672066696C65DD
:101EC0003A20002220706F73002220706172656ECC
:101ED000743A2200535542524F5554494E452043BF
:101EE000414C4C207461726765743A2200747279B7
:101EF000696E6720746F2063616C6C207375622D4E
:101F000067636F64652066696C65732077697468C0
:101F100020746F6F206D616E79206C6576656C73CF
:101F20002E204D4158206C6576656C2069733A000F
:101F300053442063617264206F6B006F70656E5252
:101F40006F6F74206661696C656400766F6C756D87
:101F5000652E696E6974206661696C65640053441E
:101F600020696E6974206661696C004572723A205E
:101F70004D415854454D50204245440054656D70C4
:101F8000657261747572652068656174656420624C
:101F90006564207377697463686564206F66662E74
:101FA000204D415854454D502074726967676572E1
:101FB0006564202121004572723A204D494E5445F6
:101FC0004D50003A204578747275646572207377BD
:101FD000697463686564206F66662E204D494E54AF
:101FE000454D5020747269676765726564202100F1
:101FF0004572723A204D415854454D50003A2045A3
:102000007874727564657220737769746368656447
:10201000206F66662E204D415854454D50207472F5
:1020200069676765726564202100544845524D41D7
:102030004C2052554E4157415900546865726D61AC
:102040006C2052756E617761792C20737973746599
:102050006D2073746F7070656421204865617465CC
:10206000725F49443A2000202D20496E76616C69E8
:1020700064206578747275646572206E756D626532
:10208000722021001000C90210012C014001220120
:1020900070011801B0010E01F00104015002FA00B4
:1020A000B002F0003003E600D003DC009004D20060
:1020B0007005C800A006BE000008B400B009AA0060
:1020C000D00BA000600E960060118C0000158200FD
:1020D00020197800C01D6E00A0226400B0275A00AD
:1020E000902C500000314600E0343C0010383200A3
:1020F000903A2800603C1E00A03D1400803E0A007B
:10210000203F00001000AD0330016A0150022B0196
:1021100070030A019004F500B005E500D006D80070
:10212000F007CE001009C500300ABE00500BB70002
:10213000700CB100900DAB00B00EA600D00FA20045
:10214000F0109D0010129900301395005014920069
:1021500070158E0090168B00B0178700D018840081
:10216000F0198100101B7E00301C7B00501D79008F
:10217000701E7600901F7300B0207000D0216E009A
:10218000F0226B00102469003025660050266300A1
:102190007027610090285E00B0295C00D02A5900A9
:1021A000F02B5600102D5400302E5100502F4E00B1
:1021B00070304B0090314800B0324500D0334200BF
:1021C000F0343E0010363B003037370050383300D3
:1021D00070392E00903A2900B03B2300D03C1B0000
:1021E000F03D1100103F0100F03F000048656174B0
:1021F000696E67206661696C6564005049442041DE
:1022000075746F74756E652066696E697368656450
:10221000212050757420746865206C617374204BA4
:10222000702C204B6920616E64204B6420636F6EBC
:102230007374616E74732066726F6D2061626F7665
:102240006520696E746F20436F6E66696775726191
:1022500074696F6E2E6800504944204175746F7424
:10226000756E65206661696C6564212074696D65B1
:102270006F75740020403A006F6B20543A006F6B0A
:1022800020423A00504944204175746F74756E6560
:10229000206661696C6564212054656D70657261AA
:1022A0007475726520746F6F206869676800204BD1
:1022B000643A2000204B693A2000204B703A2000FD
:1022C00020436C617373696320504944200020549B
:1022D000753A2000204B753A2000206D61783A2035
:1022E00000206D696E3A200020643A200020626967
:1022F00061733A20007C3C3E5E2B3D3F2F5B5D3B93
:102300002C2A225C0020746F6F206C6F6E67206532
:102310007874727573696F6E2070726576656E740D
:1023200065640020636F6C642065787472757369EE
:102330006F6E2070726576656E7465640045313A23
:10234000200045303A20005A3A2000593A200058DF
:102350003A20004D53312C4D53322050696E730A90
:102360000024F404D9201BC40C5C0E9804C4095F3B
:102370000265077101F405F900FB04B30048048706
:1023800000C10369005803550003034500BE023A2B
:10239000008402310053022A002902250004022091
:1023A00000E4011C00C8011900AF011700980114D6
:1023B0000084011300710110006101100051010E31
:1023C0000043010D0036010B002B010B0020010B17
:1023D00000150109000C01090003010800FB0008B9
:1023E00000F3000800EB000700E4000600DE000632
:1023F00000D8000600D2000600CC000500C700058A
:1024000000C2000500BD000400B9000400B50004CE
:1024100000B1000400AD000400A9000400A5000301
:1024200000A20003009F0004009B0003009800032B
:10243000009500020093000300900003008D00024D
:10244000008B000300880002008600020084000365
:1024500000810002007F0002007D0002007B00027C
:10246000007900020077000100760002007400028B
:102470000072000100710002006F0002006D000197
:10248000006C0002006A00010069000200670001A0
:1024900000660001006500010064000200620001A6
:1024A0000061000100600001005F0002005D0001AA
:1024B000005C0001005B0001005A000100590001AE
:1024C00000580001005700010056000100550001AE
:1024D00000540001005300000053000100520001AD
:1024E0000051000100500001004F0001004E0000AB
:1024F000004E0001004D0001004C0001004B0000A7
:10250000004B0001004A00010049000100480000A2
:10251000004800010047000100460000004600019D
:102520000045000000450001004400010043000098
:102530000043000100420000004200010041000091
:102540000041000100400001003F0000003F000189
:10255000003E0000003E0001003D0000003D000183
:10256000003C0000003C0000003C0001003B00007B
:10257000003B0001003A0000003A00010039000071
:102580000039000100380000003800000038000168
:102590000037000000370001003600000036000060
:1025A0000036000100350000003500000035000154
:1025B000003400000034000000340001003300004B
:1025C0000033000000330001003200000032000040
:1025D0000032000100310000003100000031000134
:1025E000003000000030000000300001002F00002B
:1025F000002F0000002F0000002F0001002E00001F
:10260000002E0000002E0001002D0000002D000013
:10261000002D0000002D0001002C0000002C000007
:10262000002C0000002C0001002B0000002B0000FB
:10263000002B0000002B0001002A0000002A0000EF
:10264000002A0000002A00010029000000290000E3
:1026500000290000002900000029000100280000D6
:1026600000280000002800000028000000280001C9
:1026700000270000002700000027000000270000BE
:1026800000270001002600000026000000260000B0
:1026900000260000002600010025000000250000A3
:1026A0000025000000250000002500000025000195
:1026B000002400000024000000240000002400008A
:1026C000002400010023000000230000002300007C
:1026D000002300000023000000230000002300016D
:1026E0000022000000220000002200000022000062
:1026F0000022000000220001002100000021000053
:102700000021000000210000002100000021000045
:102710000021000100200000002000000020000037
:102720000020000000200000002000000020000029
:1027300000200001001F0000001F0000001F00001B
:10274000001F0000001F0000001F0000001F00010C
:10275000001E0000001E0000001E0000001E000001
:102760000024F4D43050C38E20C2A24017828B7054
:1027700011127A910D816CD90AA861E108C75866D7
:1027800007615143061E4B5D05C145A7041A41115F
:1027900004093D9803713931034036DB02653391FA
:1027A00002D4305402802E1D02632CEE01752AC51E
:1027B00001B028A001102781018F2564012B244B33
:1027C00001E0223401AC211F018D200D01801FFC8E
:1027D00000841EED00971DDF00B81CD200E61BC66A
:1027E00000201BBC00641AB200B219A8000A19A08C
:1027F000006A189900D117910040178B00B5168414
:102800000031167E00B31579003A157300C7146FB6
:102810000058146A00EE1366008813630025135EE7
:1028200000C7125B006C12570015125400C1115101
:102830000070114F0021114B00D61049008D104738
:10284000004610440002104200C00F4000800F3EBE
:1028500000420F3C00060F3B00CB0E3800930E37B2
:10286000005C0E3500270E3400F30D3200C10D312F
:1028700000900D3000600D2E00320D2D00050D2C46
:1028800000D90C2B00AE0C2900850C29005C0C270C
:1028900000350C27000E0C2600E80B2400C40B2486
:1028A00000A00B23007D0B23005A0B2100390B21C4
:1028B00000180B2000F80A1F00D90A1E00BB0A1ED0
:1028C000009D0A1D00800A1D00630A1C00470A1BA8
:1028D000002C0A1B00110A1A00F7091A00DD091959
:1028E00000C4091900AB091900920917007B0918E7
:1028F00000630917004C0916003609160020091656
:10290000000A091500F5081500E0081400CC0814A9
:1029100000B8081400A4081400900813007D0812E1
:10292000006B081300580812004608120034081102
:1029300000230811001208110001081100F007100F
:1029400000E0071000D0071000C0071000B0070F0C
:1029500000A107100091070E0083070F0074070FF6
:102960000065070E0057070E0049070E003B070DD4
:10297000002E070E0020070D0013070D0006070D9F
:1029800000F9060C00ED060D00E0060C00D4060C64
:1029900000C8060C00BC060C00B0060C00A4060B18
:1029A0000099060C008D060B0082060B0077060BC3
:1029B000006C060B0061060A0057060B004C060A65
:1029C0000042060A0038060A002E060A0024060AFB
:1029D000001A060A001006090007060A00FD05098C
:1029E00000F4050900EB050900E2050900D9050915
:1029F00000D0050900C7050900BE050900B5050896
:102A000000AD050800A50509009C0508009405080F
:102A1000008C050800840508007C05080074050882
:102A2000006C050700650508005D050700560508F0
:102A3000004E050700470507004005080038050758
:102A400000310507002A050700230507001C0506BD
:102A500000160507000F0507000805060002050718
:102A600000FB040600F5040700EE040600E8040677
:102A700000E2040700DB040600D5040600CF0406CC
:102A800000C9040600C3040600BD040600B704061E
:102A900000B1040500AC040600A6040600A004056D
:102AA000009B04060095040500900406008A0405B6
:102AB0000085040500800406007A040500750405FD
:102AC00000700405006B0405006604050061040540
:102AD000005C04050057040500520405004D040580
:102AE0000048040500430405003E0404003A0405C0
:102AF0000035040500300404002C040500270404FC
:102B000000230405001E0404001A04040016040532
:102B100000110404000D0404000904050004040469
:102B20000000040400FC030400F8030400F40304A0
:102B300000F0030400EC030400E8030400E40304D1
:102B400000E0030400DC030400D8030400D4030401
:102B500000D0030400CC030400C8030300C5030332
:102B600000656E6473746F7073206869743A205ADC
:102B700000205A3A00656E6473746F707320686940
:102B8000743A20590020593A00656E6473746F706E
:102B900073206869743A20580020583A00656E64C2
:102BA00073746F7073206869743A20004572726F95
:102BB000723A006563686F3A0053544F5050454471
:102BC0002E20005072696E7465722073746F70707D
:102BD00065642064756520746F206572726F72730E
:102BE0002E2046697820746865206572726F7220A5
:102BF000616E6420757365204D39393920746F20FA
:102C0000726573746172742E202854656D706572DC
:102C100061747572652069732072657365742E2006
:102C200053657420697420616674657220726573DF
:102C300074617274696E6729004B494C4C45442E8F
:102C400020005072696E7465722068616C746564EE
:102C50002E206B696C6C28292063616C6C65642183
:102C600000FF01FF6F6B00526573656E643A2000D0
:102C70002200556E6B6E6F776E20636F6D6D616EA7
:102C8000643A2022004368616E67652066696C6162
:102C90006D656E74005A204F6666736574203A2025
:102CA000007A5F6D61783A20007A5F6D696E3A2034
:102CB000005A204F6666736574005A204F6666732B
:102CC0006574206F6B006C636420636F6E74726157
:102CD00073742076616C75653A20007A5F6D617857
:102CE0003A20007A5F70726F62653A20007A5F6DF9
:102CF000696E3A2000795F6D61783A2000795F6DE6
:102D0000696E3A2000785F6D61783A2000785F6DD7
:102D1000696E3A200020204C617965723A00205A91
:102D20003A0020593A0020436F756E7420583A20BB
:102D30000020453A00205A3A0020593A00583A00FB
:102D40004649524D574152455F4E414D453A4D61BE
:102D5000726C696E20312E302E322E3133204C753C
:102D60006C7A626F7420534F555243455F434F4412
:102D7000455F55524C3A68747470733A2F2F636FE5
:102D800064652E616C6570686F626A656374732E2A
:102D9000636F6D2F646966667573696F6E2F4D4141
:102DA000524C494E2F2050524F544F434F4C5F5678
:102DB000455253494F4E3A312E30204D41434849F8
:102DC0004E455F545950453A4C756C7A426F7420A9
:102DD00054415A20362045585452554445525F4379
:102DE0004F554E543A3120555549443A383435669A
:102DF000303033632D616562642D346535332D6168
:102E00003662392D37643039383466646536303986
:102E10000A004C756C7A426F742054415A20362057
:102E20004F66662E004C756C7A426F742054415A7E
:102E300020362072656164792E0042656420436FFC
:102E40006F6C696E6720646F6E652E00426564204A
:102E500048656174696E6720646F6E652E00205747
:102E60003A0020423A0020453A00543A0042656454
:102E700020436F6F6C696E672E2E2E0042656420B2
:102E800048656174696E672E2E2E00436F6F6C6902
:102E90006E6720646F6E652E0048656174696E67A9
:102EA00020646F6E652E0020573A0020453A00548A
:102EB0003A00436F6F6C696E672E2E2E0048656175
:102EC00074696E672E2E2E002042403A0020403A50
:102ED00000202F003A00205400202F0020423A000A
:102EE000202F006F6B20543A000A0A005374616E61
:102EF0006461726420446576696174696F6E3A201A
:102F0000000A004D65616E3A20000A002020207AF8
:102F10003A200000793A2000783A20003F5370654B
:102F2000636966696564206E756D626572206F669F
:102F3000206C65677320696E206D6F76656D656EB8
:102F400074206E6F7420706C61757361626C652E95
:102F50000A003F5370656369666965642059207093
:102F60006F736974696F6E206F7574206F6620725D
:102F7000616E67652E0A003F537065636966696517
:102F800064205820706F736974696F6E206F757458
:102F9000206F662072616E67652E0A003F53706570
:102FA0006369666965642073616D706C652073691F
:102FB0007A65206E6F7420706C61757361626C65E8
:102FC0002E0A0046756C6C20737570706F727420D9
:102FD00061743A20687474703A2F2F336470726988
:102FE0006E74626F6172642E636F6D2F666F72759F
:102FF0006D2E7068700A004D3438205A2D50726F53
:103000006265205265706561746162696C6974798A
:1030100020746573742E20202056657273696F6E5C
:1030200020322E30300A003F566572626F73652081
:103030004C6576656C206E6F7420706C6175736181
:10304000626C652E0A002569206D696E2C20256949
:103050002073656300456E642066696C65206C6949
:10306000737400426567696E2066696C65206C69DF
:103070007374004E6F206D6F76652E004C756C7A00
:10308000426F742054415A20362072656164792E53
:1030900000526573756D696E67207072696E740099
:1030A0005761697420666F7220757365722E2E2EBB
:1030B000000A00205A3A200020593A200020583AAD
:1030C00020004265640050726F62696E6720646F11
:1030D0006E65210020643A200020623A200045718C
:1030E0006E20636F656666696369656E74733A2006
:1030F000613A200050524F4245204641494C2043FE
:103100004C45414E204E4F5A5A4C450050524F426A
:1031100045204641494C20434C45414E204E4F5A94
:103120005A4C45004175746F206C6576656C696E0C
:103130006700486F6D6520582F59206265666F7271
:1031400065205A00486F6D6520582F5920626566CA
:103150006F7265205A005A2070726F6265206F7519
:10316000742E20626564005A2070726F6265206F51
:1031700075742E2062656400486F6D6520582F5964
:10318000206265666F7265205A00486F6D65205831
:103190002F59206265666F7265205A0020643A20BC
:1031A0000020623A200045716E20636F6566666993
:1031B0006369656E74733A20613A200044617964F2
:1031C0007265616D696E672E2E2E000000A04300AF
:1031D00080A243000087430000A0400000A0400000
:1031E0000000400000A0C1008098430000000000E3
:1031F00000A0C10000A0C100000000000096430034
:10320000809843000087430A00207A3A2000207902
:103210003A200020783A20004265640052657769C0
:1032200070696E67005265776970696E670025691D
:1032300020686F757273202569206D696E757465DD
:103240007300446F6E65207072696E74696E6720DA
:1032500066696C65004C756C7A426F742054415AF3
:1032600020362072656164792E0053544F505045CA
:10327000442E20005072696E7465722073746F70F2
:103280007065642064756520746F206572726F725A
:10329000732E2046697820746865206572726F729B
:1032A00020616E6420757365204D39393920746F43
:1032B00020726573746172742E202854656D706578
:1032C0007261747572652069732072657365742EFE
:1032D000205365742069742061667465722072657C
:1032E0007374617274696E6729004E6F204C696E49
:1032F00065204E756D626572207769746820636819
:1033000065636B73756D2C204C617374204C696E12
:10331000653A20004E6F20436865636B73756D20BE
:1033200077697468206C696E65206E756D62657270
:103330002C204C617374204C696E653A20006368E0
:1033400065636B73756D206D69736D617463682C53
:10335000204C617374204C696E653A20004C696E94
:1033600065204E756D626572206973206E6F7420E2
:103370004C617374204C696E65204E756D62657288
:103380002B312C204C617374204C696E653A2000FF
:103390004D31313000446F6E6520736176696E6720
:1033A0002066696C652E006F6B004D32390020205D
:1033B000506C616E6E6572427566666572427974B4
:1033C00065733A20002046726565204D656D6F7209
:1033D000793A20004A616E20323120323031360095
:1033E000436F6D70696C65643A2000286E6F6E657E
:1033F0002C2064656661756C7420636F6E66696706
:103400002900207C20417574686F723A20004A615F
:103410006E20323120323031362030393A33323A70
:10342000353700204C617374205570646174656495
:103430003A2000312E302E322E3133004D61726C25
:10344000696E0020536F66747761726520526573F0
:10345000657400205761746368646F6720526573F8
:103460006574002042726F776E206F75742052650C
:10347000736574002045787465726E616C205265C6
:1034800073657400506F7765725570007374617264
:1034900074002200656E717565696E6720220022D6
:1034A00000656E717565696E6720220048617264FF
:1034B000636F6465642044656661756C7420536550
:1034C0007474696E6773204C6F6164656400537433
:1034D0006F7265642073657474696E6773207265BA
:1034E000747269657665640020643A200020623A4F
:1034F0002000613A200045716E20636F6566666941
:103500006369656E74733A002044002049002020EE
:10351000204D33303120500050494420736574747D
:10352000696E67733A00205A0020590020204D32FE
:103530003036205800486F6D65206F66667365747D
:1035400020286D6D293A00204500205A002058009F
:1035500020420020540020204D32303520530041BD
:103560006476616E636564207661726961626C6520
:10357000733A20533D4D696E2066656564726174CF
:103580006520286D6D2F73292C20543D4D696E20C8
:1035900074726176656C206665656472617465201D
:1035A000286D6D2F73292C20423D6D696E696D75F4
:1035B0006D207365676D656E742074696D65202874
:1035C0006D73292C20583D6D6178696D756D20589B
:1035D00059206A65726B20286D6D2F73292C20206D
:1035E0005A3D6D6178696D756D205A206A65726B00
:1035F00020286D6D2F73292C2020453D6D61786941
:103600006D756D2045206A65726B20286D6D2F7376
:10361000290020540020204D3230342053004163D3
:1036200063656C65726174696F6E3A20533D6163C6
:1036300063656C65726174696F6E2C20543D7265B0
:10364000747261637420616363656C65726174692F
:103650006F6E00204500205A0020590020204D3276
:1036600030312058004D6178696D756D204163637C
:10367000656C65726174696F6E20286D6D2F733291
:10368000293A00204500205A0020590020204D32C0
:1036900030332058004D6178696D756D2066656521
:1036A00064726174657320286D6D2F73293A002050
:1036B0004500205A0020590020204D393220580062
:1036C00053746570732070657220756E69743A006A
:1036D00053657474696E67732053746F7265640008
:1036E0000A0020000A00207A3A200020793A2000BF
:1036F00020783A200001050800FF0601210235204C
:10370000FFFF07FF06FF09005022165680808080C9
:103710000080153353A0A0A00257575050F850F81E
:1037200050500257572070A07028702013355580D4
:10373000A040A02002475740A0A040A0A0502513C1
:10374000538080801226564080808080401226560A
:103750008040404040800245559060F060900255A6
:10376000552020F82020113353604080044151F04F
:1037700011335340E0400246561010204080801222
:10378000365640A0A0A0A04012365640C04040404F
:10379000E00246566090106080F0024656F02060CD
:1037A0001090600246562060A0F02020024656F09D
:1037B00080E01090600246566080E0909060024683
:1037C00056F0102020404002465660906090906075
:1037D000024656609090701060122555C0C000C01F
:1037E000C01136566060006040801236562040801E
:1037F000804020034353F000F012365680402020D2
:10380000408012365640A0204000400158583048B1
:1038100098A8A8904030024656609090F090900290
:103820004656E090E09090E002465660908080908E
:1038300060024656E090909090E0024656F080E09C
:103840008080F0024656F080E0808080024656601C
:103850009080B090600246569090F0909090123612
:1038600056E040404040E002465670202020A040F4
:1038700002465690A0C0A0A090024656808080804C
:1038800080F002465690F0F090909002465690D00C
:10389000F0B0B0900246566090909090600246560C
:1038A000E09090E08080014757609090D0B0601029
:1038B000024656E09090E09090024656609040207C
:1038C0009060123656E0404040404002465690908C
:1038D000909090600246569090909060600246569C
:1038E000909090F0F0900246569090606090900218
:1038F0005656888850202020024656F010204080DE
:10390000F0123656E080808080E00246568080408B
:10391000201010123656E020202020E016325240AF
:10392000A0014151F0162252804002445470909000
:10393000700246568080E09090E01234546080809F
:103940006002465610107090907002445460B0C0EF
:1039500060024656205040E040400145556090705E
:1039600010600246568080E09090901236564000DB
:10397000C04040E01137572000202020A0400246E0
:1039800056808090E09090123656C040404040E013
:10399000025454D0A8A8A8024454E0909090024445
:1039A0005460909060014555E090E080800145555D
:1039B0007090701010024454A0D080801234546073
:1039C000C020C00246564040E0405020024454907F
:1039D000909070123454A0A0A04002545488A8A81B
:1039E00050024454906060900145559090709060F2
:1039F000024454F02040F0024757304020C020409D
:103A000030221656808080808080024757C0204038
:103A1000304020C006425250A0FFFFFFFFFFFFFFD3
:103A2000FFFFFFFFFFFFFFFFFFFFFFFFFFFFFFFFA6
:103A3000FFFFFFFFFFFFFFFFFFFF090050221656A9
:103A40008000808080800146562070A0A0702002F7
:103A500046562050E04050A002555588705070885E
:103A60000256568850F820F8202217578080800090
:103A70008080800247577080E0907010E0173151CD
:103A8000A002565670A8C8C8A87014355560A0602A
:103A900000E003435350A050123353E02020143170
:103AA00051E002565670E8D8E8D870173151E01549
:103AB000335340A04012355540E04000E0143555E6
:103AC00040A02040E0143555C020C020C01622522E
:103AD0004080014555909090E08002565678E8E885
:103AE00068282824115180112252408014355540F5
:103AF000C04040E014355540A04000E0034353A0CF
:103B000050A0024757808080A060F0200247578075
:103B100080A0D010207002475780408060A0F02025
:103B200012365640004080A0400247574020609027
:103B3000F0909002475720406090F09090024757D5
:103B400060906090F0909002475750A06090F09085
:103B50009002475790006090F09090024757609015
:103B60006090F0909002465670A0A0F0A0B001477F
:103B700057609080809060400247574020F080E07E
:103B800080F00247572040F080E080F00247576005
:103B900090F080E080F00247579000F080E080F0E5
:103BA0001237578040E0404040E01237572040E055
:103BB000404040E012375740A0E0404040E012371C
:103BC00057A000E0404040E00256567048E84848A0
:103BD0007002475750A090D0B090900247574020B5
:103BE00060909090600247572040609090906002F3
:103BF00047576090609090906002475750A0609047
:103C000090906002475790006090909060123353FC
:103C1000A040A002465670B0B0D0D0E00247574056
:103C20002090909090600247572040909090906034
:103C30000247576090909090906002475790009094
:103C40009090906002575710208850202020024604
:103C50005680E09090E0800246566090A0A090A030
:103C60000247574020007090907002475720400054
:103C700070909070024757205000709090700247EB
:103C80005750A0007090907002465650007090906F
:103C90007002475760906070909070025454F068C2
:103CA000B078113555608080604002475740200051
:103CB00060B0C06002475720400060B0C06002475B
:103CC0005760900060B0C060024656500060B0C0BF
:103CD00060123757804000C04040E0123757204004
:103CE00000C04040E012375740A000C04040E01202
:103CF0003656A000C04040E0024757A040A01070D8
:103D0000906002475750A000E090909002475740C3
:103D100020006090906002475720400060909060C3
:103D20000247576090006090906002475750A00093
:103D300060909060024656900060909060123555F9
:103D40004000E0004002445470B0D0E002475740C9
:103D50002000909090700247572040009090907003
:103D600002475760900090909070024656900090E5
:103D700090907001485820400090907090600147EA
:103D8000578080E090E080800147579000909070CD
:103D9000906001070E00FE0A018A031E20FFFE0C40
:103DA000FE0BFE0E0070321A7A8080808080808048
:103DB000008080293474A0A0A0A0125A7A505050DC
:103DC000F85050F8505050016B7B10789494503854
:103DD0001494947810026A7A64949870102038646D
:103DE000A498026A7A3048484830649488986439C4
:103DF000147480808080204D7D1020404080808021
:103E0000808040402010104D7D80402020101010F8
:103E100010102020408013577720A8702070A82011
:103E2000135777202020F8202020202474C0404001
:103E300080165171F821337340E040006D7D040419
:103E40000808101010202040408080026A7A304814
:103E50008484848484844830125A7A2060A020208C
:103E600020202020F8026A7A788484040808102030
:103E700040FC026A7AFC0408103804048484780246
:103E80006A7A08182828484888FC0808026A7AFCD8
:103E90008080F8840404848478026A7A38408080C0
:103EA000B8C484848478026A7AFC0408081010205C
:103EB000204040026A7A7884844830488484847838
:103EC000026A7A788484848C7404848870223878B6
:103ED00040E040000040E040212878C0C00000C021
:103EE0004040801259790810204080402010080579
:103EF0006474FC0000FC12597980402010081020E6
:103F00004080026A7A788484081010100010100231
:103F10006A7A38449CA4A4A4A49C403C026A7A30E7
:103F200048848484FC84848484026A7AF088848847
:103F3000F088848488F0026A7A7884848080808023
:103F4000848478026A7AF08884848484848488F003
:103F5000026A7AFC808080F080808080FC026A7A2D
:103F6000FC808080F08080808080026A7A788484FF
:103F700080809C84848C74026A7A84848484FC8427
:103F800084848484125A7AF8202020202020202043
:103F9000F8026A7A1C080808080808888870026A0B
:103FA0007A848890A0C0A090888484026A7A8080F5
:103FB00080808080808080FC026A7A84CCCCB4B41B
:103FC0008484848484026A7A8484C4C4A4948C8C97
:103FD0008484026A7A7884848484848484847802E1
:103FE0006A7AF884848484F880808080006C7C788D
:103FF0008484848484E4948C780804026A7AF88443
:10400000848484F890888484026A7A7884848060C6
:104010001804848478027A7AFE10101010101010A0
:104020001010026A7A84848484848484848478026C
:104030006A7A84848484484848303030125A7A88B6
:104040008888888888A8A8A850026A7A8484484802
:10405000303048488484125A7A888888505020200A
:10406000202020026A7AFC0408101020404080FCC6
:10407000204D7DF08080808080808080808080F0F6
:10408000006D7D808040402020201010080804042E
:10409000104D7DF01010101010101010101010F0B6
:1040A0000A6373304884006171FC2A3373804020B6
:1040B0000267777884047C84847C026A7A808080BA
:1040C000B8C4848484C4B80267777884808080848C
:1040D00078026A7A040404748C8484848C74026781
:1040E00077788484FC808478026A7A18242020F807
:1040F0002020202020006979748888887040B88446
:1041000078026A7A808080B8C48484848484125A55
:104110007A202000602020202020F8105C7C0808F5
:1041200000180808080808888870026A7A80808069
:104130008890A0E0908884125A7A60202020202065
:10414000202020F8125777D0A8A8A8A8A88802672E
:1041500077B8C48484848484026777788484848470
:104160008478006979B8C4848484C4B88080006984
:1041700079748C8484848C740404026777B8C48452
:104180008080808002677778844030088478026A73
:104190007A202020F82020202024180267778484A9
:1041A0008484848C74125777888888505020201219
:1041B00057778888A8A8A8A85002677784844830D1
:1041C000488484006979848484848C7404847802AB
:1041D0006777FC0810202040FC204D7D3040404097
:1041E000404080404040404030301D7D8080808095
:1041F000808080808080808080104D7DC020202045
:104200002020102020202020C009647440A494089D
:10421000FFFFFFFFFFFFFFFFFFFFFFFFFFFFFFFFAE
:10422000FFFFFFFFFFFFFFFFFFFFFFFFFFFFFFFF9E
:10423000FF0E0070321A7A8080008080808080803B
:10424000800169792078A4A0A0A0A47820125979CF
:1042500030484040F04040F0480466768478484852
:104260007884125A7A88505020F820F82020203282
:104270001A7A80808080000080808080026B7B784A
:10428000844030488448300884781B427290900201
:104290006B7B7884B4CCC4C4C4CCB484781558780F
:1042A00070887888986800F8026777142850A050C2
:1042B0002814125474F8080808164171F0026B7B38
:1042C0007884F4CCCCF4CCCCCC84781B5171F81924
:1042D0004474609090601256762020F82020F816E2
:1042E0004777609010204080F0164777609010600C
:1042F0001090602A3373204080105878888888880E
:10430000D8A88080105C7C78A8A8A8A8682828284D
:104310002828383711718020237340408026377752
:1043200040C040404040E01646766090906000F00B
:10433000026777A05028142850A0026A7A40C44827
:104340004850242C549C84026A7A40C4484850281F
:104350003444889C026A7AC4244830D0244C549C4B
:1043600004006B7B202000202020204084847802E1
:104370006C7C20100030488484FC84848484026C2B
:104380007C10200030488484FC84848484026C7C0B
:1043900030480030488484FC84848484026C7C64CB
:1043A000980030488484FC84848484026B7B4800B9
:1043B00030488484FC84848484026B7B3048304899
:1043C0008484FC84848484026A7A3C509090FC90BB
:1043D0009090909C006C7C78848480808080848421
:1043E000781020026C7C201000FC808080F8808097
:1043F00080FC026C7C102000FC808080F880808033
:10440000FC026C7C304800FC808080F8808080FC5E
:10441000026B7B4800FC808080F8808080FC125C0E
:104420007C402000F820202020202020F8125C7CF6
:10443000102000F820202020202020F8125C7C2072
:104440005000F820202020202020F8125B7B500014
:10445000F820202020202020F8027A7A7844424256
:10446000F24242424478026C7C649800C4C4A4A422
:104470009494948C8C026C7C2010007884848484C6
:1044800084848478026C7C10200078848484848402
:10449000848478026C7C30480078848484848484AA
:1044A0008478026C7C649800788484848484848416
:1044B00078026B7B480078848484848484847802C6
:1044C000777782442810284482006E7E0404788C1A
:1044D000949494A4A4A4C4788080026C7C201000DE
:1044E000848484848484848478026C7C1020008496
:1044F0008484848484848478026C7C30480084843E
:1045000084848484848478026B7B480084848484DB
:104510008484848478125C7C102000888850502029
:1045200020202020026A7A8080F884848484F880A5
:1045300080026A7A304848487048444444F8026A25
:104540007A2010007884047C84847C026A7A0810C3
:10455000007884047C84847C026A7A304800788401
:10456000047C84847C026A7A6498007884047C8465
:10457000847C02697948007884047C84847C026BA2
:104580007B304830007884047C84847C0277777C9C
:1045900092325E90927C0069797884808080847801
:1045A0001020026A7A201000788484FC80847802CB
:1045B0006A7A102000788484FC808478026A7A30D9
:1045C0004800788484FC8084780269794800788483
:1045D00084FC808478125A7A4020006020202020B9
:1045E00020F8125A7A102000602020202020F81293
:1045F0005A7A609000602020202020F812597950CB
:1046000000602020202020F8125B7B50205008788A
:10461000888888888870026A7A649800B8C484841C
:10462000848484026A7A2010007884848484847864
:10463000026A7A10200078848484848478026A7AFA
:1046400030480078848484848478026A7A6498008C
:1046500078848484848478026979480078848484A6
:104660008484780265753000FC0030006B7B0408A0
:10467000789494A4A4C4788080026A7A201000847C
:10468000848484848C74026A7A10200084848484F4
:10469000848C74026A7A30480084848484848C74A4
:1046A000026979480084848484848C74006C7C1052
:1046B0002000848444482838109060006C7C8080FE
:1046C00080B8C4848484C4B88080006B7B48008434
:1046D00084444828381090600000210024002700FE
:1046E0002A002D0030003300010100000401070101
:1046F0000A0100002200250028002B002E003100B6
:10470000340002010000050108010B010000200037
:104710002300260029002C002F0032000001000099
:104720000301060109010505050507050808080834
:10473000020202020A0A0808040404040101010139
:104740000101010103030303030303030407070734
:104750000C0C0C0C0C0C0C0C0202020206060606D9
:10476000060606060B0B0B0B0B0B0B0B07070A0AB7
:104770000A0A0A0A0505050401021020200808108B
:1047800020401020408002010201080402010102C1
:10479000040810204080804020100804020180049A
:1047A00002018040201008040201080402010102F5
:1047B00004081020408001020408102040801008E6
:1047C000040880102040044080100000090A0208FC
:1047D0000B0C0D07060304010000000000000000A0
:1047E00000000000000000000000000000000000C9
:1047F00000000000000011100F0000000000000089
:1048000000000000000000000000000000000000A8
:1048100002494E46494E4954594E414ECDCCCC3DAD
:104820000AD7233C17B7D13877CC2B329595E6249D
:104830001FB14F0A000020410000C84200401C4642
:1048400020BCBE4CCA1B0E5AAEC59D740D944B1BAA
:104850000D94711B0D94721B0D94532A0D946D1EB3
:104860000D947D230D94B91B0D94601B0D94181BA2
:104870000D94891B0D945D220D94421B2D5F96951E
:10488000E6C92A24E1C911241FBECFEFD1E2DEBF61
:10489000CDBF00E00CBF15E0A0E0B2E0ECE1F0E637
:1048A00002E00BBF02C007900D92AE3BB107D9F7F3
:1048B0001BBE16E1AEEBB5E001C01D92A33CB107F3
:1048C000E1F718E4C4E8D8E404C02297FE010F948D
:1048D000B42FCC37D107C9F70F94B0260D9402300E
:1048E0000C940000CF93DF93BC018230910510F44B
:1048F00062E070E0A091BF16B091C016ED0140E0FB
:1049000050E0E0E0F0E021C08881998186179707A8
:1049100069F48A819B81309719F09383828304C064
:104920009093C0168093BF16FE0134C068177907B4
:1049300038F44115510519F08417950708F4AC01B6
:10494000FE018A819B819C01E9012097E9F64115CE
:104950005105A9F1CA01861B970B049708F4BA0107
:10496000E0E0F0E02AC08D919C91119784179507A3
:10497000F9F46417750781F412968D919C91139741
:10498000309719F09383828304C09093C01680936C
:10499000BF16FD0132964CC0CA01861B970BFD0164
:1049A000E80FF91F6193719302978D939C9340C018
:1049B000FD01828193819C01D9011097A1F680911C
:1049C000BD169091BE16892B41F480913A049091C6
:1049D0003B049093BE168093BD1640913C045091C9
:1049E0003D044115510541F44DB75EB7809138043F
:1049F00090913904481B590B2091BD163091BE1679
:104A0000CA01821B930B8617970780F0AB014E5F9C
:104A10005F4F8417950750F0420F531F5093BE16F7
:104A20004093BD16F9016193719302C0E0E0F0E09C
:104A3000CF01DF91CF910895CF93DF93009709F4D1
:104A400050C0EC0122971B821A82A091BF16B09130
:104A5000C016109709F140E050E0AC17BD0708F10F
:104A6000BB83AA83FE0121913191E20FF31FAE17A0
:104A7000BF0779F48D919C911197280F391F2E5FF4
:104A80003F4F3983288312968D919C9113979B8376
:104A90008A834115510571F4D093C016C093BF1697
:104AA00020C012968D919C911397AD01009711F043
:104AB000DC01D3CFFA01D383C28321913191E20F7C
:104AC000F31FCE17DF0769F488819981280F391FFA
:104AD0002E5F3F4FFA01318320838A819B8193832C
:104AE0008283DF91CF910895A0E0B0E0EAE7F5E29C
:104AF0000D94D12FEC015B016115710519F0FB01DB
:104B000091838083F9908F2D90E00F94B82F892B9B
:104B1000C9F7FDE2FF1621F4F990EE24E39405C0F5
:104B20002BE2F21609F4F990EE248E0101501040A8
:104B3000C80161E178E443E050E072D2892BF9F4D6
:104B40008E010E5F1F4FC80164E178E445E050E03C
:104B500067D2892B19F48E01095F1F4FA114B1048C
:104B600019F0F50111830083E0FC04C070E090E0CF
:104B700080E813C070E090E080E86FEF07C1C801E3
:104B800069E178E443E050E04BD2892B69F4A11449
:104B9000B10429F470E090E080EC6FE7F7C0229652
:104BA000F501D183C083F6CF8824992440E050E0FA
:104BB00060E070E0EF2DE053EA30A0F5F2E0EF2A7C
:104BC0008E2D90E09C0128703070E2FE06C0232BF1
:104BD00079F50894811C911C2BC0232B19F00894A3
:104BE00081089108DB01CA0112E0880F991FAA1FF2
:104BF000BB1F1A95D1F7480F591F6A1F7B1F440F1F
:104C0000551F661F771F4E0F511D611D711D4839BD
:104C100029E9520729E9620729E1720748F084E08F
:104C2000E82A06C0EE3F31F4E3FC39C098E0E92AF7
:104C3000F990C0CFE53311F0E53189F529912D3296
:104C400019F4E0E1EE2A05C02B3219F081E090E082
:104C500003C0299182E090E0E22FE053EA3018F09F
:104C6000C81BD90B1CC020E030E0FCE020383F0717
:104C70005CF4C901880F991F880F991F280F391FED
:104C8000220F331F2E0F311DE991E053EA3068F3F4
:104C9000E4FE03C0309521953F4F820E931ECE2C2B
:104CA000DD24E1FE07C0A114B10421F02197F50134
:104CB000D183C083CB01BA010F941D2C7B018C01E1
:104CC000F3E0CF22DD2423E0C216D10421F417FB48
:104CD000109517F9109557016801C801B70120E038
:104CE00030E040E050E00F947D2B882309F44AC067
:104CF00097FE0DC020E3E22E28E4F22E90948194DA
:104D000091089394C0E2D0E000E010E012C098E473
:104D1000E92E98E4F92EF6CFF701259135914591CA
:104D20005491C601B5010F945D2E5B016C018C1A84
:104D30009D0A8C169D0684F7D595C7950F5F1F4F6A
:104D40000630110529F08CEF9FEFE80EF91EF1CF28
:104D5000C501D6017C018D018C2D880F8D2D881FFA
:104D60008F3F51F0C601B50120E030E040E050E057
:104D70000F947D2B882331F482E290E09093C21649
:104D80008093C1167E2D9F2D802F612F272F392FC5
:104D9000482F562FB901CA01CDB7DEB7ECE00D940C
:104DA000ED2F2F923F925F926F927F928F929F9200
:104DB000AF92BF92CF92DF92EF92FF920F931F9329
:104DC000CF93DF938C011B01EA016115710519F086
:104DD000FB0191838083209749F0CE01029783974E
:104DE00028F020E030E040E050E0F6C0F801A1906B
:104DF0008F018A2D90E00F94B82F892BB9F7FDE22F
:104E0000AF1631F4F801A1908F015524539407C0D7
:104E1000FBE2AF1619F4F801A1908F0155242097F9
:104E200019F0C031D105C1F4F0E3AF1679F4F801FF
:104E30008081883711F0883549F4F801A1800E5F30
:104E40001F4FF2E05F2AC0E1D0E006C0209721F4B6
:104E500080E3A816E9F427C0C830D10531F1C93084
:104E6000D10524F4C230D10531F50CC0CA30D105CA
:104E700089F0C031D105F9F4C12CD12CE12CB8E076
:104E8000FB2E28C0C12CD12CE12CA0E4FA2E22C08C
:104E9000CAE0D0E0FCECCF2EFCECDF2EFCECEF2ED9
:104EA000FCE0FF2E17C0C8E0D0E0C12CD12CE12CD3
:104EB000E0E1FE2E0FC09E01442737FD4095542FA0
:104EC00060E070E080E090E80F94752FC901DA018E
:104ED0006C017D0120E030E040E050E060E03E0108
:104EE000882477FC8094982C70EDB72EBA0CE9E0FA
:104EF000EB1570F48A2D81548A3118F499ECB92E8F
:104F000006C08A2D81568A3150F589EAB82EBA0C2E
:104F10008B2D90E08C179D0714F56F3FE1F0C216C2
:104F2000D306E406F506B0F0CA01B901A401930165
:104F30000F942F2F9B01AC012B0D311D411D511DD5
:104F40002130F0E03F07F0E04F07F0E85F0710F492
:104F500061E001C06FEFF801A1908F01C5CF21146E
:104F6000310481F0662331F001501040F1011183CA
:104F7000008308C051FE1AC002501040F101118395
:104F8000008314C067FF12C050FC05C02FEF3FEF35
:104F90004FEF5FE704C020E030E040E050E882E2FD
:104FA00090E09093C2168093C11616C050FE08C0C0
:104FB00050954095309521953F4F4F4F5F4F0CC016
:104FC00057FF0AC082E290E09093C2168093C11608
:104FD0002FEF3FEF4FEF5FE7B901CA01DF91CF91AC
:104FE0001F910F91FF90EF90DF90CF90BF90AF9007
:104FF0009F908F907F906F905F903F902F9008953B
:10500000FB01DC0105900D920020E1F70895FC0101
:1050100005900020E9F7809590958E0F9F1F0895C9
:10502000FB01DC014150504088F08D9181341CF02F
:105030008B350CF4805E659161341CF06B350CF49B
:10504000605E861B611171F3990B0895881BFCCF7C
:10505000FB01DC014150504048F005900D920020CA
:10506000C9F701C01D9241505040E0F70895FB017F
:1050700055915523A9F0BF01DC014D914517411110
:10508000E1F759F4CD010590002049F04D9140150C
:105090004111C9F3FB014111EFCF81E090E001978D
:1050A0000895FB01DC0104C08D910190801921F469
:1050B00041505040C8F7881B990B0895FB01DC0153
:1050C00002C001900D9241505040D8F70895FB0165
:1050D000DC018D9181341CF08B350CF4805E619184
:1050E00061341CF06B350CF4605E861B611189F332
:1050F000990B0895FB01DC010D900020E9F7119751
:1051000001900D920020E1F70895FC01819186172E
:1051100021F08823D9F7992708953197CF01089571
:10512000FB01DC018D91019080190110D9F3990BDD
:105130000895FB01DC0101900D920020E1F7089534
:10514000FB01DC014150504030F08D9101908019FD
:1051500019F40020B9F7881B990B0895FB01DC01B5
:105160004150504048F001900D920020C9F701C015
:105170001D9241505040E0F70895FB015191552395
:10518000A9F0BF01DC014D9145174111E1F759F438
:10519000CD010190002049F04D9140154111C9F316
:1051A000FB014111EFCF81E090E001970895AEE05F
:1051B000B0E0EDEDF8E20D94D92F0E891F898EE055
:1051C0008C831A8309838FEF9FE79E838D839E01D3
:1051D000265E3F4FCE010196688D798DA9010AD0D8
:1051E0002F813885020F131FF80110822E96E4E0FC
:1051F0000D94F52FABE0B0E0E0E0F9E20D94CB2F99
:105200003C012B015A01FC0117821682838181FD2A
:1052100003C06FEF7FEFB9C19AE0892E1E01089499
:10522000211C311CF3012381F20123FD859123FF11
:1052300081912F01882309F4A5C1853239F423FD1A
:10524000859123FF81912F01853221F490E0B301F4
:10525000B7D1E8CF982FFF24EE249924FFE1FF1562
:10526000D0F09B3269F09C3228F4903259F093329E
:1052700091F40EC09D3249F0903369F441E024C0AE
:1052800052E0F52A84E0F82A28C098E0F92A25C0DF
:10529000E0E1FE2A22C0F7FC29C0892F80538A3022
:1052A00070F4F6FE05C0989C902C1124980E15C041
:1052B000E89CE02C1124E80EF0E2FF2A0EC09E329A
:1052C00029F4F6FC5FC140E4F42A07C09C3619F4C7
:1052D00050E8F52A02C0983649F4F20123FD959171
:1052E00023FF91912F01992309F0B8CF892F85547D
:1052F000833018F08052833038F444E050E0A40E3C
:10530000B51E5FE359830FC0933631F0933779F0C0
:10531000933509F052C01FC0F5018081898342E0B6
:1053200050E0A40EB51E610101E010E011C0F501CE
:10533000C080D180F6FC03C06FEF7FEF02C0692D03
:1053400070E042E050E0A40EB51EC6012ED18C01E3
:105350005FE7F52213C0F501C080D180F6FC03C0E1
:105360006FEF7FEF02C0692D70E042E050E0A40EC5
:10537000B51EC6010FD18C0150E8F52AF3FE06C018
:1053800018C080E290E0B3011BD1EA948E2D90E02A
:1053900008171907B0F30DC0F601F7FC8591F7FE69
:1053A00081916F0190E0B3010BD1E110EA940150BB
:1053B00010400115110581F7E2C0943611F09936BD
:1053C00061F5F7FE08C0F5012081318142815381EA
:1053D00084E090E00AC0F501808191819C0144271E
:1053E00037FD4095542F82E090E0A80EB91E9FE64D
:1053F000F92257FF09C050954095309521953F4FB0
:105400004F4F5F4FE0E8FE2ACA01B901A1012AE02F
:1054100030E002D1D82ED2183FC0953729F41F2D85
:105420001F7E2AE030E01DC01F2D197F9F3661F0DE
:10543000903720F4983509F0A5C00FC0903739F0A7
:10544000983709F09FC004C028E030E00AC010611E
:1054500014FD146020E130E004C014FD166020E16A
:1054600032E017FF08C0F50160817181828193816C
:1054700044E050E008C0F50180819181BC0180E0EA
:1054800090E042E050E0A40EB51EA101C5D0D82E98
:10549000D2188FE7F82EF122F6FE0BC05EEFF52250
:1054A000D91438F4F4FE07C0F2FC05C08FEEF822E0
:1054B00002C01D2D01C0192DF4FE0DC0FE01ED0D21
:1054C000F11D8081803319F499EEF92208C01F5F25
:1054D000F2FE05C003C08F2D867809F01F5F0F2DE7
:1054E000F3FC13C0F0FE0EC01E1510F09D2C0AC078
:1054F0009D2C9E0C911A1E2D05C080E290E0B301F8
:105500005FD01F5F1E15C8F304C01E1510F4E11A0A
:1055100001C0EE2404FF0EC080E390E0B30150D040
:1055200002FF1BC001FD03C088E790E00EC088E5C4
:1055300090E00BC0802F867881F001FF02C08BE2E3
:1055400001C080E2F7FC8DE290E0B30139D005C0E4
:1055500080E390E0B30134D09A94D914C8F3DA947C
:10556000F101ED0DF11D808190E0B30129D0DD2026
:10557000B1F705C080E290E0B30122D0EA94EE20BA
:10558000C9F750CEF30166817781CB012B96E2E11A
:105590000D94E72FFC010590615070400110D8F781
:1055A000809590958E0F9F1F0895FC01615070406B
:1055B00001900110D8F7809590958E0F9F1F089548
:1055C0000F931F93CF93DF938C01EB018B8181FFAE
:1055D0001BC082FF0DC02E813F818C819D812817C9
:1055E000390764F4E881F9810193F983E88306C0FF
:1055F000E885F985802F1995892B31F48E819F815B
:1056000001969F838E8302C00FEF1FEFC801DF91C9
:10561000CF911F910F910895FA01AA27283051F1D7
:10562000203181F1E8946F936E7F6E5F7F4F8F4FD3
:105630009F4FAF4FB1E03ED0B4E03CD0670F781F32
:10564000891F9A1FA11D680F791F8A1F911DA11D17
:105650006A0F711D811D911DA11D20D009F4689450
:105660003F912AE0269F11243019305D3193DEF6F8
:10567000CF010895462F4770405D4193B3E00FD0AE
:10568000C9F7F6CF462F4F70405D4A3318F0495D99
:1056900031FD4052419302D0A9F7EACFB4E0A6957C
:1056A0009795879577956795BA95C9F7009761059E
:1056B000710508959B01AC010A2E069457954795F4
:1056C00037952795BA95C9F7620F731F841F951FE9
:1056D000A01D08958091C407882399F14091BE05CB
:1056E0005091BF056091C0057091C1058091C207BE
:1056F0009091C30722EC35E00E943398882319F17A
:105700004091C5075091C6076091C7077091C807BF
:10571000411551056105710591F08091C207909185
:10572000C30722EC35E00E943398882361F0109281
:10573000C5071092C6071092C7071092C8071092AB
:10574000C40781E0089580E00895DF92EF92FF9210
:105750000F931F937B018C01D42E8091BE059091F5
:10576000BF05A091C005B091C1058E159F05A0078A
:10577000B107B9F0AFDF8823E1F08091C2079091C3
:10578000C307B801A70122EC35E00E94E698882300
:1057900081F0E092BE05F092BF050093C005109322
:1057A000C105DD2011F481E005C081E08093C407CC
:1057B00001C080E01F910F91FF90EF90DF9008955E
:1057C0008F929F92AF92BF92CF92DF92EF92FF9211
:1057D0000F931F93CF93DF936C01142F7093C30724
:1057E0006093C207FC01178A82E090E0A0E0B0E07D
:1057F00080839183A283B3831092C4071092C5075C
:105800001092C6071092C7071092C8078FEF9FEF3C
:10581000AFEFBFEF8093BE059093BF05A093C00587
:10582000B093C105442321F48824992454013FC036
:10583000453008F01CC160E070E080E090E040E09E
:1058400084DF882309F413C1C12FD0E02197FE0122
:1058500074E0EE0FFF1F7A95E1F7EE53FA4FE25432
:10586000FE4F8081EE5BF14090E08F779070892B46
:1058700009F0FDC0E653FE4F80819181A281B38182
:1058800084369105A105B10508F4F1C064E0CC0FA0
:10589000DD1F6A95E1F7C857D84F88809980AA80A4
:1058A000BB8081149104A104B10409F4E0C0C501D6
:1058B000B40140E04ADF882309F4D9C08091CD05C6
:1058C0009091CE058050924009F0D1C02091D20530
:1058D000222309F4CCC08091D0059091D105892B69
:1058E00009F4C5C08091CF05882309F4C0C0F60132
:1058F000228B8091CF058483158661E070E007C01C
:105900004F5FF60145874150483008F0B0C0F601BE
:105910004585848190E09B01042E02C0220F331F35
:105920000A94E2F78217930759F72091D80530912E
:10593000D9052115310519F040E050E008C020914B
:10594000E6053091E7054091E8055091E905F6013B
:105950002583368347835087E090D005F090D105AA
:1059600000E010E0E80CF91C0A1D1B1DE38AF48A14
:10597000058B168B8091D3059091D405918F808FE4
:105980006091D20570E080E090E00F942F2F6E0DB3
:105990007F1D801F911FF601628F738F848F958FFB
:1059A0002091D3053091D40555E0220F331F5A952D
:1059B000E1F721503E4F232F3327269540E050E05A
:1059C000260F371F481F591F26873787408B518B5B
:1059D0008091D5059091D605009719F0A0E0B0E030
:1059E00008C08091E2059091E305A091E405B09193
:1059F000E50585017401E21AF30A040B150BA801F1
:105A00009701280F391F4A1F5B1FF601058404C048
:105A100056954795379527950A94D2F7218732876F
:105A200043875487253FFFE03F07F0E04F07F0E052
:105A30005F0720F48CE0F601878B19C0255F3F4F8C
:105A40004040504018F480E1F6010EC08091EE0510
:105A50009091EF05A091F005B091F105F601828FCC
:105A6000938FA48FB58F80E2878B81E001C080E0A7
:105A7000DF91CF911F910F91FF90EF90DF90CF902A
:105A8000BF90AF909F908F9008956F927F928F926A
:105A90009F92AF92BF92CF92DF92EF92FF920F93BD
:105AA0001F93CF93DF93EC015A016B013801490139
:105AB000423051056105710508F45DC089859A85FC
:105AC000AB85BC850196A11DB11D84179507A6075E
:105AD000B70708F450C08F89803129F4E52EF62EDF
:105AE000072F11270CC0803209F045C07A018B01C5
:105AF00087E016950795F794E7948A95D1F78B89F7
:105B00009C89AD89BE89E80EF91E0A1F1B1FC801BA
:105B1000B70141E01ADE882371F18F89803149F4A1
:105B2000F501F070EE0FFF1FEE53FA4F71826082A5
:105B30000DC0F501EF77F070EE0FFF1FEE0FFF1FA6
:105B4000EE53FA4F60827182828293828A89823018
:105B500080F08D819E81AF81B885E80EF91E0A1F05
:105B60001B1FE092C507F092C6070093C70710936A
:105B7000C80781E001C080E0DF91CF911F910F91B4
:105B8000FF90EF90DF90CF90BF90AF909F908F905D
:105B90007F906F900895CF92DF92EF92FF920F93D4
:105BA0001F93CF93DF93EC017A018B016901898503
:105BB0009A85AB85BC850196A11DB11D84179507FB
:105BC000A607B70708F452C08F89803129F45527FA
:105BD000412F302F2F2D0CC0803209F047C09A0181
:105BE000AB0167E056954795379527956A95D1F7AC
:105BF0008B899C89AD89BE89280F391F4A1F5B1F7D
:105C00008091BE059091BF05A091C005B091C105DE
:105C1000281739074A075B0731F0CA01B90140E08C
:105C200094DD882319F18F89803159F4F701F070E0
:105C3000EE0FFF1FEE53FA4F80819181A0E0B0E09C
:105C40000EC0F701EF77F070EE0FFF1FEE0FFF1F92
:105C5000EE53FA4F80819181A281B381BF70F6012A
:105C600080839183A283B38381E001C080E0DF91D0
:105C7000CF911F910F91FF90EF90DF90CF900895FB
:105C8000AF92BF92CF92DF92EF92FF920F931F934A
:105C9000DF93CF9300D00F92CDB7DEB76C017A01BE
:105CA0008B0182E090E0A0E0B0E0F6018083918378
:105CB000A283B3835E010894A11CB11CC601B80184
:105CC000A701950168DF882339F1C601B801A70152
:105CD00000E010E020E030E0D8DE8823E9F0E98041
:105CE000FA800B811C81F6018789803151F4F8EF2D
:105CF000EF16FFEFFF06F0E00F07F0E01F07F0F2EE
:105D000009C088EFE8168FEFF8068FEF08078FE0DD
:105D10001807A0F281E001C080E00F900F900F9073
:105D20000F90CF91DF911F910F91FF90EF90DF9037
:105D3000CF90BF90AF9008954F925F926F927F92F5
:105D40008F929F92AF92BF92CF92DF92EF92FF928B
:105D50000F931F93DF93CF9300D00F92CDB7DEB791
:105D60006C0149835A836B837C833901EE24FF24C1
:105D700087012E010894411C511C812CE2E09E2ECB
:105D8000A12CB12C49815A816B817C81C601920181
:105D900002DF882339F1D501C401F601058404C06E
:105DA000880F991FAA1FBB1F0A94D2F7E80EF91E8D
:105DB0000A1F1B1F29813A814B815C8187898031B1
:105DC00031F4285F3F4F40405040E0F205C0285F6B
:105DD0003F4F4F4F5F40B0F2F301E082F182028308
:105DE000138381E00F900F900F900F90CF91DF9170
:105DF0001F910F91FF90EF90DF90CF90BF90AF90E9
:105E00009F908F907F906F905F904F9008952F920A
:105E10003F924F925F926F927F928F929F92AF923A
:105E2000BF92CF92DF92EF92FF920F931F93DF9377
:105E3000CF93CDB7DEB72F970FB6F894DEBF0FBE66
:105E4000CDBF1C014A875B876C877D873F872E8784
:105E5000DC0119968D919D910D90BC91A02D01961C
:105E6000A11DB11D8E839F83A887B987F901008189
:105E7000118122813381011511052105310549F078
:105E8000480159010894811C911CA11CB11C1D8260
:105E900010C0D1018D909D90AD90BC901D828A85DF
:105EA0009B85AC85BD850197A105B10511F491E0F5
:105EB0009D83750164014424552432018E010F5FD6
:105EC0001F4FF10181859285A385B4854816590637
:105ED0006A067B0608F08CC08E819F81A885B985F3
:105EE0008C159D05AE05BF0550F4A2E08A2E912CBD
:105EF000A12CB12CF2E0CF2ED12CE12CF12CC10140
:105F0000B701A601980147DE882309F471C0898191
:105F10009A81AB81BC81A70196012F5F3F4F4F4F04
:105F20005F4F0097A105B10519F049015A010DC055
:105F3000281939094A095B098A859B85AC85BD8585
:105F4000281739074A075B0759F00894411C511C70
:105F5000611C711C0894C11CD11CE11CF11CB1CF47
:105F6000C101A601B7010FEF1FEF2FEF3FE08DDD5D
:105F7000882391F43DC02601370108944108510857
:105F800061087108C101B301A201970186017DDD9D
:105F9000882371F1730162018C149D04AE04BF0467
:105FA00050F3AE85BF854D915D916D917C9141150A
:105FB00051056105710531F0C1019501840165DD6F
:105FC0008823B1F0EE85FF8580829182A282B38220
:105FD000FD81FF2359F00894811C911CA11CB11C68
:105FE000D1018D929D92AD92BC92139781E001C038
:105FF00080E02F960FB6F894DEBF0FBECDBFCF91D5
:10600000DF911F910F91FF90EF90DF90CF90BF90A5
:10601000AF909F908F907F906F905F904F903F9048
:106020002F900895382F20E09FB7F89480910501B4
:106030008B7F809305019FBF37FF02C0A39A01C0E9
:10604000A3989FB7F894809105018460809305011F
:106050009FBF2F5F283011F0330FE6CF08956F9266
:106060007F928F929F92AF92BF92CF92DF92EF92E8
:10607000FF920F931F933B01609161047091620442
:1060800070932A0A6093290A60911D0A70911E0A72
:1060900070932C0A60932B0A62E0609363046EECA9
:1060A00075E5709362046093610490932E0A809367
:1060B0002D0A7092300A60922F0ACA01B9010F941A
:1060C0001D2C2AE037ED43E25CE30F945D2E0F9424
:1060D000EC2B6093310A7093320A8093330A9093C9
:1060E000340A0F941F2C4B015C01C801B7010F94B7
:1060F0001D2C2AE037ED43E25CE30F945D2EA501F1
:1061000094010F94A32A0F94EC2B6093350A70939B
:10611000360A8093370A9093380AF30160817181BF
:10612000828193810F941D2C2AE037ED43E25CE3DA
:106130000F945D2EA50194010F94A32A0F94F12BC7
:1061400060931D0A70931E0A80931F0A9093200A81
:10615000D0923A0AC092390A1F910F91FF90EF90A6
:10616000DF90CF90BF90AF909F908F907F906F9077
:1061700008958093270A1092280A08951092D7074D
:10618000089581E008958091160A90E0969587958C
:106190009695879581700895FC012081822F90E06B
:1061A0006AE070E00F94622FCB016AE070E00F9418
:1061B000622F805D8093470A822F90E06AE070E052
:1061C0000F94622F805D8093480A1092490A87E4F9
:1061D0009AE00895FC01608171818281938120E0C1
:1061E00030E040E251E40F945D2E0F94EC2B9B01C4
:1061F00077FF02C08DE201C08BE28093470A37FF30
:1062000003C0309521953F4FC90168EE73E00F94AC
:10621000622FCB016AE070E00F94622F805D809363
:10622000480AC90164E670E00F94622FCB016AE06E
:1062300070E00F94622F805D8093490AC9016AE083
:1062400070E00F94622FCB016AE070E00F94622F30
:10625000805D80934A0A8EE280934B0AC9016AE00E
:1062600070E00F94622F805D80934C0A10924D0A6B
:1062700087E49AE00895FC016081718182819381B5
:1062800020E030E040E251E40F945D2E0F94EC2BBF
:106290009B0177FF03C0309521953F4FC90168EE00
:1062A00073E00F94622FCB016AE070E00F94622FCD
:1062B000805D8093470AC90164E670E00F94622F05
:1062C000CB016AE070E00F94622F805D8093480AF2
:1062D000C9016AE070E00F94622FCB016AE070E0C0
:1062E0000F94622F805D8093490A8EE280934A0A60
:1062F000C9016AE070E00F94622F805D80934B0AC1
:1063000010924C0A87E49AE00895AF92BF92CF9220
:10631000DF92EF92FF920F931F93FC0160817181D6
:106320008281938120E030E04AE754E40F945D2EAF
:106330000F94EC2B5B016C0197FD48C028EE33E015
:1063400040E050E00F94972FCA01B9012AE030E0F5
:1063500040E050E00F94972F605D6093470A8EE213
:106360008093480AC601B50124E630E040E050E0E1
:106370000F94972FCA01B9012AE030E040E050E0C5
:106380000F94972F605D6093490AC601B5012AE01A
:1063900030E040E050E00F94972FCA01B9012AE0A5
:1063A00030E040E050E00F94972F605D60934A0A20
:1063B000C601B5012AE030E040E050E00F94972F8D
:1063C000605D60934B0A10924C0A53C08DE280933B
:1063D000470AEE24FF248701EA18FB080C091D096F
:1063E000C801B70128EE33E040E050E00F94972F4A
:1063F000CA01B9012AE030E040E050E00F94972F45
:10640000605D6093480A8EE28093490AC801B70133
:1064100024E630E040E050E00F94972FCA01B90124
:106420002AE030E040E050E00F94972F605D6093E9
:106430004A0AC801B7012AE030E040E050E00F947A
:10644000972FCA01B9012AE030E040E050E00F94F4
:10645000972F605D60934B0AC801B7012AE030E0D6
:1064600040E050E00F94972F605D60934C0A1092CB
:106470004D0A87E49AE01F910F91FF90EF90DF9013
:10648000CF90BF90AF900895EF92FF920F931F931C
:10649000FC01608171818281938120E030E040E2E3
:1064A00051E40F945D2E0F94EC2BAC01CB01DA017B
:1064B0007C018D0117FF08C010950095F094E094C1
:1064C000E11CF11C011D111DC801B70124E630E0DB
:1064D00040E050E00F94972FCA01B9012AE030E064
:1064E00040E050E00F94972F605D6093470AC80129
:1064F000B7012AE030E040E050E00F94972FCA0146
:10650000B9012AE030E040E050E00F94972F605D41
:106510006093480A8EE28093490AC801B7012AE0D5
:1065200030E040E050E00F94972F605D60934A0A9E
:1065300010924B0A87E49AE01F910F91FF90EF9021
:106540000895FC010190F081E02DF7FF07C08DE276
:106550008093470AF095E195FF4F14C0E436F105AA
:1065600074F0CF0164E670E00F94622FCB016AE013
:1065700070E00F94622F805D8093470A06C080E22E
:106580008093470AEA30F10564F0CF016AE070E0D9
:106590000F94622FCB016AE070E00F94622F805D50
:1065A00001C080E28093480ACF016AE070E00F9456
:1065B000622F805D8093490A10924A0A87E49AE02C
:1065C0000895DF93CF930F920F92CDB7DEB7FC0102
:1065D00060817181828193810F94EC2B7A8369832E
:1065E000CE010196AEDF0F900F90CF91DF9108950D
:1065F000EF92FF920F931F93FC01E080F1800281E4
:106600001381C801B70120E030E040E050E00F9472
:106610008B2D18161CF4C801B70103C0C801B701BF
:1066200090580F94EC2B7B018C0180E1E81687E2F7
:10663000F80680E0080780E0180714F460E211C053
:10664000C801B70120E137E240E050E00F94972FF6
:10665000CA01B9012AE030E040E050E00F94972FE2
:10666000605D6093470A88EEE81683E0F80680E0F4
:10667000080780E0180714F460E211C0C801B701F0
:1066800028EE33E040E050E00F94972FCA01B901A3
:106690002AE030E040E050E00F94972F605D609377
:1066A000480A84E6E816F1040105110514F460E2D5
:1066B00011C0C801B70124E630E040E050E00F947B
:1066C000972FCA01B9012AE030E040E050E00F9472
:1066D000972F605D6093490A8AE0E816F10401058E
:1066E000110514F460E211C0C801B7012AE030E0DE
:1066F00040E050E00F94972FCA01B9012AE030E042
:1067000040E050E00F94972F605D60934A0AC80103
:10671000B7012AE030E040E050E00F94972F605D31
:1067200060934B0A10924C0A87E49AE01F910F91F4
:10673000FF90EF900895EF92FF920F931F93FC014B
:10674000608171818281938120E030E040E251E4F8
:106750000F945D2E0F94EC2B97FF02C02DE201C029
:106760002BE22093470A7B018C0197FF08C010950C
:106770000095F094E094E11CF11C011D111DC8016D
:10678000B70120E137E240E050E00F94972FCA01B3
:10679000B9012AE030E040E050E00F94972F605DAF
:1067A0006093480AC801B70128EE33E040E050E0AA
:1067B0000F94972FCA01B9012AE030E040E050E081
:1067C0000F94972F605D6093490AC801B70124E6D2
:1067D00030E040E050E00F94972FCA01B9012AE061
:1067E00030E040E050E00F94972F605D60934A0ADC
:1067F000C801B7012AE030E040E050E00F94972F45
:10680000CA01B9012AE030E040E050E00F94972F30
:10681000605D60934B0A8EE280934C0AC801B70119
:106820002AE030E040E050E00F94972F605D6093E5
:106830004D0A10924E0A87E49AE01F910F91FF9043
:10684000EF900895EF92FF920F931F93FC016081E8
:1068500071818281938120E030E048EC52E40F9412
:106860005D2E0F94EC2B97FF02C02DE201C02BE2AE
:106870002093470A7B018C0197FF08C01095009573
:10688000F094E094E11CF11C011D111DC801B70139
:1068900020E137E240E050E00F94972FCA01B901A0
:1068A0002AE030E040E050E00F94972F605D609365
:1068B000480AC801B70128EE33E040E050E00F94E9
:1068C000972FCA01B9012AE030E040E050E00F9470
:1068D000972F605D6093490AC801B70124E630E054
:1068E00040E050E00F94972FCA01B9012AE030E050
:1068F00040E050E00F94972F605D60934A0A8EE26B
:1069000080934B0AC801B7012AE030E040E050E034
:106910000F94972FCA01B9012AE030E040E050E01F
:106920000F94972F605D60934C0AC801B7012AE06D
:1069300030E040E050E00F94972F605D60934D0A87
:1069400010924E0A87E49AE01F910F91FF90EF900A
:1069500008950F93DF93CF9300D00F92CDB7DEB79A
:1069600000910301029506950770009501708091D2
:10697000030186FF02602091180A3091190A4091A4
:106980001A0A50911B0A29833A834B835C830F9424
:10699000E72529813A814B815C8126173707480713
:1069A000590710F4629B04600093160A9091160A2E
:1069B00091708091160A81FD926080911C0A98174F
:1069C00029F19130B1F0913028F0923041F09330BC
:1069D000E9F40AC0813079F08230C1F412C0882312
:1069E00051F0833099F40DC0823029F0813071F478
:1069F00008C0833021F48091C9078F5F05C08823C8
:106A000029F48091C90781508093C90790931C0A8B
:106A10000F900F900F900F90CF91DF910F910895ED
:106A2000CF93DF93EC0104C08AED99E00F947D2AA7
:106A3000FE01219664916623B9F7DF91CF91089505
:106A4000EF92FF920F931F93CF93DF93F82EEB01FA
:106A5000142FE22E4E3311F04B3FA9F48EED99E046
:106A600061E00F94F11F4CE0F49EA00111244D5FF2
:106A70008EED99E060E020E80CE00F94231E8EED8F
:106A800099E060E003C08EED99E061E00F94F11FA2
:106A90001092130A2F2D30E02F5F3F4FC901880F4E
:106AA000991F820F931F880F991F880F991F80933A
:106AB000140A1E3309F410E28AED99E0612F0F9455
:106AC0007D2A01E106C08AED99E00F947D2A219686
:106AD0000150FE0164916623B1F706C08AED99E08A
:106AE00060E20F947D2A01500023C1F78AED99E0FE
:106AF0006E2D0F947D2A8AED99E060E20F947D2A35
:106B00008EED99E061E00F94F11FDF91CF911F911D
:106B10000F91FF90EF900895EF92FF920F931F93C4
:106B2000CF93DF93182FEA01F901F02E808188239B
:106B300011F0138AE901EE20B1F08EED99E061E0E9
:106B40000F94F11F4CE0149FA00111244D5F8EEDB6
:106B500099E060E020E80CE00F94231E8EED99E0B0
:106B600060E00F94F11F1092130A212F30E02F5F85
:106B70003F4FC901880F991F820F931F880F991FDC
:106B8000880F991F8093140A8AED99E060E20F94B0
:106B90007D2AFF2029F08AED99E069EF0F947D2A84
:106BA00003E106C08AED99E00F947D2A21960150F9
:106BB00068816623B9F706C08AED99E060E20F9418
:106BC0007D2A01500023C1F7EE2029F08EED99E0D7
:106BD00061E00F94F11FDF91CF911F910F91FF9012
:106BE000EF900895DF92EF92FF920F931F93DF9340
:106BF000CF9300D00F92CDB7DEB7D82E8B01E12E08
:106C0000FF24E7FCF094EE24FF0CEE1CFF2481E14E
:106C100090E0E80EF91E8EED99E06FE271E00F94BE
:106C20006522D092130A86E08093140A17FD09C0EA
:106C3000E02FF0E0EE0FFF1FEC5AF54F60817181FD
:106C400004C06091560A7091570A882777FD809595
:106C5000982F0F941F2C20E030E040E05FE30F946A
:106C6000A42A0F94EC2B7A836983CE01019669DC08
:106C7000BC018AED99E00F94A12A8BEB96E1D0DE5E
:106C8000D092130A8BE18093140A17FD0DC0E02FF8
:106C9000F0E0EE0FFF1FEE0FFF1FE65AF54F608189
:106CA00071818281938108C06091600A7091610A4C
:106CB0008091620A9091630A0F94EC2B882777FDEC
:106CC0008095982F0F941F2C20E030E040E05FE388
:106CD0000F94A42A0F94EC2B7C836B83CE01039634
:106CE00030DCBC018AED99E00F94A12A88EB96E193
:106CF00097DE6091540A7091550A882777FD809538
:106D0000982F0F941F2C20915A0A30915B0A4091C2
:106D10005C0A50915D0A0F948B2D1D2D195F18167A
:106D20004CF08EED99E0612F4E2D22E002E00F94A1
:106D3000231E12C08EED99E060E00F94F11F8EEDDE
:106D400099E0612F4E2D22E002E00F94231E8EED7C
:106D500099E061E00F94F11F0F900F900F900F904A
:106D6000CF91DF911F910F91FF90EF90DF900895E9
:106D7000AF92BF92CF92DF92EF92FF920F931F9349
:106D8000DF93CF93CDB7DEB728970FB6F894DEBF69
:106D90000FBECDBF8EED99E061E00F94F11F8091A1
:106DA0004F0A80FF09C08091D8139091D913892B85
:106DB00019F0E4E6F4E102C0E1E8F5E18EED99E0D6
:106DC00069E041E02FE003E17F010F9446238EED5F
:106DD00099E06AE24AE228E007E00F94231E8EED74
:106DE00099E062E34CE222E005E00F94231E8EED71
:106DF00099E06AE241E32AE004E00F943E1E8EED42
:106E000099E062E34BE20F94DA1F8EED99E066E3BE
:106E100041E329E40F943E1E8EED99E06FE271E0AC
:106E20000F94652280911C11882309F450C0809131
:106E3000EB12882369F0A0909513B0909613C09040
:106E40009713D0909813A114B104C104D10429F46C
:106E500060E070E080E090E022C060919D1370914E
:106E60009E1380919F139091A0130F941D2C7B0172
:106E70008C01C601B5010F941D2C20E030E046ECDA
:106E800052E40F94A42A20E030E048EC52E40F943E
:106E9000842B9B01AC01C801B7010F94842B20E027
:106EA00030E04EE852E40F945D2E20E030E048ECF4
:106EB00052E40F94842B0F94F12B8B019C018EEDE7
:106EC00099E067E342E3202F02E00F94231E87E35B
:106ED0008093130A8FE28093140A8091EA139091B1
:106EE000EB13A091EC13B091ED130097A105B10540
:106EF00009F4ACC00F94E72520E63AEE40E050E0FC
:106F00000F94752F79018A016091EA137091EB1348
:106F10008091EC139091ED1320E63AEE40E050E0C2
:106F20000F94752FE21AF30AC7016CE370E00F9417
:106F30004E2F6983CE0101962FD9BC018AED99E0CD
:106F40000F94A12A8AED99E06AE30F947D2AC70184
:106F50006CE370E00F944E2F8A83CE0102961CD909
:106F6000BC018AED99E00F94A12A20919D133091E4
:106F70009E1340919F135091A0138091951390916F
:106F80009613A0919713B0919813281739074A07C1
:106F90005B0708F058C085EB96E142DD8091EB126B
:106FA000882319F4E0E070E010C0A0909513B09031
:106FB0009613C0909713D0909813A114B104C104F4
:106FC000D10429F4E0E070E080E060E024C060914A
:106FD0009D1370919E1380919F139091A0130F9415
:106FE0001D2C7B018C01C601B5010F941D2C20E0E6
:106FF00030E046EC52E40F94A42A20E030E048EC64
:1070000052E40F94842B9B01AC01C801B7010F948B
:10701000842BE62F692F2E2F372F482F562FC9018B
:10702000DA018D839E83AF83B887CE0105962CDA73
:10703000BC018AED99E00F94A12A8AED99E065E2FE
:107040000F947D2A06C08DEA96E102C080EA96E19F
:10705000E7DC86E090E060E070E0C4DD81E590E090
:107060006FEF7FEFBFDD8EED99E06FE271E00F947F
:10707000652288E68093130A8BE18093140A20919D
:10708000D8133091D91384E690E0AC01249FC0015D
:10709000259F900D349F900D11246FEF70E00F9499
:1070A000622F7C836B83CE0103964BDABC018AEDA1
:1070B00099E00F94A12A8AED99E060E072E00F94C4
:1070C000A12A8EED99E06FE271E00F9465228EEDBA
:1070D00099E060E04DE120E80AE00F94231E8EED78
:1070E00099E060E00F94F11F82E08093130A15E2AB
:1070F0001093140A8AED99E062E072E00F94A12ADD
:1071000088E08093130A1093140A8FEA93E162D8FF
:10711000BC018AED99E00F94A12A8FE28093130AB3
:107120001093140A8EE996E17BDC85E38093130AC1
:107130001093140A83EB93E14DD8BC018AED99E0DA
:107140000F94A12A8BE58093130A1093140A8AEDF9
:1071500099E064E072E00F94A12A81E68093130A1B
:107160001093140A87EB93E186D8BC018AED99E06D
:107170000F94A12A8EED99E061E00F94F11F8EED3E
:1071800099E06BE27AE00F94652283E08093130A22
:1071900081E38093140A8AED99E06DEF0F947D2AC4
:1071A0008EED99E06FE271E00F9465228CE08093A0
:1071B000130A80E38093140A8EEB94E0C2D9BC01D9
:1071C0008AED99E00F94A12A8AED99E065E20F9487
:1071D0007D2A8EED99E06FE271E00F9465221092A6
:1071E000130A8DE38093140A8AED99E06EE374E04C
:1071F0000F94A12A28960FB6F894DEBF0FBECDBF1C
:10720000CF91DF911F910F91FF90EF90DF90CF9082
:10721000BF90AF90089582E0809363040F94E725B8
:107220006C507E4F8F4F9F4F6093180A7093190ACE
:1072300080931A0A90931B0A6E9A8FE467E174E0B8
:1072400020E030E040E050E00F9465276AE070E015
:1072500080E090E00F94F5258FE40D94F126FC0179
:1072600080916104909162048E179F0779F0F093EA
:107270006204E093610440931D0A50931E0A6093D8
:107280001F0A7093200A222309F0C5CF089540E019
:1072900050E060E070E021E0E2CF40E050E060E0EC
:1072A00070E021E0DCCF8DE99DE340E050E060E05C
:1072B00070E020E0D4CF1092550A1092540A109238
:1072C000570A1092560A1092D9131092D813EBCF86
:1072D000AF92BF92CF92DF92EF92FF920F931F93E4
:1072E00080911D0A90911E0AA0911F0AB091200A58
:1072F00081509048A040B04040F010921D0A10927A
:107300001E0A10921F0A1092200A60911D0A7091A5
:107310001E0A80911F0A9091200A25E030E040E08B
:1073200050E00F94752F79018A018091170A90E03F
:10733000A0E0B0E0E816F9060A071B0710F4209356
:10734000170A0091170A8091160A90E09695879582
:1073500096958795FF24F394F82210E083E1A82EF8
:10736000B12CC12CD12CEE24E394002381F5809123
:1073700063048823B9F080911D0A90911E0AA091A0
:107380001F0AB091200A0597A105B10528F4812FA5
:1073900060EA7CE14BEF04C0812F60EA7CE140E2CF
:1073A0002BEF4EDBFF2009F4D1C080911D0A909194
:1073B0001E0AA0911F0AB091200A0597A105B105E8
:1073C00008F0C4C028DF85E99EE361DFF7C0013023
:1073D00009F03DC0809163048823F1F060911D0A9B
:1073E00070911E0A80911F0A9091200A25E030E0DA
:1073F00040E050E00F94752F2130310541055105D3
:1074000029F4812F66E97CE14EE304C0812F66E90F
:107410007CE140E22AEF14DBFF2009F497C0609181
:107420001D0A70911E0A80911F0A9091200A25E082
:1074300030E040E050E00F94752F213031054105D8
:10744000510509F083C0E7DE80EC9CE37DC002308B
:1074500009F03DC0809163048823F1F060911D0A1A
:1074600070911E0A80911F0A9091200A25E030E059
:1074700040E050E00F94752F223031054105510551
:1074800029F4812F6DE87CE14EE304C0812F6DE883
:107490007CE140E22AEFD4DAFF2009F457C0609182
:1074A0001D0A70911E0A80911F0A9091200A25E002
:1074B00030E040E050E00F94752F22303105410557
:1074C000510509F043C0A7DE83EB9CE33DC00330C8
:1074D00009F03CC0809163048823F1F060911D0A9B
:1074E00070911E0A80911F0A9091200A25E030E0D9
:1074F00040E050E00F94752F2330310541055105D0
:1075000029F4812F62E87CE14EE304C0812F62E818
:107510007CE140E22AEF94DAFF20C1F060911D0A7D
:1075200070911E0A80911F0A9091200A25E030E098
:1075300040E050E00F94752F23303105410551058F
:1075400029F469DE86EA9CE3A8DE38C080911D0A32
:1075500090911E0AA0911F0AB091200A4497A1059C
:10756000B10540F0A0921D0AB0921E0AC0921F0AF7
:10757000D092200A60911D0A70911E0A80911F0A04
:107580009091200A25E030E040E050E00F94752F04
:10759000422F8091170A90E0049630E082179307FB
:1075A00044F444504093170AE0926304042F0150BE
:1075B0001FEF1F5F153010F40F5FD7CE1F910F9193
:1075C000FF90EF90DF90CF90BF90AF900895AF9273
:1075D000BF92CF92DF92EF92FF920F931F93809111
:1075E0001D0A90911E0AA0911F0AB091200A815095
:1075F0009048A040B04040F010921D0A10921E0A20
:1076000010921F0A1092200A60911D0A70911E0AA2
:1076100080911F0A9091200A25E030E040E050E080
:107620000F94752F79018A018091170A90E0A0E0EC
:10763000B0E0E816F9060A071B0710F42093170AB2
:107640000091170A8091160A90E096958795969575
:107650008795FF24F394F82210E038E1A32EB12C93
:10766000C12CD12CEE24E394002381F58091630496
:107670008823B9F080911D0A90911E0AA0911F0ADB
:10768000B091200A0597A105B10528F4812F67EC78
:107690007CE14BEF04C0812F67EC7CE140E22BEFF3
:1076A000CFD9FF2009F411C180911D0A90911E0AC3
:1076B000A0911F0AB091200A0597A105B10508F015
:1076C00004C1A9DD88E699E3E2DD37C1013009F0A4
:1076D0003DC0809163048823F1F060911D0A709190
:1076E0001E0A80911F0A9091200A25E030E040E0B8
:1076F00050E00F94752F213031054105510529F4D3
:10770000812F60EC7CE14EE304C0812F60EC7CE1D2
:1077100040E22AEF95D9FF2009F4D7C060911D0AF5
:1077200070911E0A80911F0A9091200A25E030E096
:1077300040E050E00F94752F21303105410551058F
:1077400009F0C3C068DD8FE09FE5BDC0023009F0DD
:107750003DC0809163048823F1F060911D0A70910F
:107760001E0A80911F0A9091200A25E030E040E037
:1077700050E00F94752F223031054105510529F451
:10778000812F69EB7CE14EE304C0812F69EB7CE142
:1077900040E22AEF55D9FF2009F497C060911D0AF5
:1077A00070911E0A80911F0A9091200A25E030E016
:1077B00040E050E00F94752F22303105410551050E
:1077C00009F083C028DD86E09FE57DC0033009F025
:1077D0003DC0809163048823F1F060911D0A70918F
:1077E0001E0A80911F0A9091200A25E030E040E0B7
:1077F00050E00F94752F233031054105510529F4D0
:10780000812F62EB7CE14EE304C0812F62EB7CE1CF
:1078100040E22AEF15D9FF2009F457C060911D0AF4
:1078200070911E0A80911F0A9091200A25E030E095
:1078300040E050E00F94752F23303105410551058C
:1078400009F043C0E8DC8DEF9EE53DC0043009F04F
:107850003CC0809163048823F1F060911D0A70910F
:107860001E0A80911F0A9091200A25E030E040E036
:1078700050E00F94752F243031054105510529F44E
:10788000812F69EA7CE14EE304C0812F69EA7CE143
:1078900040E22AEFD5D8FF20C1F060911D0A709117
:1078A0001E0A80911F0A9091200A25E030E040E0F6
:1078B00050E00F94752F243031054105510529F40E
:1078C000AADC87EF9CE5E9DC38C080911D0A909125
:1078D0001E0AA0911F0AB091200A4997A105B1057F
:1078E00040F0A0921D0AB0921E0AC0921F0AD092C8
:1078F000200A60911D0A70911E0A80911F0A9091C2
:10790000200A25E030E040E050E00F94752F422F30
:107910008091170A90E0049630E08217930744F4B0
:1079200044504093170AE0926304042F01501FEF64
:107930001F5F153010F40F5F97CE1F910F91FF90CE
:10794000EF90DF90CF90BF90AF9008958DEC9CECBE
:10795000ACECBDE38093430A9093440AA093450A9C
:10796000B093460A34CE80E090E0A0E8BFE3809375
:10797000430A9093440AA093450AB093460A27CE3F
:1079800080E090E0A0E2B1E48093430A9093440A3F
:10799000A093450AB093460A1ACE1F93CF93DF9364
:1079A000EC01162F8BAD882331F481E08BAFCE0133
:1079B00004960F94B41FCE010496612F0F94D51F27
:1079C000DF91CF911F910895682F70E06F737070F1
:1079D0007093D9096093D8098AED99E0DECFCF93EF
:1079E000DF93EC018BAD882331F481E08BAFCE01C6
:1079F00004960F94B41FCE0104960F94C21FDF911A
:107A0000CF910895EF92FF920F938AED99E06091E4
:107A1000D809C3DF8AED99E0E2DF8EED99E06BE2F1
:107A20007AE00F9465228EED99E061E00F94F11FEA
:107A30008EED99E060E040E02091DE090091DF09E1
:107A40000F94231E8EED99E061E00F94F11F8EEDEF
:107A500099E00F94C61F882301F78AED99E0BFDFF4
:107A60008EED99E060E040E028E000E45EEBE52E7A
:107A700056E1F52E0F9446238EED99E06BE27AE005
:107A80000F9465228EED99E06DE341E126E032E04E
:107A90000F94DE228EED99E065EF76E30F94652278
:107AA0008EED99E06FE541E12CE032E00F94DE22AB
:107AB0008EED99E06BE27AE00F9465228EED99E00D
:107AC0006EE34CE123E132E00F94DE228EED99E08B
:107AD00065EF76E30F9465228EED99E06FE349E25E
:107AE0002EE132E00F94DE228EED99E065EF76E331
:107AF0000F9465228EED99E06EE345E32AE232E0D1
:107B00000F94DE228EED99E06EE34EE322E332E045
:107B10000F94DE228EED99E063E44EE324E332E03D
:107B20000F94DE228EED99E00F94C61F882309F092
:107B300097CF0F91FF90EF9008958091260A8823A8
:107B400021F081508093260A03C081E08093630472
:107B500080916304882321F00BD98AE08093260A60
:107B60008091160A90E09695879596958795982F1F
:107B700091708091270A882391F08091280A8823A8
:107B800039F09923B9F41092280A1092270A12C0EA
:107B9000992381F040DB81E08093280A0BC0992370
:107BA00049F084E79FE540E050E060E070E021E0CC
:107BB00056DB28DF2091BE043091BF042436310506
:107BC00054F480911D0A90911E0A280F391F253602
:107BD00031056CF41AC025363105BCF080911D0AC0
:107BE00090911E0A280F391F2436310574F4109223
:107BF0001D0A10921E0A10921F0A1092200A84E693
:107C000090E09093BF048093BE042091BE04309115
:107C1000BF042436310589F480911D0A90911E0A13
:107C20008B3091051CF0865A9F4F0DC02FEF863F79
:107C30009207ACF482599F4F06C080911D0A909123
:107C40001E0A820F931F9093BF048093BE0410926C
:107C50001D0A10921E0A10921F0A1092200A80918B
:107C6000BE049091BF048A3091053CF48AE090E014
:107C70009093BF048093BE040895885E934034F0CF
:107C800087EE93E09093BF048093BE0408950F9312
:107C90001F93DF93CF93CDB7DEB76E970FB6F894EF
:107CA000DEBF0FBECDBF00D000D0EDB7FEB731961E
:107CB0009E012F5F3F4FADB7BEB712963C932E93F8
:107CC000119726E939E133832283958384830E94C7
:107CD000D7288E010B5F1F4FEDB7FEB736960FB654
:107CE000F894FEBF0FBEEDBF08C0992787FD9095A1
:107CF0000F94C02FD8018D938D01F80180818823C6
:107D0000A1F7CE0101960F94910982E999E10F94B0
:107D10001809C9DA6E960FB6F894DEBF0FBECDBF54
:107D2000CF91DF911F910F910895AF92BF92CF92A3
:107D3000DF92EF92FF920F931F9380911D0A909113
:107D40001E0AA0911F0AB091200A81509048A040BD
:107D5000B04040F010921D0A10921E0A10921F0AA5
:107D60001092200A60911D0A70911E0A80911F0ACC
:107D70009091200A25E030E040E050E00F94752F0C
:107D800079018A018091170A90E0A0E0B0E0E8163E
:107D9000F9060A071B0710F42093170A0091170A27
:107DA0008091160A90E09695879596958795FF2481
:107DB000F394F82210E073E1A72EB12CC12CD12C42
:107DC000EE24E394002389F5809163048823C1F0B5
:107DD00080911D0A90911E0AA0911F0AB091200A5D
:107DE0000597A105B10528F4812F6DE77CE14BEFE4
:107DF00004C0812F6DE77CE140E22BEF0E9420352B
:107E0000FF2009F4D6C080911D0A90911E0AA0910E
:107E10001F0AB091200A0597A105B10508F0C9C055
:107E2000FAD984E79FE533DAFCC0013009F03EC09F
:107E3000809163048823F9F060911D0A70911E0AF5
:107E400080911F0A9091200A25E030E040E050E048
:107E50000F94752F213031054105510529F4812FEB
:107E600063E77CE14EE304C0812F63E77CE140E2FD
:107E700020E20E942035FF2009F49BC060911D0A7A
:107E800070911E0A80911F0A9091200A25E030E02F
:107E900040E050E00F94752F213031054105510528
:107EA00009F087C0B8D98FE69CE140C0023009F0E4
:107EB00040C0809163048823F9F060911D0A70919D
:107EC0001E0A80911F0A9091200A25E030E040E0D0
:107ED00050E00F94752F223031054105510529F4EA
:107EE000812F6EE57CE14EE304C0812F6EE57CE1DD
:107EF00040E220E20E942035FF2009F45AC0609140
:107F00001D0A70911E0A80911F0A9091200A25E097
:107F100030E040E050E00F94752F223031054105EC
:107F2000510509F046C077D98AE59CE10F941809FC
:107F300078C0033009F03DC0809163048823F9F0D4
:107F400060911D0A70911E0A80911F0A9091200A6B
:107F500025E030E040E050E00F94752F23303105EC
:107F60004105510529F4812F60E57CE14EE304C011
:107F7000812F60E57CE140E22AEF0E942035FF205E
:107F8000C1F060911D0A70911E0A80911F0A9091A4
:107F9000200A25E030E040E050E00F94752F2330B8
:107FA00031054105510529F436D988E699E375D99B
:107FB00038C080911D0A90911E0AA0911F0AB091AD
:107FC000200A4497A105B10540F0A0921D0AB09285
:107FD0001E0AC0921F0AD092200A60911D0A709159
:107FE0001E0A80911F0A9091200A25E030E040E0AF
:107FF00050E00F94752F422F8091170A90E004965D
:1080000030E08217930744F444504093170AE092FB
:108010006304042F01501FEF1F5F153010F40F5F32
:10802000D1CE1F910F91FF90EF90DF90CF90BF9036
:10803000AF9008958AE191E10E946A651092170A53
:1080400008954F925F926F927F928F929F92AF921C
:10805000BF92CF92DF92EF92FF920F931F93CF9335
:10806000DF9380916304882309F0D0C18091160AC0
:1080700082FDCCC1DFC110921D0A10921E0A10921F
:108080001F0A1092200A60911D0A70911E0A8091A9
:108090001F0A9091200A25E030E040E050E00F9464
:1080A000752F79018A018091170A90E0A0E0B0E075
:1080B000E816F9060A071B0710F42093170AB09078
:1080C000170A8091160A90E0969587959695879560
:1080D000AA24A394A822FF2444244394340108949E
:1080E00061087108F5E05F2EBB2079F5809163048B
:1080F0008823C1F080911D0A90911E0AA0911F0A49
:10810000B091200A0597A105B10528F48F2D6DE8DF
:1081100079E14BEF04C08F2D6DE879E140E22BEF60
:108120000E942035AA2089F080911D0A90911E0A94
:10813000A0911F0AB091200A0597A105B10528F466
:108140006AD884E79FE5A3D875C18EE691E16EE118
:1081500071E10E947A9B80911E118F3211F411E01F
:1081600029C021E0B21629F5809163048823F9F033
:1081700060911D0A70911E0A80911F0A9091200A39
:1081800025E030E040E050E00F94752F21303105BC
:108190004105510529F48F2D69E879E14EE304C0CA
:1081A0008F2D69E879E140E220E20E942035AA2083
:1081B00029F412E06301C0E0D0E0D7C060911D0A4D
:1081C00070911E0A80911F0A9091200A25E030E0EC
:1081D00040E050E00F94752F2130310541055105E5
:1081E00041F719D827DF26C11B1509F0B9C08AE16C
:1081F00091E1B60140E050E00E94996D80914611F6
:1082000090916304882309F45BC0992369F160911C
:108210001D0A70911E0A80911F0A9091200A25E084
:1082200030E040E050E00F94752F812F90E0A0E007
:10823000B0E0281739074A075B0759F48F2D6BE721
:1082400079E14EE151E12BE231E101E0EE24E394EA
:1082500009C08F2D6BE779E14EE151E12BE231E16D
:1082600001E0EE240E948C35AA2009F479C06091C7
:108270001D0A70911E0A80911F0A9091200A25E024
:1082800030E040E050E00F94752F812F90E0A0E0A7
:10829000B0E0281739074A075B0709F061C00E9460
:1082A0000B398AE191E16EE171E10E94BD651092A6
:1082B0001D0A10921E0A10921F0A1092200ABAC0BC
:1082C000992369F160911D0A70911E0A80911F0A1D
:1082D0009091200A25E030E040E050E00F94752FA7
:1082E000812F90E0A0E0B0E0281739074A075B072C
:1082F00059F48F2D6DE679E14EE151E12BE231E148
:1083000000E0EE24E39409C08F2D6DE679E14EE1A3
:1083100051E12BE231E100E0EE240E948C35AA20ED
:10832000F9F060911D0A70911E0A80911F0A9091C8
:10833000200A25E030E040E050E00F94752F812FB7
:1083400090E0A0E0B0E0281739074A075B0741F446
:108350000E940B398EE191E16BE271E198DC6AC019
:108360001F5F21960894C108D108C815D90508F4E3
:108370003BCF60911D0A70911E0A80911F0A909157
:10838000200A25E030E040E050E00F94752F812F67
:1083900090E0A0E0B0E0281739074A075B0780F0BB
:1083A000159DC00111240197AA2797FDA095BA2F0A
:1083B00080931D0A90931E0AA0931F0AB093200A6F
:1083C00060911D0A70911E0A80911F0A9091200AE7
:1083D00025E030E040E050E00F94752F422F80916F
:1083E000170A90E0049630E0821793074CF444504B
:1083F0004093170A40926304B42EBA94FF24FA946F
:10840000F39484E08F15B0F0B3946ECE8AE191E1DD
:108410000E94386D4C0180911D0A90911E0AA09116
:108420001F0AB091200A81509048A040B04008F047
:1084300022CE29CEDF91CF911F910F91FF90EF9027
:10844000DF90CF90BF90AF909F908F907F906F9074
:108450005F904F9008958AE191E10C945E658AE106
:1084600091E10C946565AF92BF92CF92DF92EF924B
:10847000FF920F931F9380911D0A90911E0AA09165
:108480001F0AB091200A81509048A040B04040F0AF
:1084900010921D0A10921E0A10921F0A1092200AB2
:1084A00060911D0A70911E0A80911F0A9091200A06
:1084B00025E030E040E050E00F94752F79018A010B
:1084C0008091170A90E0A0E0B0E0E816F9060A07EC
:1084D0001B0710F42093170A0091170A8091160ABF
:1084E00090E09695879596958795FF24F394F822CA
:1084F00010E0B8E1AB2EB12CC12CD12CEE24E394CA
:10850000002399F5809163048823C1F080911D0AAE
:1085100090911E0AA0911F0AB091200A0597A1050B
:10852000B10528F4812F6CEE79E14BEF04C0812F67
:108530006CEE79E140E22BEF0E942035FF2009F438
:108540001BC180911D0A90911E0AA0911F0AB09133
:10855000200A0597A105B10508F00EC10E940B394C
:1085600084E79FE50E9447393FC1013009F041C0CF
:10857000809163048823F9F060911D0A70911E0AAE
:1085800080911F0A9091200A25E030E040E050E001
:108590000F94752F213031054105510529F4812FA4
:1085A0006AED79E14EE304C0812F6AED79E140E2A2
:1085B0002AEF0E942035FF2009F4DEC060911D0AD9
:1085C00070911E0A80911F0A9091200A25E030E0E8
:1085D00040E050E00F94752F2130310541055105E1
:1085E00009F0CAC00E940B3981E694E40E944D391B
:1085F000FBC0023009F03FC0809163048823F9F08A
:1086000060911D0A70911E0A80911F0A9091200AA4
:1086100025E030E040E050E00F94752F2230310526
:108620004105510529F4812F6CEC79E14EE304C03A
:10863000812F6CEC79E140E220E20E942035FF209E
:1086400009F49AC060911D0A70911E0A80911F0A58
:108650009091200A25E030E040E050E00F94752F23
:10866000223031054105510509F086C00E940B39C1
:108670000F94EB0BB9C0033009F03FC08091630445
:108680008823F9F060911D0A70911E0A80911F0ADB
:108690009091200A25E030E040E050E00F94752FE3
:1086A000233031054105510529F4812F6EEB79E125
:1086B0004EE304C0812F6EEB79E140E220E20E949C
:1086C0002035FF2009F458C060911D0A70911E0AE0
:1086D00080911F0A9091200A25E030E040E050E0B0
:1086E0000F94752F233031054105510509F044C021
:1086F0000E940B390F94391477C00430E9F580914A
:1087000063048823F9F060911D0A70911E0A80911C
:108710001F0A9091200A25E030E040E050E00F94DD
:10872000752F243031054105510529F4812F6BEA5D
:1087300079E14EE304C0812F6BEA79E140E220E267
:108740000E942035FF20C1F060911D0A70911E0A21
:1087500080911F0A9091200A25E030E040E050E02F
:108760000F94752F243031054105510529F40E94DD
:108770000B390F94730E38C080911D0A90911E0A18
:10878000A0911F0AB091200A4997A105B10540F0B8
:10879000A0921D0AB0921E0AC0921F0AD092200A0F
:1087A00060911D0A70911E0A80911F0A9091200A03
:1087B00025E030E040E050E00F94752F422F80918B
:1087C000170A90E0049630E08217930744F444506F
:1087D0004093170AE0926304042F01501FEF1F5FBC
:1087E000153010F40F5F8CCE1F910F91FF90EF901A
:1087F000DF90CF90BF90AF900895CF92DF92EF922D
:10880000FF920F931F93CF93DF93D82EEB01C42ECB
:10881000F22EE32E002339F0822F932F0E94072897
:1088200011E1181B09C0E22FF32FDF010D9000208A
:10883000E9F7122F1A1B1E5E1092130A2D2D30E03D
:108840002F5F3F4FC901880F991F820F931F880F19
:10885000991F880F991F8093140A8AED99E06C2D57
:108860000F947D2A06C08AED99E00F947D2A219607
:108870001150FE0164916623B1F78AED99E06AE335
:108880000F947D2A06C08AED99E060E20F947D2A5C
:1088900011501123C1F7002329F08F2D9E2D0E9426
:1088A000103506C08AED99E06F2D7E2D0F94A12A18
:1088B000DF91CF911F910F91FF90EF90DF90CF90BC
:1088C00008952F923F924F925F926F927F928F9274
:1088D0009F92AF92BF92CF92DF92EF92FF920F934F
:1088E0001F93DF93CF93CDB7DEB7A0970FB6F89461
:1088F000DEBF0FBECDBF80911D0A90911E0AA091D0
:108900001F0AB091200A81509048A040B04040F02A
:1089100010921D0A10921E0A10921F0A1092200A2D
:1089200060911D0A70911E0A80911F0A9091200A81
:1089300025E030E040E050E00F94752F79018A0186
:108940008091170A90E0A0E0B0E0E816F9060A0767
:108950001B0710F42093170AF090170A8091160A4B
:1089600090E09695879596958795EE24E394E82276
:1089700010E02DE1C22ED12CCC0EDD1E99E1A92EE6
:10898000B12CAC0EBD1E85E1882E912C8C0E9D1E47
:1089900001E1602E712C6C0E7D1EBDE04B2E512C22
:1089A0004C0E5D1EA9E02A2E312C2C0E3D1EFF2000
:1089B000B1F5809163048823C1F080911D0A9091E4
:1089C0001E0AA0911F0AB091200A0597A105B105C2
:1089D00028F4812F6AE27BE14BEF04C0812F6AE229
:1089E0007BE140E22BEF0E942035EE2011F40C9445
:1089F000B64F80911D0A90911E0AA0911F0AB09156
:108A0000200A0597A105B10510F00C94B64F0E94FD
:108A10000B3983E392E40E9447390C94F54F81E0CF
:108A2000F81609F044C0809163048823F9F060913E
:108A30001D0A70911E0A80911F0A9091200A25E05C
:108A400030E040E050E00F94752F213031054105B2
:108A5000510529F4812F61E27BE14EE304C0812FAF
:108A600061E27BE140E22AEF0E942035EE2011F422
:108A70000C94B64F60911D0A70911E0A80911F0AD6
:108A80009091200A25E030E040E050E00F94752FEF
:108A9000213031054105510511F00C94B64F0E946B
:108AA0000B398BED98E50E944D390C94F54F22E07F
:108AB000F21609F098C080916304882341F1609117
:108AC0001D0A70911E0A80911F0A9091200A25E0CC
:108AD00030E040E050E00F94752F22303105410521
:108AE000510551F48DE89BE00E94F8329C01812FE2
:108AF0006BE17BE14EE309C08DE89BE00E94F83218
:108B00009C01812F6BE17BE140E200E076DEEE200C
:108B100011F40C94B64F60911D0A70911E0A809159
:108B20001F0A9091200A25E030E040E050E00F94C9
:108B3000752F223031054105510511F00C94B64FC7
:108B40000E940B39809161049091620490932A0AEB
:108B50008093290A80911D0A90911E0A90932C0AF5
:108B600080932B0A82E08093630483E297E59093DD
:108B700062048093610485E19BE190932E0A8093C7
:108B80002D0A8DE89BE09093300A80932F0A85E0B0
:108B900090E0A0E0B0E08093310A9093320AA09375
:108BA000330AB093340A89ED93E0A0E0B0E08093FB
:108BB000350A9093360AA093370AB093380A609129
:108BC0008D0B70918E0B80918F0B9091900B2AE002
:108BD00037ED43E25CE30F945D2E20E030E040EAA5
:108BE00050E40C94A94F83E0F81609F08DC08091F1
:108BF0006304882341F160911D0A70911E0A8091DF
:108C00001F0A9091200A25E030E040E050E00F94E8
:108C1000752F233031054105510551F485E99BE05D
:108C20000E94E1329C01812F6CE07BE14EE309C0A0
:108C300085E99BE00E94E1329C01812F6CE07BE1A1
:108C400040E200E0DADDEE2011F40C94B64F6091C2
:108C50001D0A70911E0A80911F0A9091200A25E03A
:108C600030E040E050E00F94752F2330310541058E
:108C7000510511F00C94B64F0E940B39809161049C
:108C80009091620490932A0A8093290A80911D0A88
:108C900090911E0A90932C0A80932B0A82E0809375
:108CA000630488EC97E5909362048093610483E009
:108CB0009BE190932E0A80932D0A85E99BE0909387
:108CC000300A80932F0A81E090E0A0E0B0E080932A
:108CD000310A9093320AA093330AB093340A8DED8F
:108CE00093E0A0E0B0E08093350A9093360AA09319
:108CF000370AB093380A6091950B7091960B80916A
:108D0000970B9091980BCDC624E0F21609F098C00D
:108D100080916304882341F160911D0A70911E0ABD
:108D200080911F0A9091200A25E030E040E050E059
:108D30000F94752F243031054105510551F489E90F
:108D40009BE00E9422349C01812F6BEF7AE14EE37D
:108D500009C089E99BE00E9422349C01812F6BEFBE
:108D60007AE140E200E049DDEE2011F40C94B64FC8
:108D700060911D0A70911E0A80911F0A9091200A2D
:108D800025E030E040E050E00F94752F24303105AD
:108D90004105510511F00C94B64F0E940B3980919A
:108DA00061049091620490932A0A8093290A809129
:108DB0001D0A90911E0A90932C0A80932B0A82E040
:108DC0008093630489ED95E5909362048093610438
:108DD00083EF9AE190932E0A80932D0A89E99BE014
:108DE0009093300A80932F0A8AE090E0A0E0B0E0F0
:108DF0008093310A9093320AA093330AB093340AD5
:108E00008EEA92E8A1E0B0E08093350A9093360AAA
:108E1000A093370AB093380A6091990B70919A0B1E
:108E200080919B0B90919C0B20E030E048EC52E449
:108E30000F945D2E20E030E040E251E40C94A94F05
:108E400085E0F81609F08DC080916304882341F114
:108E500060911D0A70911E0A80911F0A9091200A4C
:108E600025E030E040E050E00F94752F25303105CB
:108E70004105510551F48DE99BE00E94E1329C01CE
:108E8000812F6BEE7AE14EE309C08DE99BE00E94F1
:108E9000E1329C01812F6BEE7AE140E200E0ADDC33
:108EA000EE2011F40C94B64F60911D0A70911E0AC9
:108EB00080911F0A9091200A25E030E040E050E0C8
:108EC0000F94752F253031054105510511F00C9493
:108ED000B64F0E940B398091610490916204909387
:108EE0002A0A8093290A80911D0A90911E0A909364
:108EF0002C0A80932B0A82E08093630488EC97E528
:108F0000909362048093610483EE9AE190932E0A19
:108F100080932D0A8DE99BE09093300A80932F0A6D
:108F200081E090E0A0E0B0E08093310A9093320AB3
:108F3000A093330AB093340A8DED93E0A0E0B0E043
:108F40008093350A9093360AA093370AB093380A73
:108F500060919D0B70919E0B80919F0B9091A00B47
:108F6000A0C526E0F21609F08BC080916304882327
:108F700041F160911D0A70911E0A80911F0A909123
:108F8000200A25E030E040E050E00F94752F2630B5
:108F900031054105510551F489E59BE00E94E1321C
:108FA0009C01812F6CED7AE14EE309C089E59BE0DD
:108FB0000E94E1329C01812F6CED7AE140E200E0F9
:108FC0001CDCEE2009F4D2C760911D0A70911E0AC4
:108FD00080911F0A9091200A25E030E040E050E0A7
:108FE0000F94752F263031054105510509F0BEC794
:108FF0000E940B39809161049091620490932A0A37
:109000008093290A80911D0A90911E0A90932C0A40
:1090100080932B0A82E08093630488EC97E5909319
:1090200062048093610485ED9AE190932E0A809307
:109030002D0A89E59BE09093300A80932F0A81E006
:1090400090E0A0E0B0E08093310A9093320AA093C0
:10905000330AB093340A86EE93E0A0E0B0E0809348
:10906000350A9093360AA093370AB093380A609174
:10907000590B70915A0B80915B0B90915C0B11C551
:1090800087E0F81609F08BC080916304882341F1D2
:1090900060911D0A70911E0A80911F0A9091200A0A
:1090A00025E030E040E050E00F94752F2730310587
:1090B0004105510551F48DE59BE00E94E1329C0190
:1090C000812F6EEC7AE14EE309C08DE59BE00E94B2
:1090D000E1329C01812F6EEC7AE140E200E08DDB11
:1090E000EE2009F443C760911D0A70911E0A809119
:1090F0001F0A9091200A25E030E040E050E00F94F4
:10910000752F273031054105510509F02FC70E9401
:109110000B39809161049091620490932A0A8093A4
:10912000290A80911D0A90911E0A90932C0A80931F
:109130002B0A82E08093630488EC97E590936204A5
:109140008093610487EC9AE190932E0A80932D0A14
:109150008DE59BE09093300A80932F0A81E090E0A8
:10916000A0E0B0E08093310A9093320AA093330AD2
:10917000B093340A86EE93E0A0E0B0E08093350A25
:109180009093360AA093370AB093380A60915D0B2A
:1091900070915E0B80915F0B9091600B82C428E010
:1091A000F21609F08BC080916304882341F160912D
:1091B0001D0A70911E0A80911F0A9091200A25E0D5
:1091C00030E040E050E00F94752F28303105410524
:1091D000510551F481E69BE00E94E1329C01812F10
:1091E00060EC7AE14EE309C081E69BE00E94E13247
:1091F0009C01812F60EC7AE140E200E0FEDAEE2093
:1092000009F4B4C660911D0A70911E0A80911F0A6C
:109210009091200A25E030E040E050E00F94752F57
:10922000283031054105510509F0A0C60E940B39CF
:10923000809161049091620490932A0A8093290A94
:1092400080911D0A90911E0A90932C0A80932B0AFC
:1092500082E08093630488EC97E5909362048093A6
:10926000610489EB9AE190932E0A80932D0A81E69E
:109270009BE09093300A80932F0A81E090E0A0E079
:10928000B0E08093310A9093320AA093330AB093EE
:10929000340A86EE93E0A0E0B0E08093350A909324
:1092A000360AA093370AB093380A6091610B709127
:1092B000620B8091630B9091640BF3C389E0F81605
:1092C00009F08BC080916304882341F160911D0AED
:1092D00070911E0A80911F0A9091200A25E030E0CB
:1092E00040E050E00F94752F2930310541055105BC
:1092F00051F485E69BE00E94E1329C01812F62EBF4
:109300007AE14EE309C085E69BE00E94E1329C01D0
:10931000812F62EB7AE140E200E06FDAEE2009F49F
:1093200025C660911D0A70911E0A80911F0A9091B6
:10933000200A25E030E040E050E00F94752F2930FE
:1093400031054105510509F011C60E940B39809184
:1093500061049091620490932A0A8093290A809173
:109360001D0A90911E0A90932C0A80932B0A82E08A
:109370008093630488EC97E5909362048093610482
:109380008BEA9AE190932E0A80932D0A85E69BE062
:109390009093300A80932F0A81E090E0A0E0B0E043
:1093A0008093310A9093320AA093330AB093340A1F
:1093B00086EE93E0A0E0B0E08093350A9093360A01
:1093C000A093370AB093380A6091650B7091660BD1
:1093D0008091670B9091680B64C32AE0F21609F044
:1093E00087C080916304882341F160911D0A7091C8
:1093F0001E0A80911F0A9091200A25E030E040E08B
:1094000050E00F94752F2A3031054105510551F474
:1094100089E89BE00E94E1329C01812F66EA7AE1B3
:109420004EE309C089E89BE00E94E1329C01812F54
:1094300066EA7AE140E200E0E0D9EE2009F496C560
:1094400060911D0A70911E0A80911F0A9091200A56
:1094500025E030E040E050E00F94752F2A303105D0
:109460004105510509F082C50E940B3980916104C4
:109470009091620490932A0A8093290A80911D0A90
:1094800090911E0A90932C0A80932B0A82E080937D
:10949000630488EC97E5909362048093610481EA09
:1094A0009AE190932E0A80932D0A89E89BE090938D
:1094B000300A80932F0A1092310A1092320A1092C9
:1094C000330A1092340A87EE93E0A0E0B0E0809374
:1094D000350A9093360AA093370AB093380A609100
:1094E000890B70918A0B80918B0B90918C0B33C5FB
:1094F0008BE0F81609F087C080916304882341F15E
:1095000060911D0A70911E0A80911F0A9091200A95
:1095100025E030E040E050E00F94752F2B3031050E
:109520004105510551F481EA9BE00E94E1329C0122
:10953000812F67E97AE14EE309C081EA9BE00E944E
:10954000E1329C01812F67E97AE140E200E055D9E0
:10955000EE2009F40BC560911D0A70911E0A8091DE
:109560001F0A9091200A25E030E040E050E00F947F
:10957000752F2B3031054105510509F0F7C40E94C4
:109580000B39809161049091620490932A0A809330
:10959000290A80911D0A90911E0A90932C0A8093AB
:1095A0002B0A82E08093630488EC97E59093620431
:1095B000809361048DE89AE190932E0A80932D0A9E
:1095C00081EA9BE09093300A80932F0A1092310A2F
:1095D0001092320A1092330A1092340A87EE93E006
:1095E000A0E0B0E08093350A9093360AA093370A42
:1095F000B093380A6091A10B7091A20B8091A30BDC
:109600009091A40BA8C42CE0F21609F067C08091D9
:109610006304882309F444C060911D0A70911E0AF6
:1096200080911F0A9091200A25E030E040E050E050
:109630000F94752F2C30310541055105C1F460910F
:10964000790B70917A0B80917B0B90917C0B0F942E
:109650001D2C69837A838B839C83CE0101960E94A3
:10966000F8329C01812F66E87AE14EE317C06091E1
:10967000790B70917A0B80917B0B90917C0B0F94FE
:109680001D2C6D837E838F839887CE0105960E9463
:10969000F8329C01812F66E87AE140E200E0ADD823
:1096A000EE2009F463C460911D0A70911E0A809136
:1096B0001F0A9091200A25E030E040E050E00F942E
:1096C000752F2C3031054105510509F04FC40E941A
:1096D0000B398FE79AE169E77BE03CC18DE0F81632
:1096E00009F065C080916304882309F442C0609149
:1096F0001D0A70911E0A80911F0A9091200A25E090
:1097000030E040E050E00F94752F2D3031054105D9
:109710005105B9F460917D0B70917E0B80917F0BA8
:109720009091800B0F941D2C69877A878B879C877B
:10973000C1010E94F8329C01812F68E77AE14EE373
:1097400016C060917D0B70917E0B80917F0B909184
:10975000800B0F941D2C6D877E878F87988BC2019D
:109760000E94F8329C01812F68E77AE140E200E034
:1097700044D8EE2009F4FAC360911D0A70911E0AC4
:1097800080911F0A9091200A25E030E040E050E0EF
:109790000F94752F2D3031054105510509F0E6C3B1
:1097A0000E940B3981E79AE16DE77BE0D3C02EE0A0
:1097B000F21609F066C080916304882309F443C05F
:1097C00060911D0A70911E0A80911F0A9091200AD3
:1097D00025E030E040E050E00F94752F2E30310549
:1097E00041055105B9F46091810B7091820B809114
:1097F000830B9091840B0F941D2C698B7A8B8B8B30
:109800009C8BC3010E94F8329C01812F6AE67AE1A9
:109810004EE316C06091810B7091820B8091830B97
:109820009091840B0F941D2C6D8B7E8B8F8B988F5A
:10983000C4010E94F8329C01812F6AE67AE140E27D
:1098400000E00E94FD43EE2009F490C360911D0AE0
:1098500070911E0A80911F0A9091200A25E030E045
:1098600040E050E00F94752F2E3031054105510531
:1098700009F07CC30E940B3983E69AE161E87BE042
:1098800069C08FE0F81609F077C0809163048823DF
:1098900009F443C060911D0A70911E0A80911F0A4D
:1098A0009091200A25E030E040E050E00F94752FC1
:1098B0002F30310541055105B9F46091850B709148
:1098C000860B8091870B9091880B0F941D2C698FCC
:1098D0007A8F8B8F9C8FC5010E94F8329C01812F5B
:1098E0006CE57AE14EE316C06091850B7091860BB2
:1098F0008091870B9091880B0F941D2C6D8F7E8F1C
:109900008F8F98A3C6010E94F8329C01812F6CE5CD
:109910007AE140E200E00E94FD43EE2009F426C314
:1099200060911D0A70911E0A80911F0A9091200A71
:1099300025E030E040E050E00F94752F2F303105E6
:109940004105510509F012C30E940B3985E59AE1E2
:1099500065E87BE024E630E040E050E0F8EBEF2EF5
:10996000F2E8FF2EF1E00F2F112DE2E1CE2EE4EA16
:10997000DE2E0E942F3039C320E1F21609F096C086
:1099800080916304882349F160911D0A70911E0A39
:1099900080911F0A9091200A25E030E040E050E0DD
:1099A0000F94752F203131054105510551F481E99E
:1099B0009BE00E94F8329C01812F6BE47AE14EE338
:1099C00009C081E99BE00E94F8329C01812F6BE481
:1099D0007AE140E200E00E94FD43EE2009F4C6C2B5
:1099E00060911D0A70911E0A80911F0A9091200AB1
:1099F00025E030E040E050E00F94752F2031310534
:109A00004105510509F0B2C20E940B3980916104F1
:109A10009091620490932A0A8093290A80911D0AEA
:109A200090911E0A90932C0A80932B0A82E08093D7
:109A3000630483E297E5909362048093610481E478
:109A40009AE190932E0A80932D0A81E99BE09093EE
:109A5000300A80932F0A81E090E0A0E0B0E080938C
:109A6000310A9093320AA093330AB093340A8DEDF1
:109A700093E0A0E0B0E08093350A9093360AA0937B
:109A8000370AB093380A6091910B7091920B8091D4
:109A9000930B9091940B2AE037ED43E25CE30F9433
:109AA0005D2E20E030E040E85FE353C281E1F8162C
:109AB00009F08CC080916304882349F160911D0AEC
:109AC00070911E0A80911F0A9091200A25E030E0D3
:109AD00040E050E00F94752F2131310541055105CB
:109AE00051F489E69BE00E9422349C01812F67E3B8
:109AF0007AE14EE309C089E69BE00E9422349C0192
:109B0000812F67E37AE140E200E00E94FD43EE200E
:109B100009F42CC260911D0A70911E0A80911F0ADF
:109B20009091200A25E030E040E050E00F94752F3E
:109B3000213131054105510509F018C20E940B3948
:109B4000809161049091620490932A0A8093290A7B
:109B500080911D0A90911E0A90932C0A80932B0AE3
:109B600082E08093630489ED95E59093620480938D
:109B700061048DE29AE190932E0A80932D0A89E682
:109B80009BE09093300A80932F0A84EF91E0A0E04D
:109B9000B0E08093310A9093320AA093330AB093D5
:109BA000340A88EE9FE3AFE0B0E08093350A9093EB
:109BB000360AA093370AB093380A6091690B709106
:109BC0006A0B80916B0B90916C0B8FC022E1F216A7
:109BD00009F096C080916304882349F160911D0AC1
:109BE00070911E0A80911F0A9091200A25E030E0B2
:109BF00040E050E00F94752F2231310541055105A9
:109C000051F48DE69BE00E9422349C01812F63E297
:109C10007AE14EE309C08DE69BE00E9422349C016C
:109C2000812F63E27AE140E200E00E94FD43EE20F2
:109C300009F49CC160911D0A70911E0A80911F0A4F
:109C40009091200A25E030E040E050E00F94752F1D
:109C5000223131054105510509F088C10E940B39B7
:109C6000809161049091620490932A0A8093290A5A
:109C700080911D0A90911E0A90932C0A80932B0AC2
:109C800082E08093630489ED95E59093620480936C
:109C9000610489E19AE190932E0A80932D0A8DE662
:109CA0009BE09093300A80932F0A84EF91E0A0E02C
:109CB000B0E08093310A9093320AA093330AB093B4
:109CC000340A88EE9FE3AFE0B0E08093350A9093CA
:109CD000360AA093370AB093380A60916D0B7091E1
:109CE0006E0B80916F0B9091700B20E030E048EC90
:109CF00052E40F945D2E20E030E04AEF53E429C196
:109D000083E1F81609F08CC080916304882349F13F
:109D100060911D0A70911E0A80911F0A9091200A7D
:109D200025E030E040E050E00F94752F23313105FD
:109D30004105510551F481E79BE00E949B339C0152
:109D4000812F6FE07AE14EE309C081E79BE00E943A
:109D50009B339C01812F6FE07AE140E200E00E949A
:109D6000FD43EE2009F402C160911D0A70911E0AA4
:109D700080911F0A9091200A25E030E040E050E0F9
:109D80000F94752F233131054105510509F0EEC0BF
:109D90000E940B39809161049091620490932A0A89
:109DA0008093290A80911D0A90911E0A90932C0A93
:109DB00080932B0A82E0809363048EE796E590936C
:109DC00062048093610485E09AE190932E0A809367
:109DD0002D0A81E79BE09093300A80932F0A82E35B
:109DE00090E0A0E0B0E08093310A9093320AA09313
:109DF000330AB093340A84E696E8A1E0B0E0809399
:109E0000350A9093360AA093370AB093380A6091C6
:109E1000710B7091720B8091730B9091740B8FC0CA
:109E200024E1F21609F0A2C080916304882349F16D
:109E300060911D0A70911E0A80911F0A9091200A5C
:109E400025E030E040E050E00F94752F24313105DB
:109E50004105510551F485E79BE00E949B339C012D
:109E6000812F6BEF79E14EE309C085E79BE00E940B
:109E70009B339C01812F6BEF79E140E200E00E946F
:109E8000FD43EE2009F472C060911D0A70911E0A14
:109E900080911F0A9091200A25E030E040E050E0D8
:109EA0000F94752F243131054105510509F05EC02D
:109EB0000E940B39809161049091620490932A0A68
:109EC0008093290A80911D0A90911E0A90932C0A72
:109ED00080932B0A82E0809363048EE796E590934B
:109EE00062048093610481EF99E190932E0A80933C
:109EF0002D0A85E79BE09093300A80932F0A82E336
:109F000090E0A0E0B0E08093310A9093320AA093F1
:109F1000330AB093340A84E696E8A1E0B0E0809377
:109F2000350A9093360AA093370AB093380A6091A5
:109F3000750B7091760B8091770B9091780B20E0E8
:109F400030E040E251E40F945D2E20E030E048E440
:109F500052E40F94A32A0F94F12B60931D0A70937F
:109F60001E0A80931F0A9093200A3FC080911D0A09
:109F700090911E0AA0911F0AB091200A893691057E
:109F8000A105B10560F088E690E0A0E0B0E0809324
:109F90001D0A90931E0AA0931F0AB093200A609195
:109FA0001D0A70911E0A80911F0A9091200A25E0D7
:109FB00030E040E050E00F94752F422F8091170A57
:109FC00090E0049630E0821793074CF4445040939D
:109FD000170A81E080936304F42EFA941FEF1F5F49
:109FE000153018F4F3940C94D744A0960FB6F89457
:109FF000DEBF0FBECDBFCF91DF911F910F91FF90BC
:10A00000EF90DF90CF90BF90AF909F908F907F9018
:10A010006F905F904F903F902F9008952F923F92B6
:10A020004F925F926F927F928F929F92AF92BF9268
:10A03000CF92DF92EF92FF920F931F93DF93CF9314
:10A04000CDB7DEB72C970FB6F894DEBF0FBECDBFED
:10A0500080911D0A90911E0AA0911F0AB091200ABA
:10A0600081509048A040B04040F010921D0A1092DC
:10A070001E0A10921F0A1092200A60911D0A709108
:10A080001E0A80911F0A9091200A25E030E040E0EE
:10A0900050E00F94752F79018A018091170A90E0A2
:10A0A000A0E0B0E0E816F9060A071B0710F42093B9
:10A0B000170AC090170A8091160A90E09695879526
:10A0C00096958795BB24B394B822DD2469E0462E8B
:10A0D000512C4C0E5D1E55E0252E312C2C0E3D1EB4
:10A0E00047E2642E712C812C912CAA24A394CC20BD
:10A0F00099F5809163048823C1F080911D0A9091A5
:10A100001E0AA0911F0AB091200A0597A105B1056A
:10A1100028F48D2D61E47DE14BEF04C08D2D61E4C9
:10A120007DE140E22BEF0E942035BB2009F4D7C22D
:10A1300080911D0A90911E0AA0911F0AB091200AD9
:10A140000597A105B10508F0CAC20E940B3984E742
:10A150009FE50E94473902C481E0C81609F088C013
:10A1600080916304882349F160911D0A70911E0A51
:10A1700080911F0A9091200A25E030E040E050E0F5
:10A180000F94752F213031054105510551F48EEBA7
:10A1900094E00E94A1329C018D2D6BE37DE14EE3A2
:10A1A00009C08EEB94E00E94A1329C018D2D6BE3DF
:10A1B0007DE140E200E00E94FD43BB2009F48FC234
:10A1C00060911D0A70911E0A80911F0A9091200AC9
:10A1D00025E030E040E050E00F94752F213031054C
:10A1E0004105510509F07BC20E940B398091610441
:10A1F0009091620490932A0A8093290A80911D0A03
:10A2000090911E0A90932C0A80932B0A82E08093EF
:10A21000630481E698E5909362048093610485E38A
:10A220009DE190932E0A80932D0A8EEB94E09093FB
:10A23000300A80932F0A8AE090E0A0E0B0E080939B
:10A24000310A9093320AA093330AB093340A8DED09
:10A2500093E0A0E0B0E08093350A9093360AA09393
:10A26000370AB093380A8091BE049091BF04A7C109
:10A2700022E0C21609F090C080916304882349F15E
:10A2800060911D0A70911E0A80911F0A9091200A08
:10A2900025E030E040E050E00F94752F223031058A
:10A2A0004105510551F484E59AE00E94A1329C01D8
:10A2B0008D2D6EE27DE14EE309C084E59AE00E94B7
:10A2C000A1329C018D2D6EE27DE140E200E00E9412
:10A2D000FD43BB2009F403C260911D0A70911E0A60
:10A2E00080911F0A9091200A25E030E040E050E084
:10A2F0000F94752F223031054105510509F0EFC14A
:10A300000E940B39809161049091620490932A0A13
:10A310008093290A80911D0A90911E0A90932C0A1D
:10A3200080932B0A82E08093630481E698E5909302
:10A3300062048093610487E29DE190932E0A8093EA
:10A340002D0A84E59AE09093300A80932F0A1092A8
:10A35000310A1092320A1092330A1092340A82E2C1
:10A3600091E0A0E0B0E08093350A9093360AA09384
:10A37000370AB093380A8091540A9091550AAA2757
:10A3800097FDA095BA2F80931D0A90931E0AA09363
:10A390001F0AB093200AE2C283E0C81609F084C005
:10A3A00080916304882349F160911D0A70911E0A0F
:10A3B00080911F0A9091200A25E030E040E050E0B3
:10A3C0000F94752F233031054105510551F486E571
:10A3D0009AE00E94A1329C018D2D63E27DE14EE363
:10A3E00009C086E59AE00E94A1329C018D2D63E2AE
:10A3F0007DE140E200E00E94FD43BB2009F46FC113
:10A4000060911D0A70911E0A80911F0A9091200A86
:10A4100025E030E040E050E00F94752F2330310507
:10A420004105510509F05BC10E940B39809161041F
:10A430009091620490932A0A8093290A80911D0AC0
:10A4400090911E0A90932C0A80932B0A82E08093AD
:10A45000630481E698E590936204809361048FE140
:10A460009DE190932E0A80932D0A86E59AE09093C1
:10A47000300A80932F0A1092310A1092320A1092F9
:10A48000330A1092340A87E890E0A0E0B0E08093AD
:10A49000350A9093360AA093370AB093380A809110
:10A4A000560A9091570A6BCF24E0C21609F08FC06C
:10A4B00080916304882349F160911D0A70911E0AFE
:10A4C00080911F0A9091200A25E030E040E050E0A2
:10A4D0000F94752F243031054105510551F480EC5E
:10A4E00094E00E94A1329C018D2D6AE17DE14EE352
:10A4F00009C080EC94E00E94A1329C018D2D6AE19C
:10A500007DE140E200E00E94FD43BB2009F4E7C08A
:10A5100060911D0A70911E0A80911F0A9091200A75
:10A5200025E030E040E050E00F94752F24303105F5
:10A530004105510509F0D3C00E940B398091610497
:10A540009091620490932A0A8093290A80911D0AAF
:10A5500090911E0A90932C0A80932B0A82E080939C
:10A56000630481E698E5909362048093610485E139
:10A570009DE190932E0A80932D0A80EC94E09093B5
:10A58000300A80932F0A8AE090E0A0E0B0E0809348
:10A59000310A9093320AA093330AB093340A8DEDB6
:10A5A00093E0A0E0B0E08093350A9093360AA09340
:10A5B000370AB093380A8091C0049091C104AA2749
:10A5C00097FDA095BA2F0A97A109B109DCCE85E0C5
:10A5D000C81609F084C080916304882349F1609112
:10A5E0001D0A70911E0A80911F0A9091200A25E091
:10A5F00030E040E050E00F94752F253031054105E3
:10A60000510551F488ED93E10E94A1329C018D2DFA
:10A610006BE07DE14EE309C088ED93E10E94A13239
:10A620009C018D2D6BE07DE140E200E00E94FD4346
:10A63000BB2009F454C060911D0A70911E0A8091DC
:10A640001F0A9091200A25E030E040E050E00F948E
:10A65000752F253031054105510509F040C00E9494
:10A660000B39809161049091620490932A0A80933F
:10A67000290A80911D0A90911E0A90932C0A8093BA
:10A680002B0A82E08093630481E698E5909362044C
:10A690008093610481E09DE190932E0A80932D0ABE
:10A6A00088ED93E19093300A80932F0A1092310A3B
:10A6B0001092320A1092330A1092340A8FEF90E00F
:10A6C000A0E0B0E08093350A9093360AA093370A51
:10A6D000B093380A8091D8139091D91350CE8091BD
:10A6E000B50B9091B60B7C0100E010E0E982FA8294
:10A6F0000B831C8326E0C21609F0B3C0809163046B
:10A700008823B9F160911D0A70911E0A80911F0A79
:10A710009091200A25E030E040E050E00F94752F42
:10A72000263031054105510589F4C801B7010F9460
:10A730001D2C6D837E838F839887C1010E94F83220
:10A740009C018D2D6BEF7CE14EE310C0C801B70179
:10A750000F941D2C69877A878B879C87C2010E9482
:10A76000F8329C018D2D6BEF7CE140E200E00E940D
:10A77000FD43BB2009F4B8C060911D0A70911E0A08
:10A7800080911F0A9091200A25E030E040E050E0DF
:10A790000F94752F263031054105510509F0A4C0ED
:10A7A0000E940B3969817A818B819C81209161049F
:10A7B0003091620430932A0A2093290A20911D0ABD
:10A7C00030911E0A30932C0A20932B0A22E020930A
:10A7D000630427E235E5309362042093610425EF9A
:10A7E0003CE130932E0A20932D0A9E012F5F3F4FAC
:10A7F0003093300A20932F0A0F941D2C2AE037ED56
:10A8000043E25CE30F945D2E7B018C010F94EC2BF3
:10A810006093310A7093320A8093330A9093340A1A
:10A820000F941F2C9B01AC01C801B7010F94A32A00
:10A830007B018C010F94EC2B6093350A7093360AE0
:10A840008093370A9093380AC801B7010F94F12B0F
:10A8500060931D0A70931E0A80931F0A9093200A2A
:10A860007DC087E0C81609F03FC08091630488234B
:10A87000F9F060911D0A70911E0A80911F0A909153
:10A88000200A25E030E040E050E00F94752F27309B
:10A8900031054105510529F48D2D65EE7CE14EE32E
:10A8A00004C08D2D65EE7CE140E220E20E9420355F
:10A8B000BB20D1F060911D0A70911E0A80911F0A81
:10A8C0009091200A25E030E040E050E00F94752F91
:10A8D000273031054105510539F40E940B3980EECE
:10A8E0009CE10F9418093AC080911D0A90911E0AAC
:10A8F000A0911F0AB091200A8897A105B10540F0E8
:10A9000060921D0A70921E0A80921F0A9092200A7D
:10A9100060911D0A70911E0A80911F0A9091200A71
:10A9200025E030E040E050E00F94752F422F8091F9
:10A93000170A90E0049630E0821793074CF44450D5
:10A940004093170AA0926304C42ECA94DD24DA94BB
:10A95000D39424E02D1510F0C394C9CB2C960FB6D8
:10A96000F894DEBF0FBECDBFCF91DF911F910F9145
:10A97000FF90EF90DF90CF90BF90AF909F908F901F
:10A980007F906F905F904F903F902F900895EEE3EF
:10A99000F4E001900020E9F73197EE53F4401E16E1
:10A9A0001F0654F4DF01A25CBB4F80E202C08D930E
:10A9B0003196E431F105DCF31092520482E0809389
:10A9C00063040895CF92DF92EF92FF920F931F934B
:10A9D0007C01D62EC72E0FED19E08091DF098B5137
:10A9E0001092130A8093140AC801019762E97DE36B
:10A9F0000F946522C7010E94103505501040C80110
:10AA00006AE30F947D2AED2DFC2DDF010D900020CF
:10AA1000E9F72091DF092B51EA1BFB0B7396CF015D
:10AA2000A3E0880F991FAA95E1F78E1B9F0B8093D7
:10AA3000130A2093140AC8016D2D7C2D0F94A12AAE
:10AA40001F910F91FF90EF90DF90CF9008950F939B
:10AA50001F93DF93CF9300D00F92CDB7DEB78091D5
:10AA60001D0A90911E0AA0911F0AB091200AB7FFFB
:10AA700008C010921D0A10921E0A10921F0A10920E
:10AA8000200A2091350A3091360A4091370A5091B8
:10AA9000380A80911D0A90911E0AA0911F0AB09158
:10AAA000200A281739074A075B0744F420931D0A38
:10AAB00030931E0A40931F0A5093200A809163042A
:10AAC000882359F100912D0A10912E0A60911D0AD8
:10AAD00070911E0A80911F0A9091200A2091310ADC
:10AAE0003091320A4091330A5091340A620F731F39
:10AAF000841F951F0F941D2C2AE037ED43E25CE381
:10AB00000F94842B69837A838B839C83CE01019677
:10AB10000E94F832BC01C80155DF8091160A82FFFD
:10AB200034C000912F0A1091300A60911D0A709173
:10AB30001E0A80911F0A9091200A2091310A3091BB
:10AB4000320A4091330A5091340A620F731F841FF6
:10AB5000951F0F941D2C2AE037ED43E25CE30F9420
:10AB6000842B0F94F12BF80160837183828393838C
:10AB700040912B0A50912C0A60E070E08091290AE4
:10AB800090912A0A21E00E942F390F900F900F9088
:10AB90000F90CF91DF911F910F91089558DF809111
:10ABA000160A82FF05C0E091390AF0913A0A199518
:10ABB00008950F931F93DF93CF9300D00F92CDB7DB
:10ABC000DEB780911D0A90911E0AA0911F0AB091D4
:10ABD000200AB7FF08C010921D0A10921E0A109298
:10ABE0001F0A1092200A2091350A3091360A4091AE
:10ABF000370A5091380A80911D0A90911E0AA0913F
:10AC00001F0AB091200A281739074A075B0744F446
:10AC100020931D0A30931E0A40931F0A5093200A66
:10AC200080916304882359F100912D0A10912E0A16
:10AC300060911D0A70911E0A80911F0A9091200A4E
:10AC40002091310A3091320A4091330A5091340AEE
:10AC5000620F731F841F951F0F941F2C20E030E09C
:10AC600048EC52E40F94842B69837A838B839C8312
:10AC7000CE0101960E942234BC01C801A3DE80915E
:10AC8000160A82FF32C000912F0A1091300A60919B
:10AC90001D0A70911E0A80911F0A9091200A20912E
:10ACA000310A3091320A4091330A5091340A620FCE
:10ACB000731F841F951F0F941F2C20E030E048EC79
:10ACC00052E40F94842BF801608371838283938311
:10ACD00040912B0A50912C0A60E070E08091290A83
:10ACE00090912A0A21E00E942F390F900F900F9027
:10ACF0000F90CF91DF911F910F9108950F931F93A4
:10AD0000DF93CF9300D00F92CDB7DEB780911D0AAD
:10AD100090911E0AA0911F0AB091200AB7FF08C0A7
:10AD200010921D0A10921E0A10921F0A1092200AF9
:10AD30002091350A3091360A4091370A5091380AED
:10AD400080911D0A90911E0AA0911F0AB091200ABD
:10AD5000281739074A075B0744F420931D0A3093EC
:10AD60001E0A40931F0A5093200A8091630488238F
:10AD700059F100912D0A10912E0A60911D0A7091CF
:10AD80001E0A80911F0A9091200A2091310A309169
:10AD9000320A4091330A5091340A620F731F841FA4
:10ADA000951F0F941F2C20E030E040E251E40F94F7
:10ADB000842B69837A838B839C83CE0101960E94C6
:10ADC0009B33BC01C801FEDD8091160A82FF32C0B0
:10ADD00000912F0A1091300A60911D0A70911E0A8D
:10ADE00080911F0A9091200A2091310A3091320AF5
:10ADF0004091330A5091340A620F731F841F951FCC
:10AE00000F941F2C20E030E040E251E40F94842B9B
:10AE1000F801608371838283938340912B0A509160
:10AE20002C0A60E070E08091290A90912A0A21E0C2
:10AE30000E942F390F900F900F900F90CF91DF91BC
:10AE40001F910F9108950F931F93DF93CF9300D01D
:10AE50000F92CDB7DEB780911D0A90911E0AA09186
:10AE60001F0AB091200AB7FF08C010921D0A109265
:10AE70001E0A10921F0A1092200A2091350A309162
:10AE8000360A4091370A5091380A80911D0A9091F4
:10AE90001E0AA0911F0AB091200A281739074A07F5
:10AEA0005B0744F420931D0A30931E0A40931F0A47
:10AEB0005093200A80916304882359F100912D0A50
:10AEC00010912E0A60911D0A70911E0A80911F0A2E
:10AED0009091200A2091310A3091320A4091330A30
:10AEE0005091340A620F731F841F951F0F941F2CFB
:10AEF0002AE037ED43E25CE30F94842B69837A8385
:10AF00008B839C83CE0101960E94F832BC01C8015C
:10AF100059DD8091160A82FF32C000912F0A1091EC
:10AF2000300A60911D0A70911E0A80911F0A90914B
:10AF3000200A2091310A3091320A4091330A50910F
:10AF4000340A620F731F841F951F0F941F2C2AE071
:10AF500037ED43E25CE30F94842BF8016083718347
:10AF60008283938340912B0A50912C0A60E070E019
:10AF70008091290A90912A0A21E00E942F390F908E
:10AF80000F900F900F90CF91DF911F910F91089527
:10AF90000F931F93DF93CF9300D00F92CDB7DEB7FF
:10AFA00080911D0A90911E0AA0911F0AB091200A5B
:10AFB000B7FF08C010921D0A10921E0A10921F0AB5
:10AFC0001092200A2091350A3091360A4091370AB2
:10AFD0005091380A80911D0A90911E0AA0911F0A73
:10AFE000B091200A281739074A075B0744F42093D9
:10AFF0001D0A30931E0A40931F0A5093200A809125
:10B000006304882329F100912D0A10912E0A609182
:10B010001D0A70911E0A80911F0A9091200A2091AA
:10B02000310A3091320A4091330A5091340A620F4A
:10B03000731F841F951F0F941F2C69837A838B8342
:10B040009C83CE0101960E94E132BC01C801BADCAA
:10B050008091160A82FF2CC000912F0A1091300AAD
:10B0600060911D0A70911E0A80911F0A9091200A1A
:10B070002091310A3091320A4091330A5091340ABA
:10B08000620F731F841F951F0F941F2CF80160839C
:10B0900071838283938340912B0A50912C0A60E044
:10B0A00070E08091290A90912A0A21E00E942F39AC
:10B0B0000F900F900F900F90CF91DF911F910F91F4
:10B0C00008950F931F93DF93CF930F920F92CDB7F5
:10B0D000DEB780911D0A90911E0AA0911F0AB091BF
:10B0E000200AB7FF08C010921D0A10921E0A109283
:10B0F0001F0A1092200A2091350A3091360A409199
:10B10000370A5091380A80911D0A90911E0AA09129
:10B110001F0AB091200A281739074A075B0744F431
:10B1200020931D0A30931E0A40931F0A5093200A51
:10B13000809163048823B9F000912D0A10912E0AA2
:10B140008091310A9091320A20911D0A30911E0A95
:10B15000820F931F9A838983CE0101960E94A132A8
:10B16000BC01C8012FDC8091160A82FF1DC0E0914E
:10B170002F0AF091300A8091310A9091320A209181
:10B180001D0A30911E0A820F931F91838083409184
:10B190002B0A50912C0A60E070E08091290A90916E
:10B1A0002A0A21E00E942F390F900F90CF91DF9152
:10B1B0001F910F910895AF92BF92CF92DF92EF92BD
:10B1C000FF920F93DF93CF9300D00F92CDB7DEB7EE
:10B1D000E0901D0AF0901E0AF7FC11C06091CE139A
:10B1E0007091CF138091D0139091D11320E030E073
:10B1F00040E050E00F948B2D18160CF04BC0A0903F
:10B20000CE13B090CF13C090D013D090D113C601FD
:10B21000B50120E030E040E050E40F947D2B87FD45
:10B2200003C01E141F04B4F58091690A90916A0A44
:10B230008E0D9F1D90936A0A8093690AB701882733
:10B2400077FD8095982F0F941F2C2091710B3091D2
:10B25000720B4091730B5091740B0F94842B9B01D4
:10B26000AC01C601B5010F94A32A6093CE1370936D
:10B27000CF138093D0139093D11310921D0A109284
:10B280001E0A10921F0A1092200A81E08093D607AE
:10B290008093630480916304882309F4BCC0809187
:10B2A000CE139091CF13A091D013B091D113B05879
:10B2B00089839A83AB83BC83CE0101960E9485313A
:10B2C000BC0188E39BE17EDB6091CE137091CF13CC
:10B2D0008091D0139091D11320E030E040EC50E405
:10B2E0000F945D2E0F94F12B9B01AC018EED99E034
:10B2F00062E4422F22E00CE0B1E4EB2EBBE1FB2E36
:10B300000F9446238EED99E06CE348E123E001E0E1
:10B31000A9E5EA2EABE1FA2E0F9446238EED99E0D3
:10B3200060E04FE223E000E1FCE5EF2EFBE1FF2EC1
:10B330000F9446238EED99E06BE14CE324E032E07C
:10B340000F94DE228EED99E062E241E322E00AE012
:10B35000ECE8EE2EEBE1FE2E0F9446238EED99E005
:10B3600065E54FE223E000E170EAE72E7BE1F72E8E
:10B370000F9446238EED99E06BE64CE324E032E037
:10B380000F94DE228EED99E061E743E322E00AE0CC
:10B3900050EDE52E5BE1F52E0F9446238091770466
:10B3A0008823E1F08EED99E060E00F94F11F8EEDBF
:10B3B00099E061E74EE220E10DE00F94231E8EED4F
:10B3C00099E061E00F94F11F8EED99E061E740E3B1
:10B3D00022E034EEE32E3BE1F32E1BC08EED99E02C
:10B3E00060E00F94F11F8EED99E062E241E320E10D
:10B3F0000DE00F94231E8EED99E061E00F94F11F94
:10B400008EED99E062E241E322E0BEEFEB2EBBE17C
:10B41000FB2E0F9446238091160A82FF0DC01092D6
:10B42000D6070F94D10B81E694E440E050E060E051
:10B4300070E021E00E942F390F900F900F900F9035
:10B44000CF91DF910F91FF90EF90DF90CF90BF9061
:10B45000AF9008959F92AF92BF92CF92DF92EF92FA
:10B46000FF920F931F9360916B0470916C04809115
:10B470006D0490916E040E94D47360933B0A7093A4
:10B480003C0A80933D0A90933E0A60916F0470914C
:10B49000700480917104909172040E94E073609333
:10B4A0003F0A7093400A8093410A9093420A809128
:10B4B0001D0A90911E0AA0911F0AB091200A815086
:10B4C0009048A040B04040F010921D0A10921E0A11
:10B4D00010921F0A1092200A60911D0A70911E0A94
:10B4E00080911F0A9091200A25E030E040E050E072
:10B4F0000F94752F79018A018091170A90E0A0E0DE
:10B50000B0E0E816F9060A071B0710F42093170AA3
:10B51000F090170A8091160A90E096958795969577
:10B520008795EE24E394E82210E008E1A02EB12CE8
:10B53000C12CD12C99249394FF2099F58091630418
:10B540008823C1F080911D0A90911E0AA0911F0AC4
:10B55000B091200A0597A105B10528F4812F6BE46D
:10B560007CE14BEF04C0812F6BE47CE140E22BEFE8
:10B570000E942035EE2009F4F8C180911D0A9091B7
:10B580001E0AA0911F0AB091200A0597A105B105D6
:10B5900008F0EBC10E940B3984E79FE50E94473910
:10B5A0001CC281E0F81609F084C0809163048823EE
:10B5B00049F160911D0A70911E0A80911F0A9091B5
:10B5C000200A25E030E040E050E00F94752F213054
:10B5D00031054105510551F484E59AE00E94A132FC
:10B5E0009C01812F64E47CE14EE309C084E59AE08C
:10B5F0000E94A1329C01812F64E47CE140E200E0E2
:10B600000E94FD43EE2009F4B0C160911D0A7091C3
:10B610001E0A80911F0A9091200A25E030E040E048
:10B6200050E00F94752F213031054105510509F087
:10B630009CC10E940B3980916104909162049093A7
:10B640002A0A8093290A80911D0A90911E0A9093DC
:10B650002C0A80932B0A82E08093630481E698E5AC
:10B6600090936204809361048DE39CE190932E0A91
:10B6700080932D0A84E59AE09093300A80932F0AF4
:10B680001092310A1092320A1092330A1092340A40
:10B6900082E291E0A0E0B0E08093350A9093360A10
:10B6A000A093370AB093380A8091540A9091550AB2
:10B6B0000FC122E0F21609F084C080916304882350
:10B6C00049F160911D0A70911E0A80911F0A9091A4
:10B6D000200A25E030E040E050E00F94752F223042
:10B6E00031054105510551F486E59AE00E94A132E9
:10B6F0009C01812F69E37CE14EE309C086E59AE075
:10B700000E94A1329C01812F69E37CE140E200E0CC
:10B710000E94FD43EE2009F428C160911D0A70913A
:10B720001E0A80911F0A9091200A25E030E040E037
:10B7300050E00F94752F223031054105510509F075
:10B7400014C10E940B39809161049091620490931E
:10B750002A0A8093290A80911D0A90911E0A9093CB
:10B760002C0A80932B0A82E08093630481E698E59B
:10B77000909362048093610485E39CE190932E0A88
:10B7800080932D0A86E59AE09093300A80932F0AE1
:10B790001092310A1092320A1092330A1092340A2F
:10B7A00087E890E0A0E0B0E08093350A9093360AF5
:10B7B000A093370AB093380A8091560A9091570A9D
:10B7C00087C083E0F81609F090C080916304882355
:10B7D00049F160911D0A70911E0A80911F0A909193
:10B7E000200A25E030E040E050E00F94752F233030
:10B7F00031054105510551F488ED93E10E94A132D4
:10B800009C01812F6BE27CE14EE309C088ED93E15E
:10B810000E94A1329C01812F6BE27CE140E200E0BA
:10B820000E94FD43EE2009F4A0C060911D0A7091B2
:10B830001E0A80911F0A9091200A25E030E040E026
:10B8400050E00F94752F233031054105510509F063
:10B850008CC00E940B398091610490916204909396
:10B860002A0A8093290A80911D0A90911E0A9093BA
:10B870002C0A80932B0A82E08093630481E698E58A
:10B88000909362048093610481E29CE190932E0A7C
:10B8900080932D0A88ED93E19093300A80932F0ACC
:10B8A0001092310A1092320A1092330A1092340A1E
:10B8B0008FEF90E0A0E0B0E08093350A9093360AD5
:10B8C000A093370AB093380A8091D8139091D91376
:10B8D000AA2797FDA095BA2F80931D0A90931E0A60
:10B8E000A0931F0AB093200A78C024E0F216E9F56D
:10B8F000809163048823F9F060911D0A70911E0AFB
:10B9000080911F0A9091200A25E030E040E050E04D
:10B910000F94752F243031054105510529F4812FED
:10B9200068E17CE14EE304C0812F68E17CE140E204
:10B9300020E20E942035EE20C1F060911D0A709136
:10B940001E0A80911F0A9091200A25E030E040E015
:10B9500050E00F94752F243031054105510529F42D
:10B960000E940B390E945B3938C080911D0A90916A
:10B970001E0AA0911F0AB091200A4997A105B1059E
:10B9800040F0A0921D0AB0921E0AC0921F0AD092E7
:10B99000200A60911D0A70911E0A80911F0A9091E1
:10B9A000200A25E030E040E050E00F94752F422F50
:10B9B0008091170A90E0049630E08217930744F4D0
:10B9C00044504093170A90926304F42EFA941FEFA8
:10B9D0001F5F153010F4F394AFCD1F910F91FF90BE
:10B9E000EF90DF90CF90BF90AF909F9008958F928F
:10B9F0009F92AF92BF92CF92DF92EF92FF920F93FE
:10BA00001F9320911D0A30911E0A40911F0A5091E8
:10BA1000200A211531054105510509F464C0B90119
:10BA2000882777FD8095982F0F941F2C2091430A2B
:10BA30003091440A4091450A5091460A0F945D2E78
:10BA40009B01AC016091BB137091BC138091BD133D
:10BA50009091BE130F94A42A6093BB137093BC13F0
:10BA60008093BD139093BE1310921D0A10921E0A6C
:10BA700010921F0A1092200A0F920F926091AF133A
:10BA80007091B0138091B1139091B2132091B313C0
:10BA90003091B4134091B5135091B613E090B713A1
:10BAA000F090B8130091B9131091BA13E7EDF3E1D8
:10BAB000ADB7BEB71296FC93EE931197EBEBCE2E7B
:10BAC000E3E1DE2E0F2EF0E08F2EF0E09F2EF0E867
:10BAD000AF2EFFE3BF2EF02D0E948CAA81E0809351
:10BAE00063040F900F9080916304882349F08BEBDF
:10BAF00093E10E94EA30BC0181ED9CE10E94E25496
:10BB00008091160A82FF09C087EE9AE340E050E078
:10BB100060E070E021E00E942F391F910F91FF90AB
:10BB2000EF90DF90CF90BF90AF909F908F9008954F
:10BB30002F923F924F925F926F927F928F929F923D
:10BB4000AF92BF92CF92DF92EF92FF920F931F932B
:10BB5000DF93CF9300D000D0CDB7DEB79A8389832F
:10BB60001B017A01690180911D0A90911E0AA09122
:10BB70001F0AB091200A0097A105B10509F405C17B
:10BB80000E94F2CAF101EC59FB4F80818F3FD1F442
:10BB9000F101E050FB4F80810F94922420E030E0CF
:10BBA000892B11F421E030E0F101ED5FFA4F808143
:10BBB00090E02817390741F580911D0A90911E0ADF
:10BBC00097FD22C0F101EC59FB4F8081813009F0D3
:10BBD00044C0F101EA5FFA4F80810F94922420E083
:10BBE00030E0892B11F421E030E0F101E75FFA4FFA
:10BBF000808190E02817390739F480911D0A9091CF
:10BC00001E0A181619064CF58101000F111F000FAE
:10BC1000111F01551C4E60911D0A70911E0A882744
:10BC200077FD8095982F0F941F2C2091430A309117
:10BC3000440A4091450A5091460A0F945D2E9B019B
:10BC4000AC01D8016D917D918D919C910F94A42AA6
:10BC5000F8016083718382839383B701882777FD1E
:10BC60008095982F0F941F2C7B018C015101AA0CF9
:10BC7000BB1CAA0CBB1C8FEA93E1A80EB91ED50110
:10BC80006D917D918D919C91A80197010F947D2BD1
:10BC900088232CF4F501E082F18202831383B6013C
:10BCA000882777FD8095982F0F941F2C7B018C019E
:10BCB0006101CC0CDD1CCC0CDD1C8FEA93E1C80EBD
:10BCC000D91ED6016D917D918D919C91A80197010E
:10BCD0000F948B2D18162CF4F601E082F18202836A
:10BCE000138310921D0A10921E0A10921F0A1092BE
:10BCF000200A0F920F92CDB6DEB60894C11CD11C5B
:10BD00004090AF135090B0136090B1137090B21385
:10BD10008091B3139091B413A091B513B091B61361
:10BD20008B839C83AD83BE83E090B713F090B813F0
:10BD30000091B9131091BA13F101EE0FFF1FEE0F2E
:10BD4000FF1FE051FB4F608171818281938120E070
:10BD500030E040E752E40F94842B4B015C0187ED07
:10BD600093E1D6018D939C93C301B2012B813C8159
:10BD70004D815E81ABEBCA2EA3E1DA2E0E948CAA24
:10BD800081E0809363040F900F9080916304882377
:10BD900071F0220C331C220C331CC10181559C4EC6
:10BDA0000E94EA30BC0189819A810E94E25480910C
:10BDB000160A82FF09C087EE9AE340E050E060E097
:10BDC00070E021E00E942F3926960FB6F894DEBF6E
:10BDD0000FBECDBFCF91DF911F910F91FF90EF90DC
:10BDE000DF90CF90BF90AF909F908F907F906F909B
:10BDF0005F904F903F902F9008958AED9CE162E014
:10BE000070E040E050E02EE031E092CE8CED9CE11D
:10BE100061E070E04CEE5FEF21E331E089CE8EED22
:10BE20009CE160E070E04CEE5FEF2CE231E080CE10
:10BE3000FF920F931F938C01262FFC01F1AC049607
:10BE40006F2D42AD0F940523F80EF801F1AE81E09D
:10BE500090E01F910F91FF9008950F931F938CED29
:10BE600099E01092DD091092DC0928E135E0FC012F
:10BE7000329322938F011092130A1092140A109297
:10BE8000150A02966BE574E00F941D2080E195E0A1
:10BE9000F801918380831F910F910895BC018091D7
:10BEA000D707882341F48EE394E044E150E00E94F8
:10BEB00028280C94C75408950E947BBB10921C1133
:10BEC0008AE191E160E02DD70E94B87381E0809310
:10BED000DA138DE999E1E2DF1092E81382E59BE045
:10BEE0000E948D950C9434CDCF92DF92EF92FF9209
:10BEF0000F931F9380911D0A90911E0AA0911F0A13
:10BF0000B091200A81509048A040B04040F010927B
:10BF10001D0A10921E0A10921F0A1092200A6091A8
:10BF20001D0A70911E0A80911F0A9091200A25E037
:10BF300030E040E050E00F94752F79018A01809144
:10BF4000170A90E0A0E0B0E0E816F9060A071B0720
:10BF500010F42093170AF090170A8091160A90E0C7
:10BF60009695879596958795EE24E394E82200E0D0
:10BF700035E0D32ECC24C394FF2089F5809163044F
:10BF80008823C1F080911D0A90911E0AA0911F0A7A
:10BF9000B091200A0597A105B10528F4802F61E62C
:10BFA00079E14BEF04C0802F61E679E140E22BEFAD
:10BFB0000E942035EE2099F080911D0A90911E0A72
:10BFC000A0911F0AB091200A0597A105B10538F488
:10BFD0000E940B398DE99DE30E944739D1C20E942E
:10BFE00002A4882329F480911C11882309F4C3C278
:10BFF00081E0F81611F082E0BFC0809163048823CD
:10C00000F9F060911D0A70911E0A80911F0A9091AB
:10C01000200A25E030E040E050E00F94752F2130F9
:10C0200031054105510529F4802F6CE579E14EE396
:10C0300004C0802F6CE579E140E22AEF0E942035B0
:10C04000EE2009F4E3C060911D0A70911E0A8091F0
:10C050001F0A9091200A25E030E040E050E00F9464
:10C06000752F213031054105510509F0CFC00E94DF
:10C070000B398EE090E530C2809163048823F9F09B
:10C0800060911D0A70911E0A80911F0A9091200AEA
:10C0900025E030E040E050E00F94752F213031056D
:10C0A0004105510529F4802F63E579E14EE304C091
:10C0B000802F63E579E140E22AEF0E942035EE20EF
:10C0C00009F459C060911D0A70911E0A80911F0ADF
:10C0D0009091200A25E030E040E050E00F94752F69
:10C0E000213031054105510509F045C00E940B3949
:10C0F00085E99EE3F1C122E0F216E9F5809163043F
:10C100008823F9F060911D0A70911E0A80911F0A20
:10C110009091200A25E030E040E050E00F94752F28
:10C12000223031054105510529F4802F67E479E17A
:10C130004EE304C0802F67E479E140E22AEF0E94D9
:10C140002035EE20C1F060911D0A70911E0A809189
:10C150001F0A9091200A25E030E040E050E00F9463
:10C16000752F223031054105510529F40E940B3904
:10C170008AE29AE5B1C183E08F1509F048C0809149
:10C180006304882319F160911D0A70911E0A809141
:10C190001F0A9091200A25E030E040E050E00F9423
:10C1A000752F8F2D90E0A0E0B0E0281739074A07DF
:10C1B0005B0729F4802F69E379E14EE304C0802F07
:10C1C00069E379E140E22AEF0E942035EE20E1F0B8
:10C1D00060911D0A70911E0A80911F0A9091200A99
:10C1E00025E030E040E050E00F94752F8F2D90E077
:10C1F000A0E0B0E0281739074A075B0729F40E943E
:10C200000B3983E392E468C18F2D01C082E0182FBF
:10C210001F5F80911D11882309F417C18091EB12D3
:10C22000882309F4E1C080911C11882309F44AC0D5
:10C230001F1509F08FC080916304882319F1609164
:10C240001D0A70911E0A80911F0A9091200A25E014
:10C2500030E040E050E00F94752F8F2D90E0A0E08B
:10C26000B0E0281739074A075B0729F4802F6DE2F1
:10C2700079E14EE304C0802F6DE279E140E220E2F3
:10C280000E942035EE2009F465C060911D0A70916E
:10C290001E0A80911F0A9091200A25E030E040E0BC
:10C2A00050E00F94752F812F90E0A0E0B0E02817A8
:10C2B00039074A075B0709F04DC00E940B390E94FD
:10C2C0002F425EC11F1509F045C080916304882389
:10C2D00019F160911D0A70911E0A80911F0A9091B8
:10C2E000200A25E030E040E050E00F94752F8F2DBC
:10C2F00090E0A0E0B0E0281739074A075B0729F46F
:10C30000802F60E279E14EE304C0802F60E279E1A2
:10C3100040E220E20E942035EE20E1F060911D0A0B
:10C3200070911E0A80911F0A9091200A25E030E04A
:10C3300040E050E00F94752F812F90E0A0E0B0E036
:10C34000281739074A075B0729F40E940B390E9416
:10C350002B4216C11F5F1F1509F0C1C080916304F5
:10C36000882319F160911D0A70911E0A80911F0A9D
:10C370009091200A25E030E040E050E00F94752FC6
:10C38000812F90E0A0E0B0E0281739074A075B074B
:10C3900029F4802F65E179E14EE304C0802F65E147
:10C3A00079E140E220E20E942035EE2009F497C0B6
:10C3B00060911D0A70911E0A80911F0A9091200AB7
:10C3C00025E030E040E050E00F94752F812F90E0A1
:10C3D000A0E0B0E0281739074A075B0709F07FC0E3
:10C3E0000E940B3969DDCCC00E9402A4882309F0A9
:10C3F00077C080911C11882309F072C01F1509F0C5
:10C400006EC080916304882309F449C060911D0ABD
:10C4100070911E0A80911F0A9091200A25E030E059
:10C4200040E050E00F94752F8F2D90E0A0E0B0E039
:10C43000281739074A075B0721F4802F67E079E165
:10C4400025C0802F67E079E126C01F1509F047C09D
:10C4500080916304882319F160911D0A70911E0A6E
:10C4600080911F0A9091200A25E030E040E050E0E2
:10C470000F94752F8F2D90E0A0E0B0E028173907BA
:10C480004A075B0729F4802F6CEF78E14EE304C084
:10C49000802F6CEF78E140E22AEF0E942035EE20F9
:10C4A000F1F060911D0A70911E0A80911F0A90910F
:10C4B000200A25E030E040E050E00F94752F812FF6
:10C4C00090E0A0E0B0E0281739074A075B0739F48D
:10C4D0000E940B3981E290E40E944D3951C01F5FE8
:10C4E00060911D0A70911E0A80911F0A9091200A86
:10C4F00025E030E040E050E00F94752F812F90E070
:10C50000A0E0B0E0281739074A075B0780F01D9DBF
:10C51000C00111240197AA2797FDA095BA2F8093F7
:10C520001D0A90931E0AA0931F0AB093200A6091DF
:10C530001D0A70911E0A80911F0A9091200A25E021
:10C5400030E040E050E00F94752F422F8091170AA1
:10C5500090E0049630E08217930744F444504093EF
:10C56000170AC0926304F42EFA940FEF0F5F0530A0
:10C5700038F4F39401CD81E0F81609F0BCCD7CCD00
:10C580001F910F91FF90EF90DF90CF90089586DC80
:10C5900081E08093D7070C945339BC018091D70771
:10C5A000882341F48EE394E044E150E00E94AE28F9
:10C5B0000C94C7540895DF92EF92FF920F931F934C
:10C5C0000E94A93429B130E0A4E036952795AA95B8
:10C5D000E1F741E050E02427352721703070809149
:10C5E000210A90E02817390709F182E0809363045B
:10C5F00089B190E0F4E096958795FA95E1F7842764
:10C60000952781708093210A0E94023D8091210A22
:10C61000882331F08AE191E13CD68BE59DE105C0AC
:10C620008AE191E147D286E49DE138DCE090220A7C
:10C63000F090230A0091240A1091250A0F94E7250F
:10C64000E616F7060807190708F0FDC02091C9078C
:10C65000222361F181E080936304332727FD309525
:10C66000432F532F80911D0A90911E0AA0911F0AFB
:10C67000B091200A820F931FA41FB51F80931D0A3B
:10C6800090931E0AA0931F0AB093200A1092C90724
:10C690000F94E7256856754C8F4F9F4F6093500A53
:10C6A0007093510A8093520A9093530A8091160A0C
:10C6B00082FF0EC00F94E7256856754C8F4F9F4F31
:10C6C0006093500A7093510A8093520A9093530AD0
:10C6D00080914F0A8F5F80934F0A8AED99E00E9404
:10C6E000EF3CEDE7DE2E8EED99E06BE27AE00F9401
:10C6F0006522D092130A1092140A80914F0A80FF8B
:10C7000004C08EED99E061E003C08EED99E060E039
:10C710000F94F11F8EED99E06FE74FE30F94DA1F4E
:10C720008EED99E061E00F94F11FE0916104F091CA
:10C73000620419958091D607882309F447C0E090D8
:10C74000500AF090510A0091520A1091530A80E564
:10C7500099ECAFEFBFEFE80EF91E0A1F1B1F0F94F5
:10C76000E725E616F7060807190780F58EED99E02C
:10C7700060E00F94F11F8EED99E062E740E320E165
:10C780000DE00F94231E8EED99E062E241E320E17B
:10C790000F94231E8EED99E061E00F94F11F8EED52
:10C7A00099E061E743E322E00AE070EDE72E7BE1E8
:10C7B000F72E0F9446238EED99E062E241E322E0EA
:10C7C0005CE8E52E5BE1F52E0F944623809163042F
:10C7D000882339F08EED99E00F94C61F882309F065
:10C7E00082CFE090500AF090510A0091520A1091C5
:10C7F000530A0F94E725E616F7060807190770F4A1
:10C8000080916104909162048D599D4339F00E949A
:10C81000533982E0809363041092D60780916304B9
:10C82000882319F08150809363040F94E7256C5995
:10C830007F4F8F4F9F4F6093220A7093230A8093FC
:10C84000240A9093250A1F910F91FF90EF90DF909B
:10C8500008950E94023DE4E0F1E080818F7D8083B5
:10C8600080818F7B80839FB7F894E5E0F1E0808141
:10C87000806280839FBF9FB7F894E5E0F1E08081FC
:10C88000806480839FBF6A98729A81E560E00F940C
:10C89000AD235C9A89B182958F7080958170809369
:10C8A000210A0E94A9341092C90708954F925F92FD
:10C8B0006F927F928F929F92AF92BF92CF92DF92B0
:10C8C000EF92FF920F931F93CF93DF933C014B01A5
:10C8D000C42E29018AE0481729F095E1491709F08B
:10C8E000D2C070C09C9AA4989B9AA398809104018E
:10C8F0008460809304019FB7F8948091050184605F
:10C90000809305019FBFA49A0F9438208AE590E098
:10C910000F942E2088EF0E9412300F94382080E070
:10C920000E94123080E80E9412300F94382080E07C
:10C930000E94123080E10E9412300F9438208AE069
:10C9400090E00F942E2080E30E94123080EE0E942F
:10C9500012300F94382000E0802F807780680E948A
:10C960001230802F8295807F0E9412300F943820E1
:10C9700080E80E94123080E00E9412300F9438202C
:10C980008AEF0E9412300F94382010E080E00E945D
:10C99000123080E00E9412300F9438201F5F103256
:10C9A000A9F788EF0E9412300F9438200F5F0032F1
:10C9B00099F680E00E94123080EC0E9412300F94B1
:10C9C000382060C0DB011296ED91FC911397D28064
:10C9D00016810781A49A0F943820812F902F7C0113
:10C9E000A12C12E0B12EAE0CBF1C88EF0E941230B9
:10C9F0000F943820BFE1BD1588F08D2D80778068B9
:10CA00000E9412308D2D8295807F0E9412300F94EB
:10CA1000382080E80E94123080E012C01D2D105294
:10CA2000812F807780680E941230812F8295807FCD
:10CA30000E9412300F94382080E80E94123080E863
:10CA40000E9412300F9438208AEF0E9412300F9407
:10CA50003820E70110E08881807F0E9412308991A0
:10CA60008295807F0E9412301F5F1031A1F780E114
:10CA700090E0E80EF91E0F943820EA14FB0411F040
:10CA8000D394B3CFA498C301B4014C2D92010F9459
:10CA9000B420DF91CF911F910F91FF90EF90DF9025
:10CAA000CF90BF90AF909F908F907F906F905F904E
:10CAB0004F900895FC01128213820895FC01838136
:10CAC000882311F081E082830895FC018281811125
:10CAD00012820895CF93DF93DC01FC01EB55FE4FEA
:10CAE000808191810097C9F1019791838083ED0145
:10CAF000CC5ADF4FFD01ED58FF4F8BE101900992B9
:10CB00008150E1F7FD01EE5AFF4FAF58BF4F8D91B5
:10CB10009C911197A157B04091838083FD01ED58FE
:10CB2000FF4F20E030E0AD014B555E4F10C02F5F4E
:10CB30003F4FEF01DF015F968BE10D90099281502D
:10CB4000E1F7858D968D329791838083B196DA01D6
:10CB50008D919C912817390750F3DF91CF9108955B
:10CB6000FC0189EA95E0918380838781882321F005
:10CB7000CF0104960C946A9B0895CF92DF92EF92B6
:10CB8000FF920F931F93DF93CF93CDB7DEB76F97CD
:10CB90000FB6F894DEBF0FBECDBF8C016B01095AF2
:10CBA0001F4FD8018C9107551040882321F42FE2A4
:10CBB000E22EF12C03C090E5E92EF12CE00EF11EDF
:10CBC00089EA95E09A8389831C821B8218861D82DC
:10CBD000B7016C5F7F4FCE010596A60121E00E9450
:10CBE0005FA2882391F5E3EBFBE2949108C080916A
:10CBF000C00085FFFCCF9093C60031969491992395
:10CC0000B1F7E7E8FDE1949108C08091C00085FF8D
:10CC1000FCCF9093C600319694919923B1F709C047
:10CC20008091C00085FFFCCF0894C11CD11C90935B
:10CC3000C600F6019081992399F78091C00085FF85
:10CC4000FCCF8AE08093C6005AC0F801EB55FE4F36
:10CC5000208131812A30310508F040C02F5F3F4FDD
:10CC60003183208321503040F90185E0EE0FFF1F12
:10CC70008A95E1F7E21BF30BED58FF4FE00FF11F30
:10CC800013C0AF01415E5F4FBF018BE1DB010D902F
:10CC9000BD01DA010D92AD018150C1F792918291EF
:10CCA0003296968F858F7F9721503040BFEF2E3F71
:10CCB0003B0739F7D801AD58BF4FF70134968BE1E8
:10CCC00001900D928150E1F70F581F4FF7018281BB
:10CCD0009381D8018D939C9301571040D801AC5A91
:10CCE000BF4FFE0135968BE101900D928150E1F727
:10CCF0000E5A1F4F8B819C81F80191838083CE0156
:10CD000001962EDF6F960FB6F894DEBF0FBECDBF33
:10CD1000CF91DF911F910F91FF90EF90DF90CF9017
:10CD20000895EF92FF920F931F938C013EECE32E38
:10CD300031E0F32EE80EF91EC7010E941B9BC701CC
:10CD40000E946A9BF801108211821F910F91FF903F
:10CD5000EF900895CF92DF92EF92FF920F931F937F
:10CD6000CF93DF937C016B01DB010D900020E9F78D
:10CD70008D0101501040061B170BEEECF1E0EE0E9A
:10CD8000FF1ED7011C92E2E3FEEFEE0EFF1ECB0169
:10CD90006EE470E00E948528EC01009731F4F80100
:10CDA0003197EC0DFD1D86010EC060E270E00E941F
:10CDB00085288C010F5F1F4FCE016AE270E00E9450
:10CDC0008528FC0131978DE081838AE0828313827C
:10CDD000C70186539E4FB8010F940D1B8EEC91E056
:10CDE000E80EF91ED7018C91882319F1ECEAFBE2D9
:10CDF000949108C08091C00085FFFCCF9093C6003D
:10CE0000319694919923B1F7E1EBFDE1949108C03B
:10CE10008091C00085FFFCCF9093C600319694911D
:10CE20009923B1F78091C00085FFFCCF8AE0809301
:10CE3000C600DF91CF911F910F91FF90EF90DF908F
:10CE4000CF900895CF93DF93EC018B81882309F471
:10CE50003BC0E9EDFDE1949108C08091C00085FFE1
:10CE6000FCCF9093C600319694919923B1F7CD579A
:10CE7000DD4F488159816A817B81C358D24082E568
:10CE80009BE02AE030E00E942F96E7EDFDE19491CF
:10CE900008C08091C00085FFFCCF9093C6003196FA
:10CEA00094919923B1F7C558DD4F488159816A8122
:10CEB0007B8182E59BE02AE030E00E942F96809102
:10CEC000C00085FFFCCF12C0E7ECFDE1949108C0E3
:10CED0008091C00085FFFCCF9093C600319694915D
:10CEE0009923B1F78091C00085FFFCCF8AE0809341
:10CEF000C600DF91CF9108952F923F924F925F929B
:10CF00006F927F928F929F92AF92BF92CF92DF9259
:10CF1000EF92FF920F931F93DF93CF93CDB7DEB7BE
:10CF2000AD970FB6F894DEBF0FBECDBF5C014B01CD
:10CF30004DA7FC018381882309F449C1C5018253AF
:10CF40009E4F0E946A9BF50112821A8A1D8A198AD5
:10CF5000188A89EA95E09F878E875EE4C52ED12CDA
:10CF6000CA0CDB1C2FE230E0A20EB31EF601B18228
:10CF7000A08221ED3FEFA20EB31EF40180818F321B
:10CF800009F090C0C4016FE270E00E9485287C0126
:10CF90000894E11CF11C3E010894611C711C2601DF
:10CFA00042E1242E312C2C0E3D1E77C0C7016FE2CA
:10CFB00070E00E9485286C01009709F481C0E81692
:10CFC000F90608F07DC08C010E191F09C301B701D5
:10CFD000A8010E94AE28060D171DF8011082F3016A
:10CFE00007C08091C00085FFFCCF31969093C600AA
:10CFF00090819923B1F78091C00085FFFCCFFAE0C2
:10D00000F093C600F201608171816115710519F418
:10D0100060E070E002C06C5F7F4FC101A30121E0BE
:10D020000E945FA2882371F5E5E1FEE1949108C0BA
:10D030008091C00085FFFCCF9093C60031969491FB
:10D040009923B1F7FE01319607C08091C00085FF9A
:10D05000FCCF31969093C60090819923B1F7E3E11C
:10D06000FEE1949108C08091C00085FFFCCF9093B1
:10D07000C600319694919923B1F78091C00085FF45
:10D08000FCCF99C02EE030E02C0F3D1FF201318320
:10D09000208376010894E11CF11CE114F10409F0ED
:10D0A00085CF0BC080E590E0A80EB91EF601B182D5
:10D0B000A08220EB3FEFA20EB31ED82C092D02C098
:10D0C000DE2C0F2D8EE490E0A80EB91EF5018081B4
:10D0D000918122EB3FEFA20EB31E009719F480E07E
:10D0E00090E001C004966D2D702F0E942BA3882321
:10D0F00009F468C03DA5332309F060C0E5E0FEE116
:10D10000949108C08091C00085FFFCCF9093C60029
:10D11000319694919923B1F78D2D902F9C01F901AF
:10D1200007C08091C00085FFFCCF31969093C60068
:10D1300090819923B1F78091C00085FFFCCF8AE0F0
:10D140008093C60083E892E0A80EB91EF501108214
:10D1500011821282138232C0EDEEFDE1949108C07B
:10D160008091C00085FFFCCF9093C60031969491CA
:10D170009923B1F78D2D902F9C01F90107C0809163
:10D18000C00085FFFCCF31969093C6009081992313
:10D19000B1F7EBEEFDE1949108C08091C00085FFEE
:10D1A000FCCF9093C600319694919923B1F780916A
:10D1B000C00085FFFCCF8AE08093C600CE010E96AA
:10D1C000CFDC05C0FDA5FF2309F4C6CFF7CFAD9690
:10D1D0000FB6F894DEBF0FBECDBFCF91DF911F9188
:10D1E0000F91FF90EF90DF90CF90BF90AF909F9006
:10D1F0008F907F906F905F904F903F902F90089509
:10D20000BF92CF92DF92EF92FF920F931F93CF9333
:10D21000DF938C01EB018FE28993EE24E394FF24EA
:10D2200075EAC72E71E0D72EC00ED11E6FE1B62E63
:10D2300014C0FB9CC00111248D589F4F800F911F7B
:10D24000BE010E947A9B02C02196E39488818823C4
:10D2500019F08CE88E15C0F7F3942F2D30E0F6010D
:10D26000808191812817390720F3E7FC07C0C801A6
:10D2700082539E4FBE010E947A9B01C01882DF91AB
:10D28000CF911F910F91FF90EF90DF90CF90BF90C3
:10D290000895EF92FF920F931F93CF93DF938C012A
:10D2A000FC01138286A9882321F0C801C3960E943D
:10D2B0006A9BE7EAEE2EE1E0FE2EE00EF11EC701CA
:10D2C00060E045E30E941799882309F5E3EBFBE250
:10D2D000949108C08091C00085FFFCCF9093C60058
:10D2E000319694919923B1F7EEE5FFE1949108C04E
:10D2F0008091C00085FFFCCF9093C6003196949139
:10D300009923B1F78091C00085FFFCCF7DC0E80173
:10D31000C455DE4FCE01B70141E00E94E02B8823C7
:10D3200041F5CE01B70140E00E94E02B882309F5CA
:10D33000ECEAFBE2949108C08091C00085FFFCCF2D
:10D340009093C600319694919923B1F7EBE4FFE1F5
:10D35000949108C08091C00085FFFCCF9093C600D7
:10D36000319694919923B1F78091C00085FFFCCF4D
:10D370004BC0C801C396BE010E945E9E882309F57A
:10D38000ECEAFBE2949108C08091C00085FFFCCFDD
:10D390009093C600319694919923B1F7EBE3FFE1A6
:10D3A000949108C08091C00085FFFCCF9093C60087
:10D3B000319694919923B1F78091C00085FFFCCFFD
:10D3C00023C081E0F8018383E3EBFBE2949108C082
:10D3D0008091C00085FFFCCF9093C6003196949158
:10D3E0009923B1F7E0E3FFE1949108C08091C00078
:10D3F00085FFFCCF9093C600319694919923B1F7A5
:10D400008091C00085FFFCCF8AE08093C600D801E0
:10D41000AC5ABF4FF801F3968BE101900D92815009
:10D42000E1F7F80181A992A90E5A1F4FF8019183E3
:10D43000808302551040C8018F96025B1F4FF80190
:10D4400091838083DF91CF911F910F91FF90EF9097
:10D4500008952F923F924F925F926F927F929F9288
:10D46000AF92BF92CF92DF92EF92FF920F931F93F2
:10D47000DF93CF93CDB7DEB7CC55D0400FB6F8943D
:10D48000DEBF0FBECDBF6C01662311F527E832E089
:10D49000C20ED31ED6018C91E9E7FDEFCE0EDF1E42
:10D4A000882309F4E3C02FE732E0C20ED31ED60171
:10D4B000ED90FD900D911C91E1E8FDEFCE0EDF1E89
:10D4C0000F94E725E616F7060807190708F4CEC0FB
:10D4D00027E832E0C20ED31ED6011C92E9E7FDEF29
:10D4E000CE0EDF1ED60113968C91882339F4C60127
:10D4F000D0DEF6018381882309F4B8C000D000D0C3
:10D50000EDB7FEB731967E010894E11CF11CADB772
:10D51000BEB71296FC92EE92119788EA9DE1938332
:10D520008283D6019D968D919C919E97958384834D
:10D530000E94D7288701EDB7FEB736960FB6F8944C
:10D54000FEBF0FBEEDBF57010AC0D8018C919927CD
:10D5500087FD90950F94C02FF80181938F01F501FD
:10D5600001900020E9F73197EA19FB09802F8E1905
:10D570008E175CF313E3A12EB12CAC0CBD1CC501BE
:10D5800040E050E060E070E00E94519A9924BDE3D1
:10D59000EB2EF12CEC0EFD1E2E010894411C511CAB
:10D5A000AFE16A2E712C6C0E7D1EF1EA2F2EFDE18B
:10D5B0003F2E42C0D8018C9190E00F94C02FF8010B
:10D5C00081938F01D7010D900020E9F71197AE19D3
:10D5D000BF09802F8E198A176CF327968FAD279776
:10D5E0008E3751F1C701B20145E050E00E94A028FA
:10D5F000009711F500D000D0EDB7FEB73196ADB76A
:10D60000BEB712967C926E92119733822282558217
:10D6100044820E94D728EDB7FEB736960FB6F8942D
:10D62000FEBF0FBEEDBFC3010F9491098DE99DE1CF
:10D630000F94180999249394C501B70140E050E074
:10D640000E947D9D181614F48701BCCF992041F4E7
:10D650008FEF9FEFD6019E969C938E939D9706C069
:10D66000F60185A596A5019696A785A7C45ADF4F12
:10D670000FB6F894DEBF0FBECDBFCF91DF911F91E3
:10D680000F91FF90EF90DF90CF90BF90AF909F9061
:10D690007F906F905F904F903F902F9008952F92C2
:10D6A0003F924F925F926F927F928F929F92AF9232
:10D6B000BF92CF92DF92EF92FF920F931F93DF936F
:10D6C000CF93CDB7DEB7CF58D0400FB6F894DEBFBA
:10D6D0000FBECDBF8C012B016A01C757DF4F3983C5
:10D6E0002883C958D04084E090E0C80ED91EF801C4
:10D6F0007196C957DF4FF983E883C758D04044E09B
:10D70000642E712C600E711ECA57DF4F1882C658E6
:10D71000D04036E6E32EF12CEC0EFD1EC7010B9631
:10D72000C557DF4F99838883CB58D04028E8822E95
:10D7300022E0922E800E911E9AE8A92E92E0B92E38
:10D74000A00EB11E87E4282E312C2C0E3D1EF101B7
:10D750003496C357DF4FF983E883CD58D040E3EBCD
:10D76000FBE28491C157DF4F8883CF58D04053C12B
:10D77000F7018385482F50E0BA01687170706031FD
:10D78000710509F056C1F401208131812130310544
:10D7900009F44FC12230310509F44BC1F701DE0114
:10D7A00011969081903239F08E2F8E19883011F4B5
:10D7B0008EE28D939D933196C557DF4F8881998175
:10D7C000CB58D040E817F90761F71C921E86F2018A
:10D7D0008081882331F4CE010E966DE372E00E94C1
:10D7E0007A28CE010E96B2010E947A28CE010E96BA
:10D7F000BE016F5F7F4F0E947A28CE010E966DE3C7
:10D8000072E00E947A281CA61FA61BA61AA689EA07
:10D8100095E099A788A7CE018C96B601AE014F5F1F
:10D820005F4F21E00E945FA2882309F03FC0F4010E
:10D8300080819181892BD1F5C157DF4F9881CF58D5
:10D84000D040E3EBFBE208C08091C00085FFFCCF35
:10D850009093C600319694919923B1F7EFE3F2E0EB
:10D8600007C08091C00085FFFCCF31969093C60021
:10D8700090819923B1F78091C00085FFFCCFFAE039
:10D88000F093C600FE01319607C08091C00085FF6D
:10D89000FCCF31969093C60090819923B1F7809187
:10D8A000C00085FFFCCF8AE08093C600C357DF4FDE
:10D8B000A881B981CD58D040FE01BC968BE1019082
:10D8C0000D928150E1F78AA59BA5F1019383828394
:10D8D00089EA95E091838083C801BE01625F7F4F32
:10D8E000A10120E030E0DBDEC1013AD9CE0188960B
:10D8F00037D991C09E3209F48EC09F3509F48BC090
:10D90000F80191899E3209F486C09F3509F483C0DD
:10D9100043FD81C080E06031710509F481E0F801C8
:10D9200084A7882349F4F7018085873409F073C000
:10D9300081858E3709F46FC0D301F7018081803271
:10D9400041F08E2F8E19883011F48EE28D938081F4
:10D950008D933196C557DF4F88819981CB58D04040
:10D96000E817F90759F71C92F4018081918100971B
:10D9700001F5F20107C08091C00085FFFCCF319610
:10D980009093C60090819923B1F7F30107C080916D
:10D99000C00085FFFCCF31969093C60090819923FB
:10D9A000B1F78091C00085FFFCCFFAE0F093C6008C
:10D9B00032C08130910539F4F50180819181019661
:10D9C0009183808328C0029731F5C757DF4F888144
:10D9D0009981C958D040009731F0B3010E9467285F
:10D9E000892B71F42BC0CA57DF4F9881C658D0409D
:10D9F000292F30E0F5018081918128173907F1F056
:10DA0000CA57DF4FF881C658D040FF5FCA57DF4F73
:10DA1000F883C658D040C601B701C957DF4F4881C7
:10DA20005981C758D0400E947D9D18160CF4A0CE95
:10DA300005C0F7019081992309F05CCFC157DF4FF2
:10DA40000FB6F894DEBF0FBECDBFCF91DF911F910F
:10DA50000F91FF90EF90DF90CF90BF90AF909F908D
:10DA60008F907F906F905F904F903F902F90089590
:10DA7000EF92FF920F931F93DF93CF93CDB7DEB753
:10DA80006F970FB6F894DEBF0FBECDBF7C018C013F
:10DA9000025B1F4F805B9F4FF8019183808328E8D2
:10DAA00032E0E20EF31E21E030E0F70121933193E2
:10DAB0007F011182108226E73DEFE20EF31E0496ED
:10DAC00040E050E060E070E00E94519AF80120814F
:10DAD0003181DE011596F90134968BE101900D92AA
:10DAE0008150E1F7F901828193819C838B8389EADC
:10DAF00095E09A838983C70162E572E08E010F5F2A
:10DB00001F4FA80120E030E0CADDC80129D8F70185
:10DB1000E657FD4F808191816F960FB6F894DEBF76
:10DB20000FBECDBFCF91DF911F910F91FF90EF906E
:10DB30000895CF92DF92EF92FF920F931F93DF939E
:10DB4000CF93CDB7DEB76F970FB6F894DEBF0FBE99
:10DB5000CDBF7C016A018C01025B1F4F805B9F4F30
:10DB6000F8019183808328E832E0E20EF31E22E080
:10DB700030E0F701219331937F017183608326E7C1
:10DB80003DEFE20EF31E049640E050E060E070E0EE
:10DB90000E94519AF80120813181DE011596F90128
:10DBA00034968BE101900D928150E1F7F901828169
:10DBB00093819C838B8389EA95E09A838983C7014B
:10DBC00062E572E08E010F5F1F4FA801960167DDCD
:10DBD000C8010E94B0656F960FB6F894DEBF0FBE05
:10DBE000CDBFCF91DF911F910F91FF90EF90DF900C
:10DBF000CF9008952F923F924F925F926F927F92B3
:10DC00008F929F92AF92BF92CF92DF92EF92FF924C
:10DC10000F931F93DF93CF93CDB7DEB7AE970FB6B9
:10DC2000F894DEBF0FBECDBF7C013B014DA70EA710
:10DC3000DC0113968C91882309F45DC3E1EDF1E0DA
:10DC4000EE0EFF1ED7018C91EFE2FEEFEE0EFF1EEF
:10DC5000882309F418C1222309F0E0C029EE31E03D
:10DC6000E20EF31ED7018C91E7E1FEEFEE0EFF1EF0
:10DC7000882371F1ECEAFBE2949108C08091C00026
:10DC800085FFFCCF9093C600319694919923B1F70C
:10DC9000EDEEFEE1949108C08091C00085FFFCCFBD
:10DCA0009093C600319694919923B1F782E59BE059
:10DCB00061E070E04AE050E00E948E968091C000E2
:10DCC00085FFFCCF8AE08093C6000E947CCA13C304
:10DCD000E3EBFBE2949108C08091C00085FFFCCF8C
:10DCE0009093C600319694919923B1F7E4EDFEE14B
:10DCF000949108C08091C00085FFFCCF9093C6002E
:10DD0000319694919923B1F7F30107C08091C00037
:10DD100085FFFCCF31969093C60090819923B1F78F
:10DD2000E9ECFEE1949108C08091C00085FFFCCF32
:10DD30009093C600319694919923B1F7C7012EEEC6
:10DD400031E0E20EF31EB7015BDA4BEF5FEFE40E5A
:10DD5000F51ED7019C91E7E1FEEFEE0EFF1E8DE868
:10DD6000989FF0011124E251FE4FEE0DFF1D07C0F8
:10DD70008091C00085FFFCCF31969093C6009081C2
:10DD80009923B1F7E3ECFEE1949108C08091C000C3
:10DD900085FFFCCF9093C600319694919923B1F7FB
:10DDA00023E832E0E20EF31ED7014D915D916D91B3
:10DDB0007C91EDE7FDEFEE0EFF1E82E59BE02AE091
:10DDC00030E00E942F968091C00085FFFCCF8AE052
:10DDD0008093C600A70147515E4FDA012C91E22FD4
:10DDE000F0E0EE0FFF1FEE0FFF1FEE0DFF1DE651DF
:10DDF000FE4F83E892E0E80EF91ED701AD90BD908A
:10DE0000CD90DC908DE79DEFE80EF91EA082B182E7
:10DE1000C282D3822F5FDA012C932FC0E3EBFBE2A7
:10DE2000949108C08091C00085FFFCCF9093C600FC
:10DE3000319694919923B1F7E2EBFEE1949108C0F9
:10DE40008091C00085FFFCCF9093C60031969491DD
:10DE50009923B1F7F30107C08091C00085FFFCCF83
:10DE600031969093C60090819923B1F78091C000BC
:10DE700085FFFCCF8AE08093C600C70182539E4F86
:10DE80000E946A9B3CC0E9EEF1E0EE0EFF1ED70156
:10DE90001C92E7E1FEEFEE0EFF1EFEA5FF2379F5D3
:10DEA000E3EBFBE2949108C08091C00085FFFCCFBA
:10DEB0009093C600319694919923B1F7E1EAFEE17F
:10DEC000949108C08091C00085FFFCCF9093C6005C
:10DED000319694919923B1F7F30107C08091C00066
:10DEE00085FFFCCF31969093C60090819923B1F7BE
:10DEF0008091C00085FFFCCF8AE08093C600D701E7
:10DF000012961C921A8A1D8A198A188A89EA95E043
:10DF10009F878E876EE4A62EB12CAE0CBF1CEFE25D
:10DF2000F0E0EE0EFF1ED501ED92FC92E1EDFFEF69
:10DF3000EE0EFF1ED3018C918F3209F090C0C30109
:10DF40006FE270E00E9485286C010894C11CD11C0E
:10DF50004E010894811C911C250152E1252E312C83
:10DF60002C0E3D1E77C0C6016FE270E00E9485282E
:10DF70005C01009709F480C0C816D90608F07CC07F
:10DF80008C010C191D09C401B601A8010E94AE281C
:10DF9000080D191DF8011082F40107C08091C0001E
:10DFA00085FFFCCF31969093C60090819923B1F7FD
:10DFB0008091C00085FFFCCFFAE0F093C600D2014B
:10DFC0006D917C916115710519F460E070E002C0FB
:10DFD0006C5F7F4FC101A40121E00E945FA28823F2
:10DFE00071F5EDE8FEE1949108C08091C00085FFD5
:10DFF000FCCF9093C600319694919923B1F7FE011E
:10E00000319607C08091C00085FFFCCF3196909378
:10E01000C60090819923B1F7EBE8FEE1949108C026
:10E020008091C00085FFFCCF9093C60031969491FB
:10E030009923B1F78091C00085FFFCCF2AC12EE063
:10E0400030E02C0F3D1FF2013183208365010894DD
:10E05000C11CD11CC114D10409F085CF0BC040E50F
:10E0600050E0E40EF51ED501ED92FC92E0EBFFEFDF
:10E07000EE0EFF1E830101C08601F701E25BFF4F38
:10E080002DA5222309F4C6C0608171816115710537
:10E0900019F460E070E002C06C5F7F4FC7018253EB
:10E0A0009E4FA80121E00E945FA2882309F485C049
:10E0B0004FED51E0E40EF51ED7014D915D916D914C
:10E0C0007C91ECE9F0E0EE0EFF1ED7014D935D93DD
:10E0D0006D937C931397E5E8FDEFEE0EFF1EFEA512
:10E0E000FF2309F035C0EDE7FEE1949108C080916F
:10E0F000C00085FFFCCF9093C60031969491992380
:10E10000B1F7F80107C08091C00085FFFCCF3196C0
:10E110009093C60090819923B1F7E5E7FEE19491D1
:10E1200008C08091C00085FFFCCF9093C600319657
:10E1300094919923B1F782E59BE02AE030E00E94B8
:10E140002F968091C00085FFFCCF8AE08093C600A7
:10E1500023E832E0E20EF31ED7011D921D921D92BC
:10E160001C921397EDE7FDEFEE0EFF1EFEA5FF23B9
:10E17000A9F4E7E6FEE1949108C08091C00085FF14
:10E18000FCCF9093C600319694919923B1F780917A
:10E19000C00085FFFCCF8AE08093C600C70160E025
:10E1A00070E0A801C6DCD70151968C91882309F450
:10E1B0009BC087010F5E1F4F97C0E3E5FEE194917E
:10E1C00008C08091C00085FFFCCF9093C6003196B7
:10E1D00094919923B1F7F80107C08091C00085FFA1
:10E1E000FCCF31969093C60090819923B1F7E1E579
:10E1F000FEE1949108C08091C00085FFFCCF909310
:10E20000C600319694919923B1F78091C00085FFA3
:10E21000FCCF3FC0608171816115710519F460E028
:10E2200070E002C06C5F7F4FC70182539E4FA80110
:10E2300026E50E945FA2882381F5EDE3FEE194913B
:10E2400008C08091C00085FFFCCF9093C600319636
:10E2500094919923B1F7F80107C08091C00085FF20
:10E26000FCCF31969093C60090819923B1F7EBE3F0
:10E27000FEE1949108C08091C00085FFFCCF90938F
:10E28000C600319694919923B1F78091C00085FF23
:10E29000FCCF8AE08093C6002AC081E0F70180832A
:10E2A000FEA5FF2309F5E9E2FEE1949108C0809103
:10E2B000C00085FFFCCF9093C600319694919923BE
:10E2C000B1F7F30107C08091C00085FFFCCF319604
:10E2D0009093C60090819923B1F78091C00085FF8B
:10E2E000FCCF8AE08093C600C8010E94CD62CE01B7
:10E2F0000E960E94B065AE960FB6F894DEBF0FBEC4
:10E30000CDBFCF91DF911F910F91FF90EF90DF90E4
:10E31000CF90BF90AF909F908F907F906F905F90C5
:10E320004F903F902F900895CF92DF92EF92FF92FF
:10E330000F93CF93DF93EC010E9432BE09EEE02EE3
:10E3400001E0F02EEC0EFD1ED7018C91BEECCB2E21
:10E35000B1E0DB2ECC0EDD1E8823A1F1C6010E94A8
:10E360006A9BF7016081615060838DE8689FB0010E
:10E37000112462517E4F6C0F7D1FCE0141E021E0E0
:10E3800000E038DCD701EC91F0E0EE0FFF1FEE0F5C
:10E39000FF1FEC0FFD1FE651FE4F4081518162814E
:10E3A0007381CD57DD4F488359836A837B83C3587C
:10E3B000D240C6010E94519A8B81882349F081E0A6
:10E3C0008A8306C00E947BBBC6010E946A9B1A8298
:10E3D000DF91CF910F91FF90EF90DF90CF90089554
:10E3E0000F93FC0181E08183CF0140E021E000E058
:10E3F00001DC0F910895EF92FF920F931F93DF932B
:10E40000CF93CDB7DEB76F970FB6F894DEBF0FBED0
:10E41000CDBF7C0188E892E0E80EF91EF701118279
:10E42000108288E79DEFE80EF91E87010D5C1F4FF3
:10E43000C80140E050E060E070E00E94519ADE01C7
:10E440001596F8018BE101900D928150E1F7F701EB
:10E4500081A992A99C838B8389EA95E09A83898319
:10E46000C70162E572E08E010F5F1F4FA80120E037
:10E4700030E015D9C8010E94B0656F960FB6F894C8
:10E48000DEBF0FBECDBFCF91DF911F910F91FF90E7
:10E49000EF9008950F931F93CF93DF93DC01D396F2
:10E4A0001C92D397D6961C92D697D2961C921E9207
:10E4B000D19789EA95E0D0969C938E939F97AC5A1A
:10E4C000BF4F1C9213961C92A755B040FD01E05B14
:10E4D000FF4FAE5ABF4F11961C921E92A255B040EC
:10E4E00091838083ED01C159DF4FFE0120E030E0D0
:10E4F000482F148217821382128240839183215EF7
:10E500003F4F7F9681E02633380799F7A855BE4FD5
:10E5100089E18C9313961C9258961C921B961C9220
:10E5200013961C92A15DB140FD01E653FE4FA4532A
:10E53000BE4F11961C921E9240839183A155BF4FEE
:10E540001D921D921D921C92139718961D921D925A
:10E550001D921C921397A358B24012961C921297C8
:10E5600013961C9213971C9211961C9211978D0171
:10E5700001581D4FF8011082118212821382AB558F
:10E58000BE4F11961C921E92AC5BBF4F1C92FE01B7
:10E59000C90111920197E9F7A256BF4F81E08C9310
:10E5A000A758B2409E961C921E929D970F94E72505
:10E5B00068577C4E8F4F9F4FF80160837183828331
:10E5C0009383DF91CF911F910F91089560E070E0E8
:10E5D0008FE793E420916B0430916C0440916D04BB
:10E5E00050916E040F94842B6093930A7093940A55
:10E5F0008093950A9093960A0895FC0197FF03C0B3
:10E600008091640A03C0EF58F54F808190E008952F
:10E610002F923F924F925F926F927F928F929F9232
:10E62000AF92BF92CF92DF92EF92FF920F931F9320
:10E63000CF93DF93EC0121E030E0A901440F551F97
:10E64000440F551FFA01EC5FFE4D85919491C81758
:10E65000D9070CF059C0B90161507040660F771F9F
:10E66000660F771FCB018A5F9E4DFC0105911491C7
:10E670006C5F7E4DFB01C590D490FA01EA5FFE4DC0
:10E68000E590F490FA01EC5FFE4DA590B490B801CE
:10E69000882777FD8095982F0F941F2C1B012C0144
:10E6A000CC19DD09BE01882777FD8095982F0F943E
:10E6B0001F2C3B014C01E01AF10A0027F7FC0095E2
:10E6C000102FC801B7010F941F2C9B01AC01C4018E
:10E6D000B3010F945D2E7B018C01AC18BD08CC24D6
:10E6E000B7FCC094DC2CC601B5010F941F2C9B0114
:10E6F000AC01C801B7010F94842B9B01AC01C2018E
:10E70000B1010F94A42A19C0822F8F5F2F5F3F4F52
:10E710002A33310509F091CF8A3329F0E0E070E027
:10E7200080E060E00CC0EAEEF1E265917491882728
:10E7300077FD8095982F0F941F2CE62F692F2E2F91
:10E74000372F482F562FB901CA01DF91CF911F9162
:10E750000F91FF90EF90DF90CF90BF90AF909F9080
:10E760008F907F906F905F904F903F902F90089583
:10E770001092550A1092540A1092710A9FB7F89499
:10E78000E2E0F1E080818F7B80839FBF1092570A87
:10E790001092560A1092640A759808952CEA35EC86
:10E7A00047E25EE30D945D2E2CEA35EC47E25EE332
:10E7B0000D94842B2CEA35EC47E25EE30D94842B18
:10E7C0002CEA35EC47E25EE30D945D2E75980E94CD
:10E7D00023C9882339F5ECEAFBE2949108C08091C3
:10E7E000C00085FFFCCF9093C60031969491992389
:10E7F000B1F7ECE7FFE1949108C08091C00085FF7C
:10E80000FCCF9093C600319694919923B1F78091F3
:10E81000C00085FFFCCF8AE08093C6008BE69FE1B5
:10E820000E94C7620C943ACA1F93182FA1DF0E945E
:10E8300023C9882309F036C0ECEAFBE2949108C0B2
:10E840008091C00085FFFCCF9093C60031969491D3
:10E850009923B1F782E59BE0612F70E04AE050E038
:10E860000E948E968091C00085FFFCCF8AE0809345
:10E87000C600E3ECFFE1949108C08091C00085FFE1
:10E88000FCCF9093C600319694919923B1F7809173
:10E89000C00085FFFCCF8AE08093C60086EB9FE135
:10E8A0000E94C7620E943ACA1F9108951F93182FB1
:10E8B0005FDF0E9423C9882309F036C0ECEAFBE23F
:10E8C000949108C08091C00085FFFCCF9093C60052
:10E8D000319694919923B1F782E59BE0612F70E026
:10E8E0004AE050E00E948E968091C00085FFFCCFE8
:10E8F0008AE08093C600EDEFFFE1949108C080911B
:10E90000C00085FFFCCF9093C60031969491992367
:10E91000B1F78091C00085FFFCCF8AE08093C600EC
:10E9200080EF9FE10E94C7620E943ACA1F9108953A
:10E930001F920F920FB60F920BB60F921124FF92F7
:10E940000F931F932F933F934F935F936F937F93F7
:10E950008F939F93AF93BF93CF93DF93EF93FF93E7
:10E9600020917A042223E9F48091710A8093780A35
:10E97000882331F09FB7F89480910201806405C02C
:10E980009FB7F894809102018F7B809302019FBF13
:10E990008091640A8093770A882311F0759A01C0E8
:10E9A00075988091780A821740F49FB7F894809107
:10E9B00002018F7B809302019FBF8091770A8217AB
:10E9C00008F475982F5F2F7720937A0480917B0449
:10E9D000853009F48BC0863090F4823009F44EC043
:10E9E000833030F48823F1F0813009F0AFC028C0C3
:10E9F000833009F451C0843009F0A8C069C0883060
:10EA000009F496C0893038F4863009F48BC0873019
:10EA100009F09CC08BC0893009F48EC08A3009F09F
:10EA200095C092C010927B0080E480937C0080911E
:10EA30007A00806480937A000E94A93481E01BC030
:10EA40008091780090917900A0E0B0E02091850A53
:10EA50003091860A4091870A5091880A280F391F01
:10EA60004A1F5B1F2093850A3093860A4093870ACA
:10EA70005093880A82E080937B0468C010927B00E8
:10EA800082E480937C0080917A00806480937A0095
:10EA90000E94A93483E0EFCF8091780090917900B3
:10EAA000A0E0B0E02091790A30917A0A40917B0A87
:10EAB00050917C0A280F391F4A1F5B1F2093790A47
:10EAC00030937A0A40937B0A50937C0A84E0D3CF38
:10EAD00010927B0081E480937C0080917A008064B6
:10EAE00080937A000E94A93485E0C5CF8091780098
:10EAF00090917900A0E0B0E02091810A3091820AE3
:10EB00004091830A5091840A280F391F4A1F5B1FC6
:10EB10002093810A3093820A4093830A5093840A97
:10EB200086E0A9CF0E94A93487E0A5CF88E0A3CFD3
:10EB30000E94A93489E09FCF10927B048091890ABA
:10EB40008F5F8093890A02C010927B048091890AAA
:10EB5000803108F463C08091720A882381F4809127
:10EB6000850A9091860A9093590A8093580A809159
:10EB7000790A90917A0A90935F0A80935E0A81E005
:10EB80008093720A1092890A1092850A1092860A5E
:10EB90001092870A1092880A1092810A1092820AB3
:10EBA0001092830A1092840A10927D0A10927E0AB3
:10EBB00010927F0A1092800A1092790A10927A0AB3
:10EBC00010927B0A10927C0A2091580A3091590ABF
:10EBD0008091730A9091740A8217930714F080E071
:10EBE00065DE2091580A3091590A809178049091FD
:10EBF00079042817390714F080E016DE20915E0AA8
:10EC000030915F0A8091750A9091760A8217930776
:10EC10002CF01092570A1092560AD8DD00E010E04E
:10EC2000FF24F394E801CC0FDD1FCB59D54F888129
:10EC300099811816190654F4F0927704802F61E038
:10EC40000E94A3BB8881998101970BC0892B59F041
:10EC500010927704802F60E00E94A3BB8881998185
:10EC60000196998388830F5F1F4F03301105D1F6FA
:10EC7000FF91EF91DF91CF91BF91AF919F918F91D4
:10EC80007F916F915F914F913F912F911F910F91C4
:10EC9000FF900F900BBE0F900FBE0F901F90189516
:10ECA000EF92FF920F931F93E0905A0AF0905B0A45
:10ECB00000915C0A10915D0A6091540A7091550AA6
:10ECC000882777FD8095982F0F941F2C20E030E047
:10ECD00040EA51E40F94A32A9B01AC01C801B7019B
:10ECE0000F947D2B882394F4C801B7010F94EC2B6B
:10ECF00070936C0A60936B0A0F94E72560936D0A1A
:10ED000070936E0A80936F0A9093700A1F910F910F
:10ED1000FF90EF9008952F923F924F925F926F92E3
:10ED20007F928F929F92AF92BF92CF92DF92EF929B
:10ED3000FF920F931F93DF93CF930F92CDB7DEB760
:10ED40004C01662389F1ECEAFBE2949108C08091C2
:10ED5000C00085FFFCCF9093C60031969491992313
:10ED6000B1F782E59BE070E04AE050E00E948E96A9
:10ED7000E7E6F0E2949108C08091C00085FFFCCFE7
:10ED80009093C600319694919923B1F78091C00079
:10ED900085FFFCCF8AE08093C6000E947CCAE0E039
:10EDA00070E080E060E08AC021E030E06FC0A9013F
:10EDB000F901EE0FFF1FEE0FFF1FEC57FF4D85917E
:10EDC00094912F5F3F4F881699060CF05FC09A010F
:10EDD00021503040220F331F220F331FC9018A57A1
:10EDE0009F4DFC01059114912C573F4DF901C590A1
:10EDF000D490440F551F440F551FFA01EA57FF4D99
:10EE0000E590F490FA01EC57FF4DA590B490B8014D
:10EE1000882777FD8095982F0F941F2C1B012C01BC
:10EE20008C189D08B401882777FD8095982F0F9442
:10EE30001F2C3B014C01E01AF10A0027F7FC00955A
:10EE4000102FC801B7010F941F2C9B01AC01C40106
:10EE5000B3010F945D2E7B018C01AC18BD08CC244E
:10EE6000B7FCC094DC2CC601B5010F941F2C9B018C
:10EE7000AC01C801B7010F94842B9B01AC01C20106
:10EE8000B1010F94A42AE62F692F09C029832032EB
:10EE9000310509F08CCFE0E070E080E060E0F981BE
:10EEA000F03261F4E2E0F1E265917491882777FD38
:10EEB0008095982F0F941F2CE62F692F2E2F372F18
:10EEC000482F562FB901CA010F90CF91DF911F91A2
:10EED0000F91FF90EF90DF90CF90BF90AF909F90F9
:10EEE0008F907F906F905F904F903F902F900895FC
:10EEF0000F931F93CF93DF9380E090E0A0E0B0E00A
:10EF000080938F0A9093900AA093910AB093920AEB
:10EF100060E070E08FE793E420916B0430916C0423
:10EF200040916D0450916E040F94842B6093930A6A
:10EF30007093940A8093950A9093960A80910101A8
:10EF400080648093010180910101806180930101BF
:10EF50006D9A8091010180628093010188E061E0F7
:10EF600070E00E9426C987ED80937A0010927E009F
:10EF700010927D0080917E00816080937E00809160
:10EF80007E00826080937E0080917E00846080930A
:10EF90007E0080E888BD80916E00846080936E0062
:10EFA0006AEF70E080E090E00F94F52585E090E056
:10EFB0009093980A8093970A09C080917804909161
:10EFC0007904409790937904809378048091780431
:10EFD0009091790460E09FDE20E030E040EA50E468
:10EFE0000F947D2B87FDE9CF81E391E090937D0421
:10EFF00080937C0409C08091730A9091740A4096B2
:10F000009093740A8093730A8091730A9091740AA2
:10F0100060E081DE20E030E848E953E40F948B2D76
:10F0200018164CF3C091750AD091760A1C2F0D2F3B
:10F03000CE01EEDA609620E030E046E153E40F9432
:10F040008B2D18169CF31093750A0093760ADF91A6
:10F05000CF911F910F9108958091580A9091590A6C
:10F0600060E059DE60935A0A70935B0A80935C0AF1
:10F0700090935D0A80915E0A90915F0AC9DA60936D
:10F08000600A7093610A8093620A9093630A8FB753
:10F09000F8941092720A8FBF08952F923F924F9268
:10F0A0005F926F927F928F929F92AF92BF92CF9218
:10F0B000DF92EF92FF920F931F93DF93CF93CDB721
:10F0C000DEB728970FB6F894DEBF0FBECDBF809194
:10F0D000720A882309F4A6C2BFDFA0905A0AB09032
:10F0E0005B0AC0905C0AD0905D0A6091540A7091EE
:10F0F000550A882777FD8095982F0F941F2C7B0148
:10F100008C0189E99AE06FE97AE0A6019501CC24A7
:10F11000DD24FFE0AF2EB12CEEE18E2E912C9BD2A0
:10F1200080915A0A90915B0AA0915C0AB0915D0AA5
:10F1300089839A83AB83BC830091540A1091550A4A
:10F14000B801882777FD8095982F0F941F2C29816F
:10F150003A814B815C810F94A32A1B012C0160939F
:10F16000AB0A7093AC0A8093AD0A9093AE0A20E08C
:10F1700030E040E251E40F948B2D181624F481E026
:10F180008093AF0AF2C0C201B10120E030E040E25A
:10F1900051EC0F947D2B87FD02C0012B21F481E0FF
:10F1A0008093AF0A0FC18091AF0A882371F080E08D
:10F1B00090E0A0E0B0E08093B00A9093B10AA093F1
:10F1C000B20AB093B30A1092AF0AC201B101209102
:10F1D0006704309168044091690450916A040F9467
:10F1E0005D2E6D837E838F8398876093B40A7093BE
:10F1F000B50A8093B60A9093B70AC201B101209173
:10F20000B00A3091B10A4091B20A5091B30A0F94FA
:10F21000A42A7B018C0160908F0A7090900A8090E4
:10F22000910A9090920AA40193010F947D2B87FD7F
:10F2300012C06090930A7090940A8090950A909002
:10F24000960AC801B701A40193010F948B2D1816DB
:10F2500014F0370148016092B00A7092B10A8092AE
:10F26000B20A9092B30AC401B30120916B043091A9
:10F270006C0440916D0450916E040F945D2E5B01FF
:10F280006C016093B80A7093B90A8093BA0A90939C
:10F29000BB0A69817A818B819C812091BC0A309163
:10F2A000BD0A4091BE0A5091BF0A0F94A32A209133
:10F2B0006F043091700440917104509172040F9466
:10F2C0005D2E20ED3CEC4CE45DE30F945D2E7B0164
:10F2D0008C016091C00A7091C10A8091C20A90911C
:10F2E000C30A23E333E343E75FE30F945D2E9B01FF
:10F2F000AC01C801B7010F94A42A7B018C01609373
:10F30000C00A7093C10A8093C20A9093C30A6D81A8
:10F310007E818F819885A60195010F94A42AA8016A
:10F3200097010F94A32A7B018C0120E030E04FE786
:10F3300053E40F948B2D18161CF5C201B10120E087
:10F3400030E040E050E00F948B2D181674F4C401A7
:10F35000B301A20191010F94A32A6093B00A7093A4
:10F36000B10A8093B20A9093B30A0F2EF0E0EF2E09
:10F37000F0E0FF2EFFE70F2FF3E41F2FF02D2CC03E
:10F38000C801B70120E030E040E050E00F947D2B51
:10F39000882314F5C201B10120E030E040E050E0E4
:10F3A0000F947D2B87FF0EC0C401B301A201910110
:10F3B0000F94A32A6093B00A7093B10A8093B20AA3
:10F3C0009093B30A0F2EF0E0EF2EF0E0FF2EF0E066
:10F3D0000F2FF0E01F2FF02D89819A81AB81BC8126
:10F3E0008093BC0A9093BD0AA093BE0AB093BF0A53
:10F3F0006091970A7091980A882777FD8095982FD9
:10F400000F941F2C9B01AC0169817A818B819C81B7
:10F410000F948B2D1816ECF460917C0470917D0490
:10F42000882777FD8095982F0F941F2C9B01AC01A6
:10F4300069817A818B819C810F947D2B88234CF488
:10F44000C801B7010F94EC2B759567956093710A0D
:10F4500002C01092710A80916D0A90916E0AA0917B
:10F460006F0AB091700A0097A105B10509F460C058
:10F470000F94E72520916D0A30916E0A40916F0A32
:10F480005091700A621B730B840B950B61547C497D
:10F490008040904008F44CC060916B0A70916C0AF7
:10F4A000665F7F4F882777FD8095982F0F941F2CDC
:10F4B0009B01AC0160915A0A70915B0A80915C0AD1
:10F4C00090915D0A0F947D2B882354F51092550A74
:10F4D0001092540A8CEE91E20E944E5FE3EBFBE245
:10F4E000949108C08091C00085FFFCCF9093C60026
:10F4F000319694919923B1F7E3E5F2E007C080914A
:10F50000C00085FFFCCF31969093C600908199236F
:10F51000B1F78091C00085FFFCCF8AE08093C600E0
:10F5200010926D0A10926E0A10926F0A1092700A71
:10F530000F94E7252091C40A3091C50A4091C60A6C
:10F540005091C70A621B730B840B950B685873416B
:10F550008040904008F466C00F94E7256093C40A89
:10F560007093C50A8093C60A9093C70AA090600A58
:10F57000B090610AC090620AD090630A6091560A06
:10F580007091570A882777FD8095982F0F941F2C2C
:10F590007B018C0188EC9AE06AEC7AE0A601950187
:10F5A000A1E0CA2ED12CFFE0AF2EB12CEAE08E2EC6
:10F5B000912C51D0E090600AF090610A0091620AAB
:10F5C0001091630AC801B70120E030E040EA50E43E
:10F5D0000F948B2D18161CF5C801B70120E030E000
:10F5E00046E153E40F947D2B8823CCF46091560AB6
:10F5F0007091570A882777FD8095982F0F941F2CBC
:10F600009B01AC01C801B7010F948B2D88231CF01E
:10F610001092640A07C087E68093640A03C01092C0
:10F62000640A759828960FB6F894DEBF0FBECDBF5A
:10F63000CF91DF911F910F91FF90EF90DF90CF90CE
:10F64000BF90AF909F908F907F906F905F904F9002
:10F650003F902F9008952F923F924F925F926F921A
:10F660007F928F929F92AF92BF92CF92DF92EF9252
:10F67000FF920F931F93DF93CF9300D000D0CDB7AD
:10F68000DEB71C017A8369832B833C834D835E83C1
:10F6900027013801C801B70120E030E040E050E028
:10F6A0000F947D2B882321F080918A0A882351F0C2
:10F6B000F10111821082E981FA8110821182128295
:10F6C000138203C1F101808191818130910531F173
:10F6D0008230910509F446C0892B09F0D3C0C801D6
:10F6E000B70120E030E040E050E00F948B2D181679
:10F6F0000CF0C8C0F601EE0FFF1FEE0FFF1FE5571D
:10F70000F54F80E090E0A0E0B0E080839183A28399
:10F71000B383F601E851FC4E10822AC06B817C81D4
:10F720008D819E81A80197010F948B2D87FF07C0C3
:10F73000F601E851FC4E8081882309F4A3C0F6014C
:10F74000E851FC4E81E080830F94E725E981FA813E
:10F75000608371838283938382E090E0F1019183DF
:10F76000808390C0F601E851FC4E8081882319F413
:10F7700081E090E0F3CFB401882777FD8095982F42
:10F780000F941F2C9B01AC01C801B7010F94A32A51
:10F790009B01AC016B817C818D819E810F948B2DAF
:10F7A00088234CF00F94E725E981FA816083718307
:10F7B0008283938367C00F94E7257B018C01E981E5
:10F7C000FA8180819181A281B381E81AF90A0A0B3A
:10F7D0001B0BB501882777FD8095982F28EE33E025
:10F7E00040E050E00F942F2F6E157F0580079107A2
:10F7F00008F048C0ECEAFBE2949108C08091C00098
:10F8000085FFFCCF9093C600319694919923B1F770
:10F81000EAE3F0E2949108C08091C00085FFFCCF3C
:10F820009093C600319694919923B1F78091C000CE
:10F8300085FFFCCF8AE08093C60082E59BE0B6019D
:10F840004AE050E00E948E968091C00085FFFCCF78
:10F850008AE08093C6008AE290E20E94C76281E05B
:10F8600080938A0A0E94B873179A1092CB13169A43
:10F870001092CC13159A1092CD13149A0EDC0E949C
:10F88000DB62F0CFF601EE0FFF1FEE0FFF1FE55713
:10F89000F54F6081718182819381A30192010F9460
:10F8A0007D2B88232CF4FCD9F601E851FC4E108204
:10F8B000CC0CDD1CCC0CDD1C8BE89AE0C80ED91EEC
:10F8C000F601408251826282738226960FB6F894C6
:10F8D000DEBF0FBECDBFCF91DF911F910F91FF9083
:10F8E000EF90DF90CF90BF90AF909F908F907F90E0
:10F8F0006F905F904F903F902F9008952F923F927E
:10F900004F925F926F927F928F929F92AF92BF922F
:10F91000CF92DF92EF92FF920F931F93DF93CF93DB
:10F92000CDB7DEB7E3970FB6F894DEBF0FBECDBFFD
:10F930006C8F7D8F8E8F9F8F5BAB4AAB39A328A3D3
:10F940000F94E725698B7A8B8B8B9C8B2AA93BA91B
:10F95000121613061CF0E2E6F2E019C0E5E7F2E049
:10F9600007C08091C00085FFFCCF31969093C60000
:10F9700090819923B1F78091C00085FFFCCF31C4FD
:10F980008091C00085FFFCCF31969093C600908196
:10F990009923B1F78091C00085FFFCCF8AE0809366
:10F9A000C6000E94B8734AA95BA9452B09F468C038
:10F9B00087E68093640A17E6A12EB12CC12CD12CC6
:10F9C000B7E62B2E312C412C512C89899A89AB8991
:10F9D000BC898D879E87AF87B88B89879A87AB87CD
:10F9E000BC871EA61FA618AA19AA1F8A1E8A91E004
:10F9F0009D8B1D821E821F82188620E030E040E031
:10FA000050E029833A834B835C830F2EF0E06F2E06
:10FA1000F0E47F2EFCE18F2EF6E49F2EF02DEDEE2C
:10FA2000F2E234913AA3E8EEF2E244914BA3E1EE24
:10FA3000F2E254915CA3EAEDF2E284918DA3E4ED4D
:10FA4000F2E294919EA3EEECF2E2A491AFA3E0EC7B
:10FA5000F2E2B491B8A7EAEBF2E2249129A7E4EB31
:10FA6000F2E234913AA7EEEAF2E244914BA7E4E7DE
:10FA7000F2E254915CA7E8E7F2E284918DA70EC010
:10FA80008FE78093710AAFE7AA2EB12CC12CD12C3D
:10FA9000FFE72F2E312C412C512C97CF8091720AE9
:10FAA000882309F4C5C2D8DAAAA9BBA9AB2B69F08F
:10FAB000B091600ABEA7E091610AEFA7F091620AD7
:10FAC000F8AB2091630A29AB0CC030915A0A3EA7CB
:10FAD00040915B0A4FA750915C0A58AB80915D0A38
:10FAE00089AB69817A818B819C812EA53FA548A92C
:10FAF00059A90F948B2D181644F08EA59FA5A8A97F
:10FB0000B9A989839A83AB83BC83C401B3012EA5B1
:10FB10003FA548A959A90F947D2B87FD06C08EA546
:10FB20009FA5A8A9B9A93C014D019D89992309F474
:10FB300050C06EA57FA588A999A92C8D3D8D4E8DAD
:10FB40005F8D0F948B2D18160CF072C20F94E72561
:10FB500029853A854B855C85621B730B840B950B5D
:10FB6000695873418040904008F462C2D601C501D3
:10FB700082199309A409B5094AA95BA9452B39F053
:10FB8000B595A795979587958093640A06C0B59516
:10FB9000A795979587958093710A0F94E7256D87B0
:10FBA0007E878F87988BDC01CB0129853A854B8531
:10FBB0005C85821B930BA40BB50B8D839E83AF8357
:10FBC000B8878C8D9D8DAE8DBF8D89839A83AB83D5
:10FBD000BC836EA57FA588A999A92C8D3D8D4E8DDE
:10FBE0005F8D0F947D2B88230CF021C20F94E725A5
:10FBF0002D853E854F855889621B730B840B950BB1
:10FC0000695873418040904008F411C20F94E72571
:10FC100069877A878B879C874E895F89452B09F492
:10FC2000E3C1DC01CB012D853E854F855889821BC0
:10FC3000930BA40BB50B2D813E814F815885280F66
:10FC4000391F4A1F5B1F288F398F4A8F5B8F2D8189
:10FC50003E814F815885281B390B4A0B5B0BCA012B
:10FC6000B901A20191010F942F2F288D398D4A8D52
:10FC70005B8D0F94972FA20EB31EC41ED51E34E1C8
:10FC8000A316B104C104D10434F14AA95BA9452BE0
:10FC900029F48BEE90E0A0E0B0E004C08AEB90E0A5
:10FCA000A0E0B0E08A159B05AC05BD05CCF48AA99F
:10FCB0009BA9892B51F42EEF30E040E050E06BEE31
:10FCC000A62EB12CC12CD12C2DC04AEBA42EB12CC8
:10FCD000C12CD12C0EC034E1A32EB12CC12CD12CBF
:10FCE000AAA9BBA9AB2B29F48FE790E0A0E0B0E074
:10FCF00004C087E690E0A0E0B0E08A159B05AC0563
:10FD0000BD051CF01501260113C0EAA9FBA9EF2BC4
:10FD100029F42EEF30E040E050E004C02DEC30E05C
:10FD200040E050E019012A012A183B084C085D0800
:10FD30009AA1EDEEF2E208C08091C00085FFFCCFF1
:10FD40009093C600319694919923B1F782E59BE098
:10FD5000B601A5012AE030E00E945B969BA1E8EE87
:10FD6000F2E208C08091C00085FFFCCF9093C600EE
:10FD7000319694919923B1F782E59BE0B201A101FC
:10FD80002AE030E00E945B969CA1E1EEF2E208C01E
:10FD90008091C00085FFFCCF9093C600319694916E
:10FDA0009923B1F782E59BE0B401A30122E030E0A2
:10FDB0000E9461979DA1EAEDF2E208C08091C00027
:10FDC00085FFFCCF9093C600319694919923B1F7AB
:10FDD00082E59BE049815A816B817C8122E030E0A1
:10FDE0000E9461978091C00085FFFCCF8AE08093DC
:10FDF000C6002E893F89233031050CF4F5C0C201BD
:10FE0000B1010F941F2C20E030E040E850E40F9443
:10FE10005D2E7B018C0169817A818B819C81A4019B
:10FE200093010F94A32A20ED3FE049E450E40F949E
:10FE30005D2E20E030E040E05FE30F945D2E9B01FB
:10FE4000AC01C801B7010F94842B7B018C01688D34
:10FE5000798D8A8D9B8D0F941F2C20E030E04AE72E
:10FE600054E40F94842B3B014C019EA1E4EDF2E29B
:10FE700008C08091C00085FFFCCF9093C6003196EA
:10FE800094919923B1F782E59BE0B801A70122E0A4
:10FE900030E00E9461979FA1EEECF2E208C08091F1
:10FEA000C00085FFFCCF9093C600319694919923B2
:10FEB000B1F782E59BE0B401A30122E030E00E94AB
:10FEC00061978091C00085FFFCCF8AE08093C600D7
:10FED000C801B7012AE939E949E15FE30F945D2ED2
:10FEE0007B018C0198A5E0ECF2E208C08091C00093
:10FEF00085FFFCCF9093C600319694919923B1F77A
:10FF00008091C00085FFFCCF8AE08093C60099A550
:10FF1000EAEBF2E208C08091C00085FFFCCF90932D
:10FF2000C600319694919923B1F782E59BE0B80120
:10FF3000A70122E030E00E9461978091C00085FF18
:10FF4000FCCF8AE08093C6009AA5E4EBF2E208C0F9
:10FF50008091C00085FFFCCF9093C60031969491AC
:10FF60009923B1F7C801B701A80197010F94A42AFA
:10FF7000A40193010F94842BAB01BC0182E59BE0AB
:10FF800022E030E00E9461978091C00085FFFCCFA5
:10FF90008AE08093C6009BA5EEEAF2E208C0809159
:10FFA000C00085FFFCCF9093C600319694919923B1
:10FFB000B1F7C801B701A40193010F945D2E20E0B1
:10FFC00030E040E05EE30F945D2EAB01BC0182E5C2
:10FFD0009BE022E030E00E9461978091C00085FFA5
:10FFE000FCCF8AE08093C600D201C1018A0D9B1D1F
:10FFF000AC1DBD1D4AA95BA9452B39F0B595A79548
:020000021000EC
:10000000979587958093640A06C0B595A7959795AF
:1000100087958093710A8E899F8901969F8B8E8B1D
:100020006C8C7D8C8E8C9F8C91E09D8B01C01D8A89
:100030006C8D7D8D8E8D9F8D20E030E040EA51E407
:100040000F94A42A9B01AC016EA57FA588A999A94C
:100050000F948B2D18169CF4E4E8F2E2949108C0FA
:100060008091C00085FFFCCF9093C600319694919B
:100070009923B1F78091C00085FFFCCFB2C00F94E7
:10008000E72529893A894B895C89621B730B840BAC
:10009000950B615D77408040904008F453C04AA9B9
:1000A0005BA9452B89F06091640AEEE7F2E2949136
:1000B00008C08091C00085FFFCCF9093C6003196A8
:1000C00094919923B1F710C06091710A9DA5E8E75A
:1000D000F2E208C08091C00085FFFCCF9093C6007B
:1000E000319694919923B1F7162F82E59BE04EA5A6
:1000F0005FA568A979A922E030E00E9461979CA5DC
:10010000E4E7F2E208C08091C00085FFFCCF909345
:10011000C600319694919923B1F782E59BE0612F57
:1001200070E04AE050E00E948E968091C00085FF0A
:10013000FCCF8AE08093C6000F94E725698B7A8B09
:100140008B8B9C8B0F94E7257B018C010F94E7250B
:100150002D853E854F855889E21AF30A040B150B4D
:1001600029853A854B855C85E21AF30A040B150B49
:10017000E60EF71E081F191F31E8E3163FE4F306E9
:1001800032E1030730E0130798F0E7E5F2E29491DB
:1001900008C08091C00085FFFCCF9093C6003196C7
:1001A00094919923B1F78091C00085FFFCCF19C0CD
:1001B0004E895F8988A199A18417950774F5EBEFA3
:1001C000F1E2949108C08091C00085FFFCCF90932C
:1001D000C600319694919923B1F78091C00085FFB4
:1001E000FCCF8AE08093C600E3960FB6F894DEBF9A
:1001F0000FBECDBFCF91DF911F910F91FF90EF9078
:10020000DF90CF90BF90AF909F908F907F906F9036
:100210005F904F903F902F9008950E94DB623ECCFC
:100220002F923F924F925F926F927F928F929F9206
:10023000AF92BF92CF92DF92EF92FF920F931F93F4
:10024000DF93CF9300D000D0CDB7DEB71C017C8305
:100250006B836A01FA01E080F18002811381C80199
:10026000B70120E030E040E050E00F948B2D87FF95
:1002700004C017FB109517F91095C101880F991F3D
:10028000880F991F9A83898326016624772443C0A7
:10029000F401A080B180C280D380C601B50120E006
:1002A00030E040E050E00F948B2D88231CF0A60135
:1002B000950103C0A60195015058C801B7010F94DC
:1002C0007D2B88239CF4C601B50120E030E040E09E
:1002D00050E00F948B2D88231CF08601750106C019
:1002E0008601750117FB109517F910958D819E8178
:1002F00001969E838D83E4E0F0E08E0E9F1E8D813B
:100300009E818215930524F20894611C711CE98179
:10031000FA814E0E5F1E8B819C816816790624F44B
:1003200042011E821D82EBCFB701C80126960FB68F
:10033000F894DEBF0FBECDBFCF91DF911F910F911B
:10034000FF90EF90DF90CF90BF90AF909F908F90F5
:100350007F906F905F904F903F902F9008952F92D5
:100360003F924F925F926F927F928F929F92AF9245
:10037000BF92CF92DF92EF92FF920F931F93DF9382
:10038000CF93CDB7DEB72A970FB6F894DEBF0FBE76
:10039000CDBF98878F834A015B0139011816190672
:1003A0000CF063C1CB01BA0120E030E040E050E046
:1003B0000F947D2B882309F458C10130110529F4CD
:1003C00021E0C216D10419F460C017FD03C020E07B
:1003D00030E00DC081E090E04F815885841B950B83
:1003E000089F9001099F300D189F300D1124D7FCF4
:1003F00003C060E070E00DC081E090E0EF81F8851F
:100400008E1B9F0BC89EB001C99E700DD89E700DAB
:100410001124CC0CDD1CCC0CDD1C1B01220C331C6C
:10042000220C331C2E0C3F1C2801440C551C440C80
:10043000551C7901EE0CFF1CEE0CFF1CE60CF71CA2
:1004400000E010E0C501B401F70120813181428153
:1004500053810F945D2E9B01AC01F101608171818C
:10046000828193810F94A42AF10160837183828336
:1004700093830F5F1F4F2C0C3D1CE40CF51C2F8148
:10048000388502171307F4F2F0C00F811885037046
:10049000107067012301222433241CC0C501B4015C
:1004A000F20121913191419151912F010F945D2ED3
:1004B0009B01AC01F60160817181828193810F946F
:1004C000A42AF60161937193819391936F0108942B
:1004D000211C311C201631060CF3C801880F991F0E
:1004E000880F991F1701280E391E9301280F391FF5
:1004F0003E832D830F5F1F4FC801880F991F880F00
:10050000991F2701480E591EA301480F591F5C83EC
:100510004B830F5F1F4FC801880F991F880F991FCA
:100520006701C80ED91EF301E80FF91FFA83E983AA
:100530000F5F1F4FC801880F991F880F991F035025
:1005400010409701280F391F3A8729877301E80E59
:10055000F91E85C0C501B401ED81FE812081318184
:10056000428153810F945D2E9B01AC01F1016081AA
:100570007181828193810F94A42AF1016083718338
:1005800082839383C501B401EB81FC812081318199
:10059000428153810F945D2E9B01AC01F201608179
:1005A0007181828193810F94A42AF2016083718307
:1005B00082839383C501B401E981FA81208131816D
:1005C000428153810F945D2E9B01AC01F601608145
:1005D0007181828193810F94A42AF60160837183D3
:1005E00082839383C501B401F70120813181428167
:1005F00053810F945D2E9B01AC01E985FA856081E2
:100600007181828193810F94A42AE985FA856083A0
:100610007183828393830C5F1F4F20E130E0220EB1
:10062000331E4D815E81405F5F4F5E834D83420E7E
:10063000531E8B819C8140969C838B83C20ED31E5C
:10064000E981FA817096FA83E98329853A85205FEA
:100650003F4F3A87298740E150E0E40EF51E8F8135
:100660009885081719070CF475CF2A960FB6F894D9
:10067000DEBF0FBECDBFCF91DF911F910F91FF90D5
:10068000EF90DF90CF90BF90AF909F908F907F9032
:100690006F905F904F903F902F9008952F923F92D0
:1006A0004F925F926F927F928F929F92AF92BF9282
:1006B000CF92DF92EF92FF920F931F93DF93CF932E
:1006C000CDB7DEB72E970FB6F894DEBF0FBECDBF05
:1006D0009E878D874B013901F801181619065CF0C9
:1006E0000F2EF0E0CF2EF0E0DF2EF0E0EF2EF0E066
:1006F000FF2EF02D93C14130510521F40130110539
:1007000019F469C057FD03C060E070E00DC081E0DE
:1007100090E02D853E85821B930B489FB001499F39
:10072000700D589F700D1124F7FD03C020E030E0DC
:100730000DC081E090E0AD85BE858A1B9B0BE89FD4
:100740009001E99F300DF89F300D11242A01440CCF
:10075000551C440C551C8B01000F111F000F111F5D
:10076000080D191D4F01880C991C880C991C190142
:10077000220C331C220C331C260C371C0F2EF0E0ED
:10078000CF2EF0E0DF2EF0E0EF2EF0E0FF2EF02D88
:10079000AA24BB24F8016081718182819381D101F7
:1007A0002D913D914D915C910F945D2E9B01AC017B
:1007B000C701B6010F94A42A6B017C010894A11C07
:1007C000B11C040D151D280C391CED85FE85AE16D7
:1007D000BF0604F323C18D859E8565E070E00F940C
:1007E000622F8C010F2EF0E0CF2EF0E0DF2EF0E034
:1007F000EF2EF0E0FF2EF02DAA24BB244424552434
:100800001FC0F401E40DF51DD301A40DB51D6081D9
:100810007181828193812D913D914D915C910F94D5
:100820005D2E9B01AC01C701B6010F94A42A6B0198
:100830007C010894A11CB11C24E030E0420E531E40
:10084000A016B106F4F2C801880F991F880F991FEE
:10085000D401A80FB91FBC87AB87F301E80FF91FBC
:10086000FA87E9870F5F1F4FC801880F991F880F0C
:10087000991F9401280F391F38872F83D301A80FA0
:10088000B91FBE83AD830F5F1F4FC801880F991F2B
:10089000880F991FF401E80FF91FFC83EB83930184
:1008A000280F391F3A8329830F5F1F4FC801880F14
:1008B000991F880F991F1401280E391E2301480E15
:1008C000591E0F5F1F4FC801880F991F880F991F6E
:1008D00004501040880E991E5301A80EB91E38010D
:1008E00097C0AB85BC856D917D918D919C91E9857B
:1008F000FA8520813181428153810F945D2E9B01C5
:10090000AC01C701B6010F94A42A7B018C01AF8111
:10091000B8856D917D918D919C91ED81FE812081B5
:100920003181428153810F945D2E9B01AC01C8013E
:10093000B7010F94A42A7B018C01AB81BC816D911E
:100940007D918D919C91E981FA8120813181428153
:1009500053810F945D2E9B01AC01C801B7010F9428
:10096000A42A7B018C01D1016D917D918D919C9187
:10097000F20120813181428153810F945D2E9B01D0
:10098000AC01C801B7010F94A42A7B018C01D401EA
:100990006D917D918D919C91F501208131814281F4
:1009A00053810F945D2E9B01AC01C801B7010F94D8
:1009B000A42A6B017C0125E030E0620E731E8B855A
:1009C0009C8544969C878B87A985BA855496BA875F
:1009D000A987EF81F8857496F887EF832D813E8192
:1009E0002C5E3F4F3E832D838B819C8144969C835C
:1009F0008B83A981BA815496BA83A983E4E1F0E09C
:100A00002E0E3F1E4E0E5F1E8E0E9F1EAE0EBF1E82
:100A10002D853E85621673060CF463CFB601C701BF
:100A20002E960FB6F894DEBF0FBECDBFCF91DF91EB
:100A30001F910F91FF90EF90DF90CF90BF90AF90FC
:100A40009F908F907F906F905F904F903F902F90EE
:100A500008952F923F924F925F926F927F928F9262
:100A60009F92AF92BF92CF92DF92EF92FF920F933D
:100A70001F93DF93CF93CDB7DEB7EC970FB6F89403
:100A8000DEBF0FBECDBF9CA78BA77EA76DA758ABBF
:100A90004FA73AAB29AB1CAB0BAB37017601BEAA13
:100AA000ADAA98AE8FAA6896EEADFFAD689700E04C
:100AB00010E0CF01815F984D8F519E4410F001E00E
:100AC00010E0CF0160E177E20F94622F9AAF89AF17
:100AD000892B21F061E070E07AAF69AF1AA619A600
:100AE000CF0168EE73E00F94622F8D599F4F873CC2
:100AF000910520F081E090E09AA789A718A61FA28F
:100B0000CF0164E670E00F94622F0996439720F0BE
:100B1000A1E0B0E0B8A7AFA3CF016AE070E00F9406
:100B2000622F9CAF8BAF892B21F0E1E0F0E0FCAFAE
:100B3000EBAF8FA598A9019729A93AA93A832983F0
:100B40008217930714F49A83898369817A81672BCA
:100B500009F068C0012B51F0F30180819181A281DD
:100B6000B381F70180839183A283B38329AD3AAD2A
:100B7000232B59F0F30180819181A281B381EDA9EA
:100B8000FEA980839183A283B3832BAD3CAD232B3D
:100B900069F0F30180819181A281B3816696EEAD07
:100BA000FFAD669780839183A283B38329A53AA57D
:100BB000232B21F1ABA5BCA5ED90FD900D911C91CF
:100BC000C801B70120E030E040E050E00F947D2BF9
:100BD000882329F4E1E0F0E0FEA3EDA311C0D301E6
:100BE0006D917D918D919C91A80197010F94842B1B
:100BF000EFA9F8AD60837183828393831EA21DA247
:100C00002FA138A5232B09F4F9C380E090E0A0E0E0
:100C1000B0E06496EEADFFAD649780839183A283CC
:100C2000B383ECC301151105E9F061E070E040E029
:100C300050E013C09701240F351FF301E40FF51F97
:100C400080819181A281B381F90180839183A28304
:100C5000B3836F5F7F4F4C5F5F4F2FA538A9261777
:100C6000370744F769AD7AAD672BF1F061E070E0CA
:100C700040E050E014C02DA93EA9240F351FF30118
:100C8000E40FF51F80819181A281B381F9018083F6
:100C90009183A283B3836F5F7F4F4C5F5F4F2FA51C
:100CA00038A9261737073CF7012B09F4C7C021E004
:100CB00030E069817A81261B370BA901440F551F4B
:100CC000440F551F509541955F4F8BA99CA9840FE8
:100CD000951F9C8B8B8BADA5BEA5A095B095AA0F3B
:100CE000BB1FAA0FBB1FBA8BA98B615070408DA58B
:100CF0009EA50196689F2001699F500C789F500C1B
:100D00001124440C551C440C551CEBA5FCA54E0E9F
:100D10005F1EAFA5B8A91196B8ABAFA7E981FA815C
:100D2000AE1BBF0BB88BAF87AFA5B8A91197B8ABF7
:100D3000AFA7880F991F880F991FEE27FF27E81B81
:100D4000F90BFE87ED878DA59EA5689F3001699FF1
:100D5000700C789F700C1124621A730A660C771C51
:100D6000660C771CABA5BCA56A0E7B1E1701240E72
:100D7000351EE1E0F0E0FAA3E9A358C0AB89BC89D5
:100D8000ED90FD900D911C91C801B70120E030E07D
:100D900040E050E00F947D2B882361F1F2018080C8
:100DA0009180A280B380D201ED92FD920D931C93AD
:100DB00013978F859889B30141E050E0910101E0DC
:100DC00010E06CDC9058F201208131814281538126
:100DD0000F94842BAB01BC018F859889930171011D
:100DE000E1E0CE2ED12CBBDAD2018D929D92AD9254
:100DF000BC921397E9A1FAA13196FAA3E9A32B8932
:100E00003C89245030403C8B2B8B69897A89460E73
:100E1000571E8F8598890196988B8F87AD85BE85E3
:100E20006A0E7B1EECEFFFEF2E0E3F1E29A13AA1AA
:100E300069817A81621773070CF0A0CF89AD9AADF2
:100E4000892B09F489C0ADA5BEA51196BEA7ADA793
:100E5000AA0FBB1FAA0FBB1FBE8BAD8BEDA5FEA5B6
:100E60003197FEA7EDA72BA43CA44FA458A8CF010F
:100E700080959095880F991F880F991F22273327F7
:100E8000281B390B3C832B83310161E070E07CA38C
:100E90006BA3188E1F8A58C0EBA9FCA98F89988D67
:100EA000E80FF91FE080F18002811381C801B701CA
:100EB00020E030E040E050E00F947D2B882369F182
:100EC000D1018D909D90AD90BC90F101E082F182B6
:100ED00002831383EDA8FEA82F89388DE20EF31E3E
:100EE000C201B30141E050E0970101E010E0D6DB20
:100EF0009058D1012D913D914D915C910F94842B8F
:100F0000AB01BC01C2019301E1E0CE2ED12C27DA66
:100F1000F10180829182A282B3822BA13CA12F5F3A
:100F20003F4F3CA32BA36F89788D6C5F7F4F788FE9
:100F30006F8B8D899E89280E391E089441085108AF
:100F4000AB81BC816A0E7B1EEBA1FCA129813A8199
:100F50002E173F070CF0A0CF69A57AA5672BF9F0F3
:100F600061E070E040E050E015C02FA938AD240FDB
:100F7000351FEDA9FEA9E40FF51F80819181A281A3
:100F8000B381F90180839183A283B3836F5F7F4F25
:100F90004C5F5F4F29A93AA92617370734F76BAD85
:100FA0007CAD672B09F161E070E040E050E017C0D4
:100FB00066962EAD3FAD6697240F351FEDA9FEA9AD
:100FC000E40FF51F80819181A281B381F9018083B3
:100FD0009183A283B3836F5F7F4F4C5F5F4F29A9DB
:100FE0003AA92617370724F76FA178A5672B41F197
:100FF00089A99AA9AFA5B8A98A179B070CF59C01E6
:10100000880F991F880F991F4DA95EA9480F591F76
:101010006496EEADFFAD6497E80FF91F0AC0DA01E0
:10102000ED90FD900D911D91AD01E192F192019332
:1010300011932F5F3F4F6FA578A9621773077CF755
:101040008BAD9CAD892B11F1A9A9BAA9EFA5F8A97F
:10105000AE17BF07DCF4CD01FD01EE0FFF1FEE0F51
:10106000FF1F66962EAD3FAD6697E20FF31F20E09F
:1010700030E040E050E004C021933193419351931C
:1010800001966FA578A968177907B4F78FA198A57D
:10109000892BA9F06496EEADFFAD649781E090E0F6
:1010A00020E030E040E050E005C0219331934193CF
:1010B00051930196A9A9BAA9A817B907B4F7E9A548
:1010C000FAA5EF2B09F49EC069A87AA808946108D4
:1010D0007108660C771C660C771C2FA938AD620E60
:1010E000731E8DA59EA5880F991F880F991F6627CF
:1010F0007727681B790B7A8F698F89A99AA901973D
:10110000ADA5BEA58A9F40018B9F900C9A9F900C25
:101110001124880C991C880C991CEBA5FCA58E0E3B
:101120009F1EA095B095AA0FBB1FAA0FBB1FBE8321
:10113000AD832DA53EA52F5F3F4F829F5001839F1A
:10114000B00C929FB00C1124215030403EA72DA727
:10115000AA0CBB1CAA0CBB1CAE0EBF1E29A83AA829
:10116000F1E04F2E512C48C0C9A8DAA8C418D50800
:10117000D501ED90FD900D911C91C801B70120E0C3
:1011800030E040E050E00F947D2B882319F43EA21C
:101190002DA23AC0F3016081718182819381A801FF
:1011A00097010F94842BD3016D937D938D939C9322
:1011B0001397B1E02B16310469F0AB01BC017058F4
:1011C000C601940101E010E0EFA8F8ACE1E0CE2EFA
:1011D000D12CC5D80894411C511CECEFFFEF6E0ECA
:1011E0007F1E089421083108298D3A8D820E931EA6
:1011F0006D817E81A60EB71E89A99AA984159505D1
:101200000CF0B2CF1EA21DA2AFA1B8A5AB2B09F462
:1012100066C041E050E0E981FA814E1B5F0B9A0104
:10122000220F331F220F331F309521953F4F6BA99B
:101230007CA9620F731F78A36F8F8DA59EA58095E3
:101240009095880F991F880F991F9E8F8D8FBF01D2
:10125000615070408DA59EA50196689F3001699FE1
:10126000700C789F700C1124660C771C660C771C30
:10127000ABA5BCA56A0E7B1E8FA498A80894811C00
:10128000911C8E1A9F0A880F991F880F991FEE27AD
:10129000FF27E81BF90BFC8FEB8F8DA59EA5689FA0
:1012A0005001699FB00C789FB00C1124A41AB50AA4
:1012B000AA0CBB1CAA0CBB1CAA0EBB1E66962EACAD
:1012C0003FAC6697220E331E64964EAC5FAC6497BB
:1012D000420E531EA1E0B0E0BC87AB8787C0EBADE8
:1012E000FCADEF2B09F095CF89C0AF8DB8A1ED9083
:1012F000FD900D911C91C801B70120E030E040E065
:1013000050E00F947D2B882309F454C0D3016D91D4
:101310007D918D919C916F83788789879A87F3015E
:10132000E082F182028313832FA138A5232BD1F011
:10133000C401B50141E050E0920101E010E0AED9F6
:101340009058D3012D913D914D915C910F94842B38
:10135000AB01BC01C40195017201F1E0CF2ED12C8B
:101360000E94AF81EBADFCADEF2BD1F0C401B50114
:1013700041E050E0910101E010E090D99058D30194
:101380002D913D914D915C910F94842BAB01BC014B
:10139000C40195017101E1E0CE2ED12C0E94AF81F4
:1013A0006F81788589859A85D3016D937D938D931F
:1013B0009C931397EB85FC853196FC87EB872F8DEB
:1013C00038A12450304038A32F8F6D8D7E8D660E4E
:1013D000771E0894811C911C8B8D9C8DA80EB91EC4
:1013E000ACEFBFEF2A0E3B1E4A0E5B1EEB85FC8561
:1013F00029813A812E173F070CF077CF8DA19EA14E
:10140000EC960FB6F894DEBF0FBECDBFCF91DF9143
:101410001F910F91FF90EF90DF90CF90BF90AF9012
:101420009F908F907F906F905F904F903F902F9004
:1014300008952F923F924F925F926F927F928F9278
:101440009F92AF92BF92CF92DF92EF92FF920F9353
:101450001F93DF93CF9300D00F92CDB7DEB79C835D
:101460008B833A8329833801260114010115110564
:1014700009F100D000D0EDB7FEB73196ADB7BEB7D9
:101480001296BC92AE921197B382A2828EE690E041
:10149000958384838B819C8198010A8D1B8D6501C6
:1014A0004201D7DAEDB7FEB736960FB6F894FEBF15
:1014B0000FBEEDBF6101F10120E030E009C0808185
:1014C0009181909581959F4F819391932F5F3F4F8D
:1014D00089819A812817390794F3F301EE0FFF1FD2
:1014E000EE0FFF1FE40DF51D830180E090E0A0E00A
:1014F000B0E006C081939193A193B1930F5F1F4F0A
:1015000029813A8102171307ACF3720101E010E060
:10151000F1E0AF2EB12C46C0D6018D919C91119770
:1015200018161906ACF122273327281B390B2D93E7
:101530003C932BC0F7014081518162817381C501C9
:10154000821B930B9C01880F991F880F991FF20132
:10155000E81BF90B6080718082809380D7016D92C7
:101560007D928D929C921397408351836283738303
:10157000220F331FF101E21BF30B8081918122279F
:101580003327281B390B318320832017310791F62D
:101590000F5F1F4FE2E0F0E0CE0EDF1E24E030E0F0
:1015A000E20EF31E89819A81801791070CF0B4CF67
:1015B0000F900F900F900F90CF91DF911F910F918F
:1015C000FF90EF90DF90CF90BF90AF909F908F9063
:1015D0007F906F905F904F903F902F9008952F9243
:1015E0003F924F925F926F927F928F929F92AF92B3
:1015F000BF92CF92DF92EF92FF920F931F93DF93F0
:10160000CF9300D00F92CDB7DEB79A8389833A018A
:101610004B012901181619060CF0EAC0013011051A
:1016200009F0AFC065E070E00F94622F8C01790182
:10163000CC24DD2412C0F701608171818281938105
:10164000A40193010F945D2EF7016193719381932F
:1016500091937F010894C11CD11CC016D1065CF384
:101660001801220C331C220C331C240C351C58018D
:101670000894A11CB11CAA0CBB1CAA0CBB1CA40C7A
:10168000B51C42E0C42ED12CC00ED11ECC0CDD1CEA
:10169000CC0CDD1CC40CD51C23E0E22EF12CE00E9A
:1016A000F11EEE0CFF1CEE0CFF1CE40CF51C980167
:1016B0002C5F3F4F220F331F220F331F240D351D88
:1016C0003C832B8357C0F1016081718182819381BA
:1016D000A40193010F945D2EF101608371838283D5
:1016E0009383F5016081718182819381A4019301CB
:1016F0000F945D2EF5016083718382839383F601DD
:101700006081718182819381A40193010F945D2E88
:10171000F6016083718382839383F7016081718115
:1017200082819381A40193010F945D2EF701608360
:10173000718382839383EB81FC81608171818281DB
:101740009381A40193010F945D2EEB81FC81608352
:101750007183828393830B5F1F4F24E130E0220E5D
:10176000331EA20EB31EC20ED31EE20EF31E7496DB
:10177000FC83EB8389819A81081719070CF4A3CFA6
:1017800037C017FD03C060E070E00DC081E090E05D
:10179000E981FA818E1B9F0B089FB001099F700D94
:1017A000189F700D11247801EE0CFF1CEE0CFF1C2D
:1017B0006B01CC0CDD1CCC0CDD1CC40CD51C00E07A
:1017C00010E0F6016081718182819381A40193010F
:1017D0000F945D2EF60160837183828393830F5F84
:1017E0001F4FCE0CDF1C29813A81021713074CF3DF
:1017F0000F900F900F900F90CF91DF911F910F914D
:10180000FF90EF90DF90CF90BF90AF909F908F9020
:101810007F906F905F904F903F902F9008954F92E0
:101820005F926F927F928F929F92AF92BF92CF9270
:10183000DF92EF92FF920F931F93CF93DF932C01D0
:101840004B013901181619060CF0F2C04130510550
:1018500009F09CC00130110509F09AC063E070E006
:101860000F94622FBC018401E901E0E0F0E014C0B4
:10187000D8012D913D914D915C911397C880D980ED
:10188000EA80FB80CD92DD92ED92FD928D0129934D
:101890003993499359933196E617F7074CF3CB01E7
:1018A000880F991F880F991F5401A80EB91E630154
:1018B000C80ED91E6F5F7F4FCB01880F991F880F0D
:1018C000991F7401E80EF91E8301080F191F6F5F3D
:1018D0007F4FCB01880F991F880F991F625070406E
:1018E000E401C80FD91FF301E80FF91F4AC0D50161
:1018F0002D913D914D915C91D6016D907D908D9093
:101900009C90D5016D927D928D929C921397D601F9
:101910002D933D934D935C931397D7012D913D915A
:101920004D915C91D8016D907D908D909C90D701E8
:101930006D927D928D929C921397D8012D933D9339
:101940004D935C931397288139814A815B81808113
:101950009181A281B38188839983AA83BB832083E9
:101960003183428353836D5F7F4F8CE090E0A80EFC
:10197000B91EC80ED91EE80EF91E045F1F4F2C9623
:101980003C96641575050CF4B2CF52C057FD03C0E8
:1019900020E030E00BC081E090E084199509489F79
:1019A0009001499F300D589F300D112417FD03C041
:1019B00060E070E00BC081E090E084199509089F19
:1019C000B001099F700D189F700D11247A01EE0C63
:1019D000FF1CEE0CFF1CE901CC0FDD1FCC0FDD1F3F
:1019E000C80DD91D000F111F000F111FFB01EE0FB5
:1019F000FF1FEE0FFF1FE60DF71D60E070E028816E
:101A000039814A815B8180819181A281B381888300
:101A10009983AA83BB8320833183428353836F5F7F
:101A20007F4FCE0DDF1DE00FF11F641575053CF3F0
:101A3000DF91CF911F910F91FF90EF90DF90CF90AA
:101A4000BF90AF909F908F907F906F905F904F90DE
:101A500008952F923F924F925F926F927F928F9252
:101A60009F92AF92BF92CF92DF92EF92FF920F932D
:101A70001F93CF93DF937C015B014A016E9DC001F0
:101A80006F9D900D7E9D900D1124880F991F880FDA
:101A9000991F0E947224792E482F592F682E6701B2
:101AA000CC0CDD1CCC0CDD1CE0E0F0E060E070E074
:101AB00012C0D8012D903D904D905D908D012992DE
:101AC0003992499259922F5F3F4F2E153F058CF363
:101AD00031966C0D7D1DEA15FB054CF48401060F53
:101AE000171FEA01C60FD71F20E030E0EECFC30179
:101AF000DF91CF911F910F91FF90EF90DF90CF90EA
:101B0000BF90AF909F908F907F906F905F904F901D
:101B10003F902F9008952F923F924F925F926F9235
:101B20007F928F929F92AF92BF92CF92DF92EF926D
:101B3000FF920F931F93DF93CF9300D00F92CDB7F7
:101B4000DEB71C01FB01181619060CF0A8C014160C
:101B500015060CF0A4C081E02816310499F4E08049
:101B6000F18002811381C801B70120E030E040E03C
:101B700050E00F948B2D87FF9CC017FB109517F931
:101B8000109597C0DA01AA0FBB1FAA0FBB1FBA831B
:101B9000A9832B011C821B820F2EF0E0EF2EF0E0B8
:101BA000FF2EF0E00F2FF0E01F2FF02D0F2EF0E0B2
:101BB0006F2EF0E07F2EF0E88F2EFFE39F2EF02DAA
:101BC000F201A080B180C280D380C601B50120E0BF
:101BD00030E040E050E00F947D2B882309F445C0AD
:101BE000C601B50120E030E040E050E00F948B2DBD
:101BF00087FF04C0D7FAD094D7F8D094C801B701B2
:101C0000A60195010F947D2B8823ECF4C801B70140
